:020000040800F2
:10000000008001200919010889E4000895E400082E
:100010009DE40008A5E40008ADE40008000000002D
:100020000000000000000000000000008DF7020842
:10003000B5E400080000000065F80208C1E400080B
:100040004D1901084D1901084D1901084D190108F4
:100050004D1901084D1901084D1901084D190108E4
:100060004D190108CDE400084D1901084D1901088A
:100070004D1901084D1901084D1901084D190108C4
:100080004D1901084D1901084D1901084D190108B4
:100090004D1901084D1901084D1901084D190108A4
:1000A0004D1901084D1901084D1901084D19010894
:1000B0004D1901084D1901084D1901084D19010884
:1000C0004D1901084D1901084D1901084D19010874
:1000D0004D1901084D1901084D1901084D19010864
:1000E000F1E400084D1901084D1901084D190108E6
:1000F0004D1901084D1901084D1901084D19010844
:100100004D1901084D1901084D1901084D19010833
:100110004D1901084D1901084D1901084D19010823
:100120004D1901084D1901084D1901084D19010813
:100130004D19010815E500084D1901084D19010870
:100140004D1901084D1901084D1901084D190108F3
:10015000A5E500084D19010875E500084D190108CD
:100160004D1901084D1901084D1901084D190108D3
:100170004D1901084D1901084D1901084D190108C3
:040180004D1901080C
:1001880070B5051C0C1C101C002A03D00E22835EBF
:10019800013302D0002C14D11CE0828982239B00F9
:1001A8001A42F7D00668002909D0311C221C2B7886
:1001B8000B7001310135013A002AF8D13619066071
:1001C80008E028780135000600160CF083FF013C92
:1001D800002CF6D170BC01BC0047000030B581B0DE
:1001E800041C02F095FA051C201C291C0022FFF7AC
:1001F800C7FF0A200CF06EFF281C01B030BC02BCFF
:100208000847C0460EB400B598B019AB04CB199294
:100218006946822292008A8100900490094A0292DB
:10022800059201225242CA811793074A1068199A07
:1002380000F00CF8009A0023137018B008BC03B043
:1002480018470000FFFFFF7FA4000020F0B55F46BD
:1002580056464D464446F0B4AFB002908A461E1C3E
:10026800904600220492089200E0099E42461378C4
:10027800002B09D0252B07D0444601342378002BC6
:1002880003D0252B01D0F8E744464346E51A002D54
:1002980007D04046291C5246FFF772FF049A5219AC
:1002A80004920023E356002B00D1FEE20134A0465D
:1002B80000226B46B7331A700392059201235B4202
:1002C800069300E01E1C4246127812061216934648
:1002D8000123984400E005915B46203B582B00D948
:1002E80030E29B00C74A9B589F46C74A08928FE155
:1002F8006A46B7320023D356002BE4D1202313706B
:10030800E1E70123039A1A430392DCE7331D3668B9
:100318000596002ED6DA724205921E1C0423039A13
:100328001A430392CFE72B226B46B7331A70CAE7FA
:1003380042461378012290441B061B162A2B06D02E
:100348009B461A1C303A092A0DD900211AE0331DA0
:1003580036680696002E04DA1E1C01235B420693BB
:10036800B1E71E1CAFE700218B005B185B009918F2
:100378004246127812061216934601239844303AE0
:10038800092AF1D900290691A6DA012252420692D9
:10039800A2E78023039A1A43039294E700215B465D
:1003A800303B8A0052185200991843461B781B06A6
:1003B8001B169B4601229044303B092B8BD8EEE755
:1003C8004023039A1A4303927DE742460023D356FB
:1003D8006C2B06D1012398441023039A1A430392E5
:1003E80071E71023039A1A4303926CE71023039AC8
:1003F8001A43039267E75B46432B02D0039AD2065F
:1004080010D500230C930D933268029869463F314A
:100418000CAB05F0D9F8071C431C00D145E20436A3
:10042800099606E0321D099232686B463F331A700E
:10043800012700226B46B7331A703F236B44994655
:100448002DE21023039A1A430392039BDB0603D57C
:10045800321D099234680BE0039B5B0605D5321DFB
:10046800099233681B041C1402E0331D0993346895
:10047800002C01DB0121ECE064422D226B46B733EE
:100488001A700121E5E0039AD20605D5331D0993B8
:100498003368049A1A60E8E6039B5B0606D5321DAA
:1004A800099233686A46128A1A80DEE6331D099378
:1004B8003368049A1A60D8E61023039A1A43039201
:1004C800039BDB0603D5321D0992346809E0039BC0
:1004D8005B0603D5321D0992348802E0331D099367
:1004E80034680021B1E0321D099234680223039A6E
:1004F8001A43039278239B460221434A0892A4E0B8
:10050800069C00226B46B7331A70331D0993366870
:10051800B146002E00D1BFE15A46532A02D0039BB0
:10052800DB0643D54D460E9500230A930B93002C0A
:1005380018DB002700250E9B5A59002A1FD0029865
:1005480069463F310AAB05F03FF8421C00D1ACE1E7
:10055800C019A04213DC0435844201D1271C0EE0E7
:10056800071CE8E70AAB0093029800210EAA0023B3
:1005780005F092F8071C431C00D196E10E95002F58
:1005880000D1EEE000250A950B956C4667340AAB5E
:1005980000930298211C0EAA3B1C05F07DF88742A7
:1005A80000D082E1E555A1460795E0E0002C0CDB80
:1005B800301C0021221C01F071F8002800D1D3E082
:1005C800871BA74200DDCFE0CBE0301C02F0A0F88B
:1005D800071C64E11023039A1A430392039BDB066A
:1005E80003D5321D0992346809E0039B5B0603D5E5
:1005F800321D0992348802E0331D099334680121C1
:1006080023E0000008290308D4420308AC4A0892F2
:10061800039BDB0603D5321D0992346809E0039B6E
:100628005B0603D5321D0992348802E0331D099315
:100638003468039AD20707D5002C05D00223039A01
:100648001A430392022100E0022100226B46B733CD
:100658001A70069B002B03DB8023039A9A430392AC
:10066800002C02D1069B002B50D0012909D001296A
:100678000CD302293AD0069A0792924B9946192729
:1006880075E0092C1CD86D46673529E067226A4455
:10069800914601235B4299440723234030334A465D
:1006A8001370E408002CF4D1039AD20743D5302BF9
:1006B80041D001235B42994430234A4613703AE003
:1006C8006D466735013D201C0A210AF073FE303162
:1006D8002970201C0A210AF03FFD041C0928F1D8C2
:1006E800013DA946231C30332B7024E067236B445B
:1006F80099460122524291440F232340089A9B5C59
:100708004A4613702409002C15D0F2E7002903D0BB
:1007180067236B4499460EE0039AD20703D46723F4
:100728006B44994607E030216A463F322723D1546B
:1007380066226A4491466B4667334A469F1A069B6F
:10074800079314E05A46002A00D1AEE069463F31CB
:100758000A7000226B46B7331A700996894601273A
:100768009DE00023079302E0069F002207923E1CAB
:10077800079B9F4200DA1E1C6B46B7331B781B068B
:100788001B16002B01D0013603E0039A920700D50F
:1007980002368423039D1D4012D1059B9C1B002C0F
:1007A8000EDD102C07DD484810215246FFF7E8FC03
:1007B800103C102CF7DC4448211C5246FFF7E0FCA3
:1007C8006846B7300023C356002B04D00121524697
:1007D800FFF7D6FC0CE0039A920709D568463D302E
:1007E800302303705B46437002215246FFF7C8FC72
:1007F800802D16D1059A941B002C12DD102C0ADDD1
:10080800314B1D1C1035281C10215246FFF7B8FC2F
:10081800103C102CF7DC2C481030211C5246FFF7F6
:10082800AFFC079BDC1B002C12DD102C0ADD264BCD
:100838001D1C1035281C10215246FFF7A1FC103C46
:10084800102CF7DC20481030211C5246FFF798FC8A
:100858004846391C5246FFF793FC039A520712D5B3
:10086800059B9C1B002C0EDD102C07DD1648102163
:100878005246FFF785FC103C102CF7DC1248211C6F
:100888005246FFF77DFC331C059A964200DA131C8A
:10089800049AD2180492E8E40C4B994606273E1EA7
:1008A80000DA0026002207926FE704982FB03CBCBC
:1008B80090469946A246AB46F0BC02BC08470000E9
:1008C800E8420308FC4203086C2A0308184303089B
:1008D80030B581B0041C0D1C131C054A1068211C7E
:1008E8002A1CFFF7B3FC01B030BC02BC084700006B
:1008F800A400002000210A2202F002BB00220A23E1
:1009080002F04CBA40F2A403C2F200031868704720
:1009180070B50C4605460E46002948D000F040FA4E
:1009280015B1AB69002B44D042F68C23C0F6030303
:100938009C4208BF6C680ED042F6AC23C0F6030395
:100948009C4208BFAC6806D042F6CC23C0F603032D
:100958009C4208BFEC68B4F90C6036B328462146BF
:1009680000F038F8236B06463BB12846216A9847C1
:1009780036EA200628BF4FF0FF36A38913F0800F10
:100988001BD1616B41B104F14403994202D028465E
:1009980000F07AFA00236363A16C21B1284600F0C5
:1009A80073FA0023A3640023A38100F0FBF9304607
:1009B80070BD284600F02CF9B6E72846216900F0FA
:1009C80063FADEE740F2A4030146C2F200031868A6
:1009D8009EE700BF2DE9F0410C460E698046002EC7
:1009E8004AD018B18369002B00F08E8042F68C2320
:1009F800C0F603039C4208BFD8F8044010D042F662
:100A0800AC23C0F603039C4208BFD8F8084007D0BF
:100A180042F6CC23C0F603039C4208BFD8F80C402A
:100A2800A689002E28D033B213F0080027D02669F3
:100A380016B313F0030F2568266008BF6369C6EB79
:100A4800050518BF0023002DA36002DC9AE0002DE5
:100A580074DD32462B46A76A4046216AB84700280B
:100A6800C0EB05050644F2DCA3894FF0FF3043F0E4
:100A78004003A381BDE8F0813046BDE8F08162689B
:100A880046F40063A381002A5BDDE66A002EF3D0FA
:100A98009BB2002213F48057D8F80050C8F8002001
:100AA80018BF626D33D013F0040F05D06168636B13
:100AB800521A0BB1236CD21A00234046216AB04760
:100AC800B0F1FF3F2FD0A3890021226923F40063EE
:100AD80061601B0422601B0CA38113F4805F03D0A8
:100AE800B0F1FF3F31D06065616BC8F80050002954
:100AF80031D004F14403994202D0404600F0C4F9D1
:100B080000206063BDE8F08100F082F86EE73A46A5
:100B180001234046216AB047B0F1FF3F02461DD08D
:100B2800A389E66ABFE7D8F800301D2B9CD84FF49C
:100B38000172C8F200029A40C5D495E70020BDE8CA
:100B4800F081226C002AA0DCF9E7D8F80030002BED
:100B5800CAD16065C8E70846BDE8F081D8F800301A
:100B6800002BDDD0A3F11D02514241EB0201162BEF
:100B780014BF0B4641F001033BB1C8F8005038469A
:100B8800BDE8F0810020BDE8F081A38943F040036F
:100B9800A381BDE8F08100BF30B140F2A403014653
:100BA800C2F20003186815E742F6EC2340F6DD119F
:100BB800C0F60303C0F60001186800F05BBA00BF76
:100BC800002070470020704740F6CD11C0F60001A4
:100BD80000F026BA70B568250E4605FB01F505F14B
:100BE8000C0100F09DFA044648B100F10C03002105
:100BF80046602A4618462160A36000F0C9FE2046D8
:100C080070BD00BF42F6EC23C0F603031868DBE7AB
:100C18002DE9F04F0546846983B0002C78D140F661
:100C2800D1320123C0F600028361826242F299291F
:100C3800C0F8D84042F2C128C0F8DC4042F2FD2A90
:100C4800C0F8E04042F2253B019300F065F8C0F699
:100C58000009C0F60008C0F6000AC0F6000B68607C
:100C6800284600F059F8A860284600F055F86F6843
:100C780021460822E86004203C60B88107F15C0046
:100C88007C60BC607C66FC813C617C61BC6100F07E
:100C98007FFEAE68019B2146082209203F62B08191
:100CA80006F15C00F381C7F82490C7F82880C7F8DC
:100CB8002CA0C7F830B034607460B46074663461D6
:100CC8007461B46100F064FEED681223022036629C
:100CD8002146E8810822C6F8249005F15C00AB8122
:100CE800C6F82880C6F82CA0C6F830B02C606C6016
:100CF800AC606C662C616C61AC6100F049FE2D62E1
:100D0800C5F82490C5F82880C5F82CA0C5F830B0DF
:100D180003B0BDE8F08F00BF42F6EC23C0F6030332
:100D280070B506461D68AB69002B29D0D8356B68AD
:100D3800AC68013B03D51FE06834013B1CD3B4F910
:100D48000C20002AF8D100254FF0FF33656604F126
:100D58005C00E381294601232560A3810822A56060
:100D6800656025616561A56100F012FE6563A56394
:100D7800A564E564204670BD286828B10546D6E715
:100D88002846FFF745FFD1E730460421FFF722FF49
:100D980028600028F2D10C2304463360EAE700BF3C
:100DA800704700BF704700BF704700BF704700BF63
:100DB80040F2A40340F6C931C2F20003C0F60001B4
:100DC800186800F02DB900BF40F2A40340F6CD31F9
:100DD800C2F20003C0F60001186800F021B900BF94
:100DE800F8B540F29814C2F200040F46054601F027
:100DF800B3F8A3685E6826F0030606F57E630F3332
:100E0800DF1B3F0B013F3F03B7F5805F07DB002186
:100E1800284601F0A5F8A3689B19984204D02846F3
:100E280001F09CF80020F8BD7942284601F098F8B6
:100E3800B0F1FF3F10D043F2A423A168C2F200032F
:100E4800F61B284646F001061A684E60D71B1F603D
:100E580001F084F80120F8BD0021284601F080F84F
:100E6800A368C21A0F2ADADD40F2A05443F2A42183
:100E7800C2F20004C2F2000142F001025A60236883
:100E8800C01A0860CBE700BF2DE9F0410D460446C3
:100E9800002958D001F060F8A5F1080240F2981036
:100EA8005668C2F2000026F00103D0F808C0D11835
:100EB8008C454F6827F0030765D016F001064F6090
:100EC80031D00026CD196D6815F0010F06D1DB1958
:100ED800002E4BD08D68C968E9608D6043F0010130
:100EE800D3505160D6B9B3F5007F2ED3590A0429DF
:100EF8006BD89E093836F5004519A968A94203D16F
:100F080069E089688D4204D0486820F00300834274
:100F1800F7D3CB68D3609160CA609A602046BDE879
:100F2800F04101F01BB855F8085C00F1080C521BA1
:100F38005B199568654546D0D2F80CC0C5F80CC059
:100F4800CCF80850BEE7BDE8F081DB08012546680B
:100F580000EBC3019B1015FA03F3D1608D6846EAD4
:100F6800030343609560EA608A60D7E78D682B4F7A
:100F7800BD42B0D1EA6043F00101AA60D560956036
:100F88005160D350CAE716F0010F3B4407D155F81A
:100F9800081C521A5B189568D168E9608D6040F2A8
:100FA800A45143F00105C2F20001556082600A684D
:100FB8009342B3D343F2A0232046C2F20003196838
:100FC800FFF70EFFAAE701267CE714290CD801F1E8
:100FD8005B06F50090E701254768B6100B46B5405B
:100FE80047EA0505456095E7542903D81E0B6E3678
:100FF800F50081E7B1F5AA7F03D8DE0B7736F50057
:101008007AE740F25455A94203D89E0C7C36F50085
:1010180072E74FF47C757E266EE700BFA0010020C2
:101028002DE9F84307468946FFF7BAFED83708BFC7
:10103800B8461AD04FF000087E68BC68002E11DD53
:101048000025B4F90C30013543B1B4F90E3020460F
:10105800B3F1FF3F02D0C84748EA0008B54204F19F
:101068006804EED13F68002FE6D1FFF79BFE4046AB
:10107800BDE8F8832DE9F04780468A46FFF790FEE1
:1010880018F1D80708BFB9461BD04FF000097E6891
:10109800BC68002E12DD0025B4F90C3001354BB1C7
:1010A800B4F90E3021464046B3F1FF3F02D0D04795
:1010B80049EA0009B54204F16804EDD13F68002F00
:1010C800E5D1FFF76FFE4846BDE8F08770B540F2FE
:1010D800A404C2F2000406462568E96B21B1304633
:1010E800BDE8704000F008B8242000F009F8236833
:1010F800E863D96BF3E700BF002200F065BD00BFCD
:1011080040F2A4030146C2F20003186800F008B8D0
:1011180040F2A4030146C2F200031868FFF7B4BE08
:101128002DE9F04F01F10B04162C83B0064631D996
:1011380024F00704E30F8C422CBF194643F0010149
:10114800002930D1304600F007FFB4F5FC7F2FD2DC
:101158004FEAD40C40F29815C2F2000505EBCC0218
:101168002F46D368934200F02D825C6803F108088B
:10117800DA68304624F0030499681B195C68CA6071
:1011880044F0010491605C6000F0E8FE404603B062
:10119800BDE8F08F002310248C422CBF194643F081
:1011A80001010029CED00C234FF000083360EDE791
:1011B8005FEA542C04BF4FEAD40C4FEACC0040F04D
:1011C800868040F29815C2F2000528182F46C36899
:1011D800984206D10DE0002980F27981DB689842B7
:1011E80007D05A6822F00302111B0F29F3DD0CF116
:1011F800FF3C0CF1010CBD4A93689A4208BF78681D
:1012080024D0586820F00300011B0F2900F3C08187
:101218000029D260926080F29480B0F5007F80F05F
:101228007781C0084FF0010ED7F8048007EBC001A2
:1012380080100EFA00F0D960D1F808E040EA080002
:101248007860C3F808E0CEF80C308B604FF0010EE0
:101258004FEAAC030EFA03FE86457DD810EA0E0F5E
:1012680008D12CF0030C4FEA4E0E0CF1040C10EAD6
:101278000E0FF8D007EBCC0AE146D046D8F80C00A0
:10128800804507D196E1002B80F2A681C068804591
:1012980000F09081416821F003010B1B0F2BF2DD58
:1012A8008046C568011944F0010E58F8087F43F0DC
:1012B8000104C0F804E030464C60FD60AF60D160C6
:1012C8009160CA608A60CB5000F048FE5EE7BCF1CE
:1012D800040F9EBF4FEA941C0CF1380C4FEACC0067
:1012E8007FF66FAFBCF1140F9CBF0CF15B0C4FEA9B
:1012F800CC007FF666AFBCF1540F9EBF4FEA143C9A
:101308000CF16E0C4FEACC007FF65BAFBCF5AA7F00
:101318009EBF4FEAD43C0CF1770C4FEACC007FF625
:1013280050AF40F254539C4595BF4FEA944C4FF44C
:101338007C700CF17C0C4FF07E0C98BF4FEACC000F
:101348003FE71A1803F108083046536843F00103D1
:10135800536000F003FE19E7D7F80880D8F8043086
:1013680023F003094C45C4EB090294BF0023012371
:101378000F2AD8BF43F00103002B00F0B98043F2D5
:10138800A02AD5F80834C2F2000A3046B3F1FF3F6C
:10139800DAF8002002F1100BA3441FBF0BF57E6B97
:1013A8000BF11F0B2BF47E6B2BF01F0B594600F033
:1013B800D7FDB0F1FF3F034600F0188108EB0901A3
:1013C800814200F21081DAF8042081425A44CAF8B6
:1013D800042000F03E81D5F808E440F29815C2F2E6
:1013E8000005BEF1FF3F17BF8218C5F80804C1EB1E
:1013F8000201CAF8041010F0070517BFC5F1080567
:101408004FF48055431905F5805503EB0B02304620
:1014180001931205120DAD1A294600F0A1FD019B9A
:10142800B0F1FF3F00F02C81C11A491941F00101C8
:10143800DAF80420B84543F2A02BBB602A44C2F274
:10144800000B5960CAF8042017D0B9F10F0F40F209
:10145800E180A9F10C03D8F8045023F00703052014
:1014680008EB03010F2B05F0010543EA0505C8F851
:1014780004504860886000F2FB80DAF82C1043F2D0
:10148800A023C2F200038A42DAF8301088BFDA6279
:1014980043F2A0238A42C2F2000340F2A780D7F8A1
:1014A80008801A63D8F8043023F003039C42C4EB85
:1014B800030294BF002301230F2AD8BF43F001037E
:1014C800B3B130464FF0000800F048FD5EE69A18C8
:1014D800D9689C6803F108085568304645F001034F
:1014E800E1608C60536000F039FD4FE6A0010020F8
:1014F80008EB040342F0010244F001043046C8F846
:10150800044008F108085A60BB6000F027FD3DE67A
:10151800410A04299CBF4FEA901E0EF1380E1DD9CE
:10152800142998BF01F15B0E18D954299CBF4FEAC2
:10153800103E0EF16E0E11D9B1F5AA7F9CBF4FEA8D
:10154800D03E0EF1770E09D940F2545E714596BF30
:101558004FEA904E4FF07E0E0EF17C0E07EBCE0850
:10156800D8F80810414503D147E08968884505D077
:10157800D1F804E02EF0030E7045F6D3D1F80CE054
:10158800C3F80CE099607868CB60CEF808305DE667
:101598001D1941F00107D56044F0010495603046FB
:1015A8005C6003F10808EA60AA606F60695000F0A7
:1015B800D5FCEBE509F1010919F0030F2FD008F16B
:1015C80008085BE603F108025B699A4208BF0CF160
:1015D800020C3FF410AEC8E580464318C268304696
:1015E80058F8081FCAE5B8453FF4EDAED7F80880AB
:1015F800D8F8043023F0030358E74FF00109D7F86F
:1016080004804FEAAE008E4609FA00F048EA00006E
:101618007860B5E7984601225A60002346E75146AC
:101628001CF0030F0B460CF1FF3C2CD053F80819A3
:101638009942F5D07B684FEA4E0E9E453FF68CAE38
:10164800BEF1000F3FF488AE1EEA030F20D0CC464F
:1016580010E64FEA015E4FEA1E5EBEF1000F7FF40E
:10166800BAAEBB680BEB090141F00101596004E710
:10167800304608F10801FFF707FCDBF80420FCE618
:1016880001210025D4E67B6823EA0E037B60D1E7BD
:101698004FEA4E0E09F10409D6E700BF10F0030F18
:1016A800034670B4C9B211D0002A22D003788B4205
:1016B8001DD0013A013005E0DAB110F8014B013ACA
:1016C8008C4218D010F0030F0346F5D1032A14D822
:1016D8007AB1187888420ED0541E5D1C03E015F8C4
:1016E800016B8E4203D0013C2846F8D2002070BC22
:1016F80070471046FBE71846F9E741EA012646EA33
:101708000646184653F8044B86EA0404A4F101354A
:1017180025EA040414F0803F03D1043A1846032A4A
:10172800EFD80346D4E700BF032A70B404460D4639
:1017380026D941EA000313F0030F13D020782B7841
:10174800984208BF294606D01EE014F8010F11F888
:10175800013F984218D1012A02F1FF32F5D1002049
:1017680070BC70470B46044651F8045B50F8046B94
:10177800AE4204D1043A0446032A0B46F2D81D4669
:101788001046002ADAD1EBE7C01AE9E7032A2DE967
:10179800F00109D82AB10023CC5CC4540133934228
:1017A800FAD1BDE8F00170470B468218014603E004
:1017B8002478013301F8014B11F0030F1C46F7D1CF
:1017C80013F003055DD06E42C5F1040CED009B5982
:1017D8004FEACC0C08E00434A7593B4607FA0CF74B
:1017E80048EA070741F8047B571A23FA05F8032F3C
:1017F800F1DC03E014F8013B01F8013B8A42F9D817
:10180800CFE753F8404C41F8404C53F83C4C41F872
:101818003C4C53F8384C41F8384C53F8344C41F8A8
:10182800344C53F8304C41F8304C53F82C4C41F8B8
:101838002C4C53F8284C41F8284C53F8244C41F8C8
:10184800244C53F8204C41F8204C53F81C4C41F8D8
:101858001C4C53F8184C41F8184C53F8144C41F8E8
:10186800144C53F8104C41F8104C53F80C4C41F8F8
:101878000C4C53F8084C41F8084C53F8044C41F808
:10188800044C561A1D460C46403340313F2EB8DCF6
:101898002B460FE053F8101C44F8101C53F80C1C8E
:1018A80044F80C1C53F8081C44F8081C53F8041C92
:1018B80044F8041C161B21461D46103410330F2E05
:1018C800E8DC2B4602E0246841F8044B551A1C4614
:1018D800032D03F10403F6DC90E700BF88420346BA
:1018E800F0B40C460ED98D18A8420BD242B1831819
:1018F80029469A1A11F8014D03F8014D9342F9D17E
:10190800F0BC70470F2A38D941EA000515F0030FDB
:1019180035D1A2F1100601F110050B460246370930
:1019280005EB07151C6814605C6854609C6894603B
:10193800DC681033D46010329D42F3D17C1C06F071
:101948000F022401032A00EB0403214414D9043AAA
:101958000C461D464FEA920C01EB8C07043754F8ED
:10196800046BBC4245F8046BF9D10CF1010402F098
:101978000302A4001B1909190C46002AC0D02146ED
:10198800A21811F8014B914203F8014BF9D1B7E7BE
:10199800032AC9B270B408D82AB10346121803F84A
:1019A800011B9342FBD170BC70478218044601E0CA
:1019B80004F8011B14F0030FFAD14FF0013303FBB5
:1019C80001F31FE044F8403C44F83C3C44F8383C00
:1019D80044F8343C44F8303C44F82C3C44F8283C67
:1019E80044F8243C44F8203C44F81C3C44F8183C97
:1019F80044F8143C44F8103C44F80C3C44F8083CC7
:101A080044F8043C161B254640343F2EDADC2C46AD
:101A180007E044F8103C44F80C3C44F8083C44F80F
:101A2800043C161B254610340F2EF2DC01E045F865
:101A3800043B541B032CFADC01E005F8011B95421A
:101A4800FBD3B0E72DE9F04F85B0044604F09EFEC5
:101A580040F2B1739C42844640F39880A4F5F66244
:101A680048F21F51C5F2EB1102F1430002F5B673BB
:101A7800561E81FB0057033381FB0458C01781FBB6
:101A88000351A0EB6710E51700EBA606023AC5EB79
:101A98006810C5EBE81840F26D15DB1742F6F0291F
:101AA80005FB02624FF4C875C3EBE113642105FB23
:101AB800184842F2934B01FB10404FF4A34AB8F187
:101AC800000F0CBF3021002165460027C0F603092E
:101AD800CDF80C80C9F2492BC0F2010A8046D31810
:101AE800029104F0030200930192CCF804402B7A8F
:101AF8004A2B4DD0442B5FD0019A002A41D0029E38
:101B0800EC684E44012C5BDD009A31460123013319
:101B180051F8040BA3420244F9D1013B9C00131D68
:101B28008BFB0310D917C018C1EBA0013059C1EBCA
:101B3800C101591A6B69591A2B6948BF0731013B12
:101B4800C3EBC303CB18834202DB073B8342FCDAB7
:101B58009B18296A0137AA69022F0A440AFB032243
:101B680045F81C2FC3D1DCF838300120DCF81C20E4
:101B78009A42ACBF00230123CCF8003005B0BDE881
:101B8800F08FB8F1000FBAD03026B9E70020F5E79A
:101B9800009A69695318019A42B9B8F1000F05D043
:101BA8003B29D4BF00210121CB18D2E7039A002A90
:101BB800F6D00021CB18CCE76B690099CB18C8E7A1
:101BC800009A0024ABE700BF2DE9F84F05460C4604
:101BD800164604F0DBFD2A684FF4A341C0F2010168
:101BE800D717834644F20750CCF22E2080FB02839D
:101BF8009B18C7EB234301FB1322002A05DA02F5E1
:101C0800A832013B12F5C072F9D44BF2C5314FEA44
:101C1800E279C9F2A21142F29348181DC9F2492883
:101C280081FB02A148F6890788FB00A88918C8F635
:101C380088074FEAE07CC9EBE1214FF46169A160B4
:101C480009FB112208EB0001CCEBA101C1EBC1019A
:101C580087FB02C7411A4FEAE27C002907EB020022
:101C6800A161CCEB60106060C0EB0010A2EB8002B9
:101C78002260C0F2A680002B75DB42F6F02C48F2F9
:101C88001F5040F2B277C0F6030CC5F2EB104FF4C8
:101C9800C8794FF0640A01E001379B1A80FB0728D6
:101CA800FA1717F0030F07D1C2EB681801210AFBD6
:101CB8001878B8F1000F09D180FB0781C2EBE11158
:101CC80009FB1171D1F1010138BF00210CEB810230
:101CD800126E9342E0DA4A00A7F5EC6052180C380D
:101CE8000021E3611201606121610CEB02085CF8DC
:101CF8000220934207DB40469B1A0131216150F8CC
:101D0800042F9A42F8DD0133E36026B10023204610
:101D18002362BDE8F88F03F015FC43F2D423C2F226
:101D280000031B68002B4FD0DBF80430BB4205D002
:101D38003846FFF787FE002800F0DD80DBF800302A
:101D4800002B00F0C5802B68DBF81C209342C0F202
:101D5800DF80DBF83820934280F2DA800123DBF859
:101D68003C10236233E042F6F02C48F21F5040F258
:101D7800B277C0F6030CC5F2EB104FF4C8794FF0F8
:101D8800640A013F17F0030F80FB07284FEAE77248
:101D980007D1C2EB681801210AFB1878B8F1000FC7
:101DA80009D180FB0781C2EBE11109FB1171D1F167
:101DB800010138BF00210CEB8102126E9B18E0D4A0
:101DC80089E70731A16156E72662DBF820104BF25C
:101DD800C532CD17C9F2A212D4F808E048F6890036
:101DE800276882FB01A6C8F6880062687618F61292
:101DF800731B4FF46166C3EB0E05A56006FB131356
:101E080080FB03C1DE17C918C6EB6111521A626064
:101E1800C1EB0111A3EB8103FB1A23603B2B2BDDE4
:101E280001323C3B626023603B2A48DD6B1C3C3A34
:101E3800A3606260172B26DDA269E1690132A26105
:101E48000131062AE16101DD0022A2612169A3F1C5
:101E58001802E368A2600133E36058F82120934236
:101E680005DD01319B1A0C292161E36047D003F09D
:101E78006BFB2046BDE8F88F002BD5DA013A3C33DE
:101E880062602360D0E7002BF1DAA269E169013AC8
:101E9800A2610139002AE1613DDBE2681833A360E1
:101EA800531EE360002BE2D12369013B2361002B21
:101EB80034DB58F82330E36003F046FBD9E7002A07
:101EC800A8BF2B46B6DA6B1E3C32A3606260B1E74E
:101ED8002B68DBF81C209342BFF640AFDBF83820B4
:101EE8009342ACBF002301232362002B3FF46DAF64
:101EF800DBF83C106BE74FF0FF33236265E762695C
:101F0800002323610132E361626103F01DFBB0E746
:101F18000023236259E70622A261BEE765690B2305
:101F28002361013D656115F0030F0BD1284664213B
:101F380009F098FB31B1012101F5B6720B2301328A
:101F4800E261B6E728464FF4C87109F08BFBD1F17E
:101F5800010138BF0021EFE7704700BF704700BF9D
:101F680038B545F68C24C2F200040546084600231D
:101F780023602DF0BFFDB0F1FF3F00D038BD2368CE
:101F8800002BFBD02B6038BD38B50446456C0DB12D
:101F9800002038BD8021FFF7C3F8606440B10346D4
:101FA800284603F1800243F8040B9342FBD138BD65
:101FB8004FF0FF3038BD00BF1F2910B5044682B06E
:101FC80007D8436C53B153F8210043F8212002B0DD
:101FD80010BD16234FF0FF302360F8E701910092FF
:101FE800FFF7D2FF0199009A08B9636CEBE74FF04D
:101FF800FF30ECE71F2970B50C46054620D8426C27
:10200800A2B152F821308BB1012B0DD0B3F1FF3FB3
:1020180006D00025084642F821509847284670BD4A
:10202800162301202B6070BD002070BD284600F0EB
:102038006BF8224601462846BDE8704000F04EB8CD
:1020480016234FF0FF302B6070BD00BF1F2910B55D
:10205800044682B012D8426CCAB152F8213002EB61
:10206800810283B1B3F1FF3F0FD0012B09D00024C7
:10207800084614609847204602B010BD4FF0FF3064
:10208800FAE70320F8E70120F6E70220F4E70191D8
:10209800FFF77AFF01990028F0D1626CDDE700BFF5
:1020A80040F2A4030146C2F200031868A2E700BF89
:1020B80040F2A4030A46C2F20003014618687BE70F
:1020C80040F2A403C2F2000318685DE740F2A403DB
:1020D8000146C2F200031868B8E700BF38B545F6F4
:1020E8008C24C2F2000405460846114600232360EA
:1020F8000FF052FCB0F1FF3F00D038BD2368002B31
:10210800FBD02B6038BD00BF0FF054BC08B4F0B54D
:10211800141E9CB0054625DB22AE4FF402730191D4
:1021280008BF2746ADF810303346059101A9219A1A
:1021380018BF671E1B96039706974FF0FF37ADF839
:10214800127000F0E9FEB0F1FF3F08DB14B1019B0B
:1021580000221A701CB0BDE8F04001B070478B2314
:102168002B60F3E78B234FF0FF302B60F2E700BFC3
:102178000CB440F2A403F0B5C2F200030C1E9DB0EB
:102188001D6826DB23AE4FF40273019001A9ADF858
:102198001030334605902846229A08BF27461B96DA
:1021A80018BF671E039706974FF0FF37ADF81270F8
:1021B80000F0B2FEB0F1FF3F08DB14B1019B002232
:1021C8001A701DB0BDE8F04002B070478B232B6039
:1021D800F3E78B234FF0FF302B60F2E70EB44FF498
:1021E8000172F0B59CB021AC42F2BD25ADF81020CB
:1021F800C0F6000554F8046B0190059000F088FAC9
:1022080040F2A4033246C2F2000301A900264FF0AF
:10221800FF3E0A95ADF812E00E9613961B940746FA
:10222800186823460297069702F096F91CB0BDE895
:10223800F04003B0704700BF0CB44FF401732DE9B0
:10224800F0419CB022AC80460846ADF8103054F8F6
:10225800046B42F2BD250191C0F60005059100F01E
:1022680057FA324601A9234600264FF0FF3E0A9549
:10227800ADF812E00E9613961B9407464046029757
:10228800069702F069F91CB0BDE8F04102B070474A
:1022980010B50C46B1F90E1005F022F80028ABBFB6
:1022A800636DA3891B1823F48053ACBF6365A381B6
:1022B80010BD00BF002070472DE9F0411D468B89F5
:1022C8000C460746164613F4807F06D00223B1F960
:1022D8000E10002204F0BEFAA38923F48053384676
:1022E800A3813246B4F90E102B46BDE8F04103F045
:1022F80017BA00BF10B50C46B1F90E1004F0AAFACF
:10230800A389B0F1FF3F15BF606523F4805343F400
:102318008053A38118BFA38110BD00BFB1F90E106F
:1023280003F014BA10F0030F38B5044612D103684D
:10233800A3F1013222EA030313F0803F0AD1031DFF
:10234800184653F8042BA2F1013525EA020212F0CF
:10235800803FF5D003782BB1431C184613F8012BA6
:10236800002AFAD100F076F9204638BDC9B2F0B497
:10237800002950D010F0030F10D00378002B79D02B
:10238800994246D0431C05E013F8012B002A3FD0A0
:1023980091423ED013F0030F1846F5D1036841EA85
:1023A80001270646A3F1013247EA074722EA03025A
:1023B80012F0803F1DD187EA0303A3F1013222EA1C
:1023C800030313F0803F14D1043002E012F0803F81
:1023D8000FD1064650F8043BA3F1013587EA030202
:1023E80025EA0303A2F1013413F0803F24EA020234
:1023F800ECD033783046002B3CD0994209D0731C7E
:1024080001E0914205D0184613F8012B002AF8D1B3
:102418001046F0BC704710F0030F0CD00378002B67
:10242800F7D0431C03E013F8012B002AF1D013F076
:10243800030F1846F7D102680346A2F1013121EAD9
:10244800020212F0803F0AD10430034650F8042BF0
:10245800A2F1013121EA020212F0803FF5D01A7888
:102468001846002AD5D00133184613F8012B002A44
:10247800FAD1CEE71846CCE780EA010212F0030F42
:102488003AD110F0030220F0030021F0030150F8C4
:1024980004CB08BF51F8043B0DD082F003024FEA89
:1024A800C2026FF07F4323FA02F251F8043B4CEA70
:1024B800020C43EA020300BFACF101329C4501BFA4
:1024C80022EA0C0212F0803F50F804CB51F8043B8A
:1024D800F2D04FEA0C604FEA1C2C012828BFB0EB61
:1024E800036F08BF1B0AF4D003F0FF034FEA106024
:1024F800A0EB0300704700BF10F0030F0AD010F8DC
:10250800012B11F8013B012A28BF9A42F4D0A2EB13
:10251800030070474DF8045D4DF8044D4FF001027B
:1025280042EA022242EA024201F0030C21F00301CE
:1025380050F8044B51F8045BBCF1020F26D04BD87D
:1025480024F07F4CBCEB152FA4EB020323EA040311
:102558000DD113EAC21308BF51F8045B0AD18CEA03
:10256800040CBCEB056F0CD150F8044BE8E74FEABC
:1025780015255CE033F07F4352D10D784FEA146C97
:1025880055E04FEA146C05F0FF0550E04FEA044CA3
:10259800A4EB02034FEA1C4C23EA0403BCEB154FDF
:1025A80017D113EAC21308BF51F8045B07D18CEAAC
:1025B800040CBCEB054F08D150F8044BE6E71B04AC
:1025C8002ED10D884FEA144C31E04FEA05454FEA09
:1025D800144C4FEA15452AE004F0FF0CBCEB156FCC
:1025E800A4EB020323EA04030DD113EAC21308BFC4
:1025F80051F8045B0AD18CEA040CBCEB052F0AD114
:1026080050F8044BE8E74FEA156510E014F0FF0FA7
:1026180006D051F8045B4FEA142C25F07F4506E0FC
:102628004FF000005DF8044B5DF8045B70470CF058
:10263800FF0205F0FF00012828BF904204BF4FEABF
:102648001C2C2D0AF3D0A2EB00005DF8044B5DF8BA
:10265800045B704780EA0102844612F0030F4FD1F1
:1026680011F0030F32D14DF8044D11F0040F51F859
:10267800043B0BD0A3F101329A4312F0803F04BF10
:102688004CF8043B51F8043B16D100BF51F8044BF9
:10269800A3F101329A4312F0803FA4F101320BD129
:1026A8004CF8043BA24312F0803F04BF51F8043BAE
:1026B8004CF8044BEAD023460CF8013B13F0FF0F0B
:1026C8004FEA3323F8D15DF8044B704711F0010F3E
:1026D80006D011F8012B0CF8012B002A08BF70470F
:1026E80011F0020FBFD031F8022B12F0FF0F16BF06
:1026F8002CF8022B8CF8002012F47F4FB3D17047CE
:1027080011F8012B0CF8012B002AF9D1704700BFF2
:1027180020F0030110F00300C0F1000051F8043B61
:1027280000F1040C4FEACC0C6FF000021CBF22FA37
:102738000CF213434FF0010C4CEA0C2C4CEA0C4CF5
:10274800A3EB0C0222EA030212EACC1204BF51F8EE
:10275800043B0430F4D013F0FF0F1FBF013013F413
:102768007F4F013013F47F0F18BF0130704700BF4F
:10277800F0B4002A46D041EA000313F003032CD139
:10278800032A07460E4643D904680D68AC423FD178
:10279800043A37D0A4F1013525EA040414F0803F47
:1027A80018BF18462CD1041D0D1D0EE054F8043B2B
:1027B80055F8041BA3F101308B4220EA030027D10E
:1027C800043A1FD010F0803F1ED1032A27462E4618
:1027D800ECD820462946002A1DD00478013A0D7805
:1027E800AC420CD172B18CB1002302E093420BD001
:1027F80064B1013310F8014FCD5CAC42F6D0601BD8
:10280800F0BC70471046FBE70020F9E72046F7E7E1
:1028180038463146E1E724782D78F0E741EA0003AD
:1028280013F0030F0B4670B414BF00240124032ACD
:1028380094BF002404F001040546D4B9BAB10E7857
:102848002B46013A03F8016B56B1AC1C7AB111F86A
:10285800015F2346013A04F8015C0134002DF5D1EB
:102868002AB19A18002103F8011B9342FBD170BCCE
:102878007047194653F8044BA4F1013626EA0406BA
:1028880016F0803FDAD1043A45F8044B032A19467A
:10289800EFD8D3E701232DE9F0071D4600264FF0B6
:1028A800FF37AC1900EB070C8C420DD21CF805C0A1
:1028B80010F80480E0452ED201252646E31BAC190A
:1028C8008C4200EB070CF1D34FF0010900264D466E
:1028D8004FF0FF3C1360AC1900EB0C08A1420ED975
:1028E80018F8058010F804A0C2451AD90125264613
:1028F800CCEB0409AC19A14200EB0C08F0D80CF1A0
:1029080001000137B8423CBF99463846C2F80090EA
:10291800BDE8F00770470BD0012337461D46F6186F
:10292800BFE709D04FF00109B4464D464E44D2E7FF
:102938009D4205D00135B4E74D4505D00135CAE7BC
:102948002B4626460125ACE7A94626460125C2E7BF
:102958002DE9F04FADF5826D81B01446074610465B
:102968000DF580628B460C3219461D46FFF792FF23
:1029780003AE04A901F57E72331F009043F8045F8B
:102988009342FBD14DB1681E0023E25CC11A0133AA
:1029980003AEAB4246F82210F7D1DDF80C142046FE
:1029A800009A6118FEF7C0FE002877D10099814689
:1029B80005F1FF380646C1F1010201925A46AB46BD
:1029C80009EB0B0501F1FF3AB8180021AA1AFEF726
:1029D80065FE00284FD1002D00F0C0807B1903A9A7
:1029E80013F8013C51F82330002B4CD1009B9E4238
:1029F80028BF334698450FD903EB0901E05C7A18E4
:102A0800795C884205D038E012F8011FE05C884202
:102A180033D101339845F7D8009A964280F0A480C4
:102A280007EB090214F80A10534612F80A209142DB
:102A380004BF0AEB0901791807D095E014F802C021
:102A480011F8010D844503D113465A1EB342F5D13E
:102A580001369E4200F28D80DDF80C642A46B144AE
:102A6800C6EB0B0609EB0B05B8180021AA1AFEF7EE
:102A780015FE0028AFD0002071E0019A002691448D
:102A880099442A46EEE7002EFAD0DDF80C2493424A
:102A98003CBFC2EB0B0306469944F2E7009E4FF099
:102AA80000080099AB1BB34238BF3346C1F101029D
:102AB8006E1E019201F1FF3A5A468946AB46013330
:102AC800CDF80C3408EB0B05B8180021AA1AFEF74C
:102AD800E5FD0028CFD1002D40D07B1903A913F8BC
:102AE800013C51F82330002B30D1B14513D208EB0B
:102AF800090314F80910FA18FB5C994218BF4B46F1
:102B080027D14B4604E012F8011FE05C884220D12F
:102B18000133B342F7D3BAF1FF3F53462CD007EB4A
:102B2800080C14F80A101CF80A2091420CD10AEB80
:102B38000802BA1804E0E05C12F8011D884203D1CB
:102B4800013BF8D260460AE0DDF80C3498442A4686
:102B5800B8E701992A4688449844B3E7284605B05F
:102B68000DF5806DBDE8F08F009B01369E427FF623
:102B780073AF07EB0900F2E707EB080C6046EEE7D6
:102B88002DE9F04F8346037885B00C46002B00F002
:102B9800F9800A78A2B106460131012002E011F855
:102BA800012B8AB1934214BF002000F0010016F8EF
:102BB800013F0D46002BF2D12B782BB14FF0000BC3
:102BC800584605B0BDE8F08F0028F9D10BF1010097
:102BD8002178FFF7CBFB2D1BA5F10102534243EBF4
:102BE8000203002808BF43F00103074683B90BEB33
:102BF8000508404594BFC0EB08084FF001081F2D99
:102C080008D9414622462B46FFF7A2FE8346D7E75E
:102C18008346D5E7294603AA2046FFF73BFE0399DA
:102C28006118814620464A46FEF77EFD00284FD1AE
:102C380009F1FF33C9F10102064601928246424674
:102C4800C84699460AEB050BB8180021C2EB0B02DF
:102C5800FEF724FD0028B1D1BBF1000FB0D04645E6
:102C68002CBF334643469D420FD903EB0A01E05C73
:102C78007A18795C884205D075E012F8011FE05C8B
:102C8800884270D101339D42F7D1B0457DD907EB19
:102C98000A0214F809104B4612F80920914202BFA3
:102CA80009EB0A01AC46791806D06EE0A55C11F86C
:102CB800010D854203D113465A1EB342F6D165462B
:102CC80001369E4267D8039E5A46B244AE1BB9E706
:102CD800C9F10101C9EB05034246002609F1FF3A93
:102CE80088464B4538BF4B460133039306EB050B2B
:102CF800B8180021C2EB0B02FEF7D0FC00287FF4C5
:102D08005DAFBBF1000F3FF45BAF4D4512D906EB49
:102D1800090314F80910FA18FB5C994208BF4B46DE
:102D280005D026E012F8011FE05C884222D1013369
:102D38009D42F7D1BAF1FF3F534628D007EB060C66
:102D480014F80A101CF80A20914217D10AEB06025F
:102D5800BA1804E0E05C12F8011D88420ED1013B6C
:102D6800F8D2E3462CE7019A002692445A469A4440
:102D780068E74B4646445A46F618B7E7039B5A4657
:102D8800F618B3E70D46012016E7434698E707EB28
:102D9800060CE34614E707EB0A0B11E72DE9F04FA1
:102DA80040F2AC54C2F2000485B01F468C46266837
:102DB8000B460390029213F8014B32191D4692F804
:102DC80001B01BF0080BF6D12D2C73D02B2C08BFAB
:102DD80015F8014BD7F1010338BF0023102F14BF9A
:102DE8001A4643F0010232B1302C73D01BB1302C9B
:102DF80000F083800A27B946BBF1000F49460CBF93
:102E08006FF0004A4FF0004ACDF804C0504608F071
:102E1800D1FA50468846494608F09EF933190022EF
:102E2800DDF804C05B78114613F0040F1ED0303C67
:102E3800A74225DD814294BF0023012353EAD272C1
:102E48002ED10A1A534243EB02034445D4BF002350
:102E580003F00103002B23D109FB014115F8014BB5
:102E6800012233195B7813F0040FE0D113F0030348
:102E780006D0012B14BF57233723E41AA742D9DC05
:102E8800B2F1FF3F1BD00846BBF1000F10D1029BE7
:102E98001BB152B90299C1F800C005B0BDE8F08F66
:102EA8004FF0FF3215F8014BDBE705F1FF3CF1E786
:102EB8004842ECE715F8014B4FF0010B8AE70399FC
:102EC800BBF1000F0CBF6FF000404FF00040222311
:102ED8000B60DCE72A78A2F17800414241EB00015F
:102EE800582A14BF0A4641F00102002A3FF47EAF77
:102EF80010276C78B94602357EE70827B9467BE784
:102F080030B440F2A404C2F200040D461346014650
:102F18002A46206830BC41E72DE9F04FC5B0144679
:102F280012930C91119003F085FC00681990FFF73B
:102F3800EFFB1C900C98838913F0800F03D0036972
:102F4800002B01F06F810DF17C0A002356460DF12C
:102F5800F7010E9309941A931B9317931D930F93DC
:102F68000791CDF8E4A03B933A93099A1378B3F10B
:102F7800250218BF0122002B0CBF002302F0010319
:102F8800002B00F0BD80099B5A1C174601323B7884
:102F9800191E18BF0121252B0CBF002301F00103C6
:102FA800002BF2D1099CB7EB040810D03A9C099881
:102FB80001343B9D072CC6F80480306045443A94A0
:102FC8003B9500F3818008360F9941440F913B7877
:102FD800002B00F081807C1C002200230D928DF8CC
:102FE8000F31202509942B217B784FF0FF37089269
:102FF80022460132A3F12000582800F21C83DFE8A2
:1030080010F02D031A031A0336031A031A031A03BE
:103018001A031A031A03C70381001A035D00850007
:103028001A039F00A500A500A500A500A500A500FE
:10303800A500A500A5001A031A031A031A031A0308
:103048001A031A031A031A031A03B70041021A03D0
:1030580041021A031A031A031A037F021A031A03F6
:1030680085021A031A031A031A031A03A3021A037E
:103078001A03B2021A031A031A031A031A031A03C9
:103088001A031A031A031A0354033C0341024102A8
:1030980041024E033C031A031A030B031A039A0353
:1030A80068037E03DD021A03E3021A03AB031A0363
:1030B8001A03D2030D9B12905B420D93089C44F0B7
:1030C80004040894137894E7119839AA0C9905F028
:1030D80093FE40B9564677E73B9B23B1119839AA2E
:1030E8000C9905F089FE0C990F9A8B8913F0400F03
:1030F80018BF4FF0FF320F920F9845B0BDE8F08F20
:10310800099F64E78DF80F11137872E712F8013BF5
:103118002A2B01F0FC81A3F13000092801F2AC81CF
:103128001446002714F8013B07EB870700EB470715
:10313800A3F1300009282246F4D947EAE77759E78E
:10314800089B43F080030893137852E71446002045
:10315800A3F1300814F8013B00EB8000A3F1300C18
:103168002246BCF1090F08EB4000F1D90D9041E768
:103178000992089A169342F010020892089B13F0DD
:10318800200F00F08182129CE31D23F0070303F156
:1031980008001290D3E90045002C75F10002C0F236
:1031A800CD8554EA05034FF001030CBF002201222C
:1031B800002FA2BF089921F080010891002F18BFA5
:1031C80042F00102002A00F0AC83012B00F0FE84DB
:1031D800022B00F0DE840DF1BC0B0BF12703EA088B
:1031E8004FEAD40848EA457804F00704114604F188
:1031F80030020D4644469C461A70013B54EA0500CD
:10320800EDD10899CDF84CC011F0010F40F0888538
:103218000BF1280BCCEB0B0210929DF80F2100202C
:10322800109C1497BC42B8BF3C4618900A9412B13F
:103238000A9801300A90089911F0020B02D00A9BF3
:1032480002330A93089C14F08404159440F0CD824C
:103258000D980A99471A002F40F3C782102F41F39F
:1032680065803B9D42F658383A9CC0F603082946CB
:103278004FF0100922460C9D4446DDF8448002E0D8
:10328800103F102F1BDD01323460C6F80490103156
:103298000836072A3A9206F108033B91F0DD4046CA
:1032A800294639AA564605F0A7FD0AF10803002861
:1032B8007FF419AF103F3B99102F3A9AE3DCA046F0
:1032C8000D4614460134C6F80080072C77603D444B
:1032D8003A943B9500F37E829DF80F211E466AB111
:1032E8003A9C43AB0333336001340123072C7360EA
:1032F8001D443A943B9500F3E9830836BBF1000F6F
:103308000CD03A9C43AB3360022301347360072C22
:103318001D443A943B9500F3CE830836159A802ACB
:1033280000F01083149910980F1A002F40F35B8354
:10333800102F40F3EB853A9C2A46DFF8988A4FF025
:10334800100B23460C9D4446DDF8448002E0103FF4
:10335800102F1BDD01333460C6F804B01032083674
:10336800072B3A9306F108093B92F0DD40462946BF
:1033780039AA0AF1080905F03FFD564600287FF4EE
:10338800B2AE103F3B9A102F3A9BE3DCA04615469D
:103398001C460134C6F80080072C77603D443A94F7
:1033A8003B9500F37D83089A12F4807F40F04E82AB
:1033B8003A9C109B01341398072C1D44C9F804301B
:1033C800C9F800003B953A9400F3358209F10809E1
:1033D800089C14F0040F46D00D980A99461A002E3E
:1033E80041DD102E40F3DA873A9C42F65838C0F691
:1033F800030810272346DDF830B04446DDF8448042
:1034080002E0103E102E19DD01331035072BC9F8E4
:103418000040C9F8047009F108093A933B95F0DDBA
:103428004046594639AAD14605F0E6FC00287FF403
:103438005AAE103E3B9D102E3A9BE5DCA0461C463A
:103448000134C9F80080072CC9F8046035443A945F
:103458003B9508DD119839AA0C9905F0CDFC002898
:103468007FF441AE3B9D0F9A0A9C0D9B9C42ACBFDA
:103478001219D2180F92002D40F0038300205646EF
:103488003A9072E508991D46099211F0080F1693B3
:1034980000F08784129AD31D23F0070303F1080470
:1034A800129418681A905B681B931A981B9904F079
:1034B8003BF9012840F050841A98002200231B99F8
:1034C80008F00AFD002840F01C879DF80F21032012
:1034D80044F2283344F224310A901698C0F60301C6
:1034E800C0F6030300244728D8BF0B460899139356
:1034F800032321F08001149408911093189496E600
:10350800089C44F008040894137872E50899099215
:1035180041F010010891089A169312F0200300F068
:10352800DF80129BDA1D002322F0070202F1080453
:103538001294D2E9004554EA05000CBF002201228A
:1035480000208DF80F0133E6089C099244F010041E
:1035580008940898169310F0200F00F0048112992F
:103568000123CA1DE0E7099244F2E821089AC0F64F
:103578000301169312F0200F179100F02081129C7E
:10358800E31D23F0070303F108001290D3E9004577
:1035980054EA0502089B0CBF00220122134200F0E6
:1035A800698316983023089901228DF80C3102237B
:1035B80041F002018DF80D010891C1E7089840F02B
:1035C80020000890137814E509920021129A1693A6
:1035D8008DF80F11141D13681393002B00F0F0865B
:1035E800002FC0F29386139800213A46FEF756F84A
:1035F800002800F03687139BC01A1090B84240F399
:10360800F484002027EAE77114900A919DF80F21AD
:103618001294109718900AE613786C2B0BBF089B2E
:10362800089C43F0200344F010040ABF0893089450
:1036380012F8013FDDE409921693002B3FF44CADDC
:10364800002201218DF8BC302FAC00230A91109183
:103658008DF80F31149218921394ECE59DF80F3100
:10366800002B40F09B838DF80F511378C1E4089824
:1036780040F0010008901378BBE41693089B099268
:1036880013F0200F7FF47FAD089911F0100F00F0B0
:10369800A383129A146804321292E5177CE50898FD
:1036A80040F0400008901378A3E416930121129B80
:1036B8000020099200221C1D0A911B681294109187
:1036C8002FA98DF80F011492189213918DF8BC3020
:1036D800B1E50992089A169312F020037FF421AFFE
:1036E800089911F0100200F09183129C22680434AA
:1036F800002512941446003A18BF012220E7129BB5
:103708007821089C0025099244F2D4201A6844F0D4
:10371800020404330894129314463023003A8DF8B7
:103728000C3118BF0122C0F603008DF80D11179057
:103738000223169104E70992089A12F0200F00F06C
:103748005883129B0F9C129819682246E31704307D
:103758001290C1E9002308E40898099210F0200F9C
:1037680016937FF4FCAE089911F0100F40F0918287
:10377800089810F0400F00F08C8212990123002560
:103788000A88043112911446003A18BF0122D7E67C
:10379800129B129C1B68201D002B0D93FFF68AAC10
:1037A8001378129025E4099244F2D420089AC0F6BE
:1037B8000300169312F0200F17907FF4E0AE0899DB
:1037C80011F0100F00F0FA82129A002514680432E2
:1037D8001292DDE6119839AA0C9905F00DFB002824
:1037E8007FF481AC9DF80F2156463B9D77E5089AFA
:1037F80012F0010F40F0FD803A9C0135139A012325
:103808000134C9F80430072CC9F800203B953A94D4
:1038180000F31F8509F1080B0BF108091D9B013402
:10382800072C1D44CBF804303EABCBF800303B9559
:103838003A947FF7CDAD119839AA0C9905F0DCFAC6
:1038480000287FF450ACD1463B9DC1E51699652907
:1038580040F3CB801A98002200231B9908F032FB12
:10386800002800F03E813A9C44F23433C0F603034A
:10387800C9F8003001340123072CC9F804301D446D
:103888003A943B95D8BF09F1080900F34683429B57
:103898000E9A934204DB089B13F0010F3FF498AD96
:1038A8003A9C1C9801341999072C0544C9F804005E
:1038B800D8BF09F10803C9F800103B953A9400F302
:1038C800BC830E9A561E002E40F31D83102E40F323
:1038D800E8853A9C1027DFF8FC842246DDF830B0F2
:1038E8004446DDF8448003E0103E102E40F3C481C6
:1038F80001321C605F6010350833072A3A9203F1E1
:1039080008093B95F0DD4046594639AA0AF10809ED
:1039180005F072FA534600287FF4E5AB3B9D3A9ACE
:10392800E2E7002B40F0B780089C14F0010F00F08C
:103938002B81012030230DF1E30110908DF8E33045
:1039480013916AE40D9B0A9C1F1B002F7FF7EAACBA
:10395800102F40F369853A9C3346DFF878844FF09E
:1039680010092246DDF830B04446DDF8448002E014
:10397800103F102F1BDD01321C60C3F80490103576
:103988000833072A3A9203F108063B95F0DD4046D2
:10399800594639AA0AF1080605F02EFA53460028B6
:1039A8007FF4A1AB103F3B9D102F3A9AE3DCA04671
:1039B80014460134C3F80080072C5F603D443A94F4
:1039C8003B957FF7AFAC119839AA0C9905F014FA1A
:1039D80000287FF488AB1499564610983B9D0F1A1F
:1039E800002F3FF7A5ACB146DDE40E9901297FF71A
:1039F800FEAE3A9C0135139B0134C9F8003001230F
:103A0800072CC9F80430D8BF09F108093B953A9446
:103A1800D8BF09F1080600F3418101341C991998AF
:103A2800072C0D44D8BF06F1080BC9F80410C9F8D3
:103A380000003A943B9500F33F811A980022002336
:103A48001B9908F03FFA002840F0CE800E9B013405
:103A580013985A1E7260431C072C336015443A941D
:103A68003B957FF7D9AE119839AA0C9905F0C4F99E
:103A780000287FF438AB0AF10809D3463B9D3A9CED
:103A8800CCE6119839AA0C9905F0B6F900283FF44C
:103A9800F5ACFFF728BB109239AA1392FFF7BDBB0C
:103AA800119839AA0C9905F0A7F900287FF41BABE7
:103AB800D1463B9D77E4119839AA0C9905F09CF9F9
:103AC80000287FF410AB3B9D564627E4119839AA8D
:103AD8000C9905F091F900287FF405AB3B9D5646FB
:103AE8000CE4429E002E40F323820E9E189C1398ED
:103AF800A642A8BF26460E99002E00EB010B0EDD4C
:103B08003A9CAD19C9F800000134C9F80460072CC3
:103B18003B953A94D8BF09F1080900F31184189A23
:103B280026EAE676961B002E40F3E983102E40F332
:103B3800E1843A9C2946DFF89C82102722460C9D96
:103B48004446DDF8448003E0103E102E40F37081B7
:103B580001321031072AC9F80040C9F8047009F188
:103B680008093A9209F108033B91EDDD40462946E0
:103B780039AAD14605F040F90AF1080300287FF474
:103B8800B2AA3B993A9ADFE7109339AB1393FFF740
:103B980044BB0DF1BC0B17990BF1270004F00F0281
:103BA800230943EA05734FEA151C8A5C1C46034641
:103BB800654601381A7054EA0502EFD10BF1280B5B
:103BC8001393C3EB0B031093FFF727BB0A2C75F174
:103BD80000017FD2303401220DF1E30310928DF8F9
:103BE800E3401393FFF719BB0E994F1E002FDCBF5C
:103BF80006F10809B3467FF711AE102FD8BFDFF8DA
:103C0800D4812CDDDFF8CC8123462A464FF01009F9
:103C180044460C9DDDF8448002E0103F102F1BDD68
:103C280001333460C6F8049010320836072B3A93F3
:103C380006F1080B3B92F0DD4046294639AA0AF105
:103C4800080B05F0D9F8564600287FF44CAA103F17
:103C58003B9A102F3A9BE3DCA04615461C460134DC
:103C6800C6F80080072C77603D443A943B957FF76F
:103C7800D3ADF8E6022363E4A04614460134C3F842
:103C88000080072C5E6035443A943B957FF7A0ABE3
:103C9800D1E5129B129C1A68012328E5119839AACC
:103CA8000C9905F0A9F800287FF41DAA3B9D0AF19C
:103CB80008063A9CD146B0E6119839AA0C9905F045
:103CC8009BF800287FF40FAA3B9D0AF1080B3A9C49
:103CD8005646B2E60DF1BC0BB1460BF1270820465B
:103CE80029460A22002308F02DFA4646204629468E
:103CF800002308F1FF3802F130040A22347008F07A
:103D080021FA04460D4654EA0500E8D113960BF152
:103D1800280B13994E46C1EB0B011091FFF77DBAA2
:103D2800302A00F0338313930BF1280B1398C3EB5D
:103D38000B04302310940370FFF76FBA644265EBED
:103D480045052D2354EA05008DF80F310CBF0022DC
:103D580001220123FFF72CBA1A981B9903F0E4FCFF
:103D6800002840F07581149044F2303344F22C322C
:103D78001698C0F60302C0F603034728D8BF1346B7
:103D88001393149B032408990A9421F080019DF849
:103D98000F21089110941893FFF749BA1378FFF789
:103DA80028B91299CB1D23F0070303F108021292D8
:103DB8001C681A945B681B93FFF777BB089B13F08A
:103DC800400F00F0268112980025048804301290D4
:103DD800FFF7DEBB682B0308089B13F0400F00F0C9
:103DE80011811298B0F9004004301290E517FFF7DE
:103DF800D3B9089911F0100F00F01281129A0F9C94
:103E08001368043212921C60FFF7AFB8089810F0DC
:103E1800400300F0FC81129B0025129C1988043491
:103E2800134612940A1E0C4618BF0122FFF788BBDE
:103E3800A0460D4614460134C9F80080072CC9F87D
:103E4800046035443A943B9500F3AF82429A0E9C45
:103E5800A2424ADB089810F0010F46D1139C18982B
:103E680021180E9CC1EB0B07A21ABA42B8BF17461D
:103E7800002F0ADD3A9CED19196001345F60072CA8
:103E88003B953A9400F37482083327EAE776961B49
:103E9800002E38DD102E40F304833A9C1027DFF8FB
:103EA800B4862246DDF830B04446DDF8448003E0AD
:103EB800103E102E7FF7E0AE01321C605F601035B7
:103EC8000833072A3A9203F108093B95F0DD40468A
:103ED800594639AA0AF1080904F08EFF534600280A
:103EE8007FF401A93B9D3A9AE2E73A9C1C99013478
:103EF8001998072C0D44596018603B953A9400F3C3
:103F08002B820833AAE79946FFF762BA06F1080937
:103F18003A9CDFF84086FFF73CBA119839AA0C9909
:103F280004F06AFF00287FF4DEA83B9DD146AEE48A
:103F38003A9C44F23433C0F60303C9F80030013424
:103F48000123072CC9F804301D443A943B95D8BF87
:103F580009F1080900F38C8136B90E9B23B9089C36
:103F680014F0010F3FF434AA3A9C1C9801341999B3
:103F7800072C0544C9F80400C9F80010D8BF09F196
:103F880008093B953A9400F3AB817642002E40F342
:103F98009881102ED8BFDFF8BC8540F37A81DFF80E
:103FA800B48523461027DDF830B04446DDF8448058
:103FB80003E0103E102E40F36A8101331035072BC1
:103FC800C9F80040C9F8047009F108093A933B950B
:103FD800EFDD4046594639AAD14604F00DFF0028C6
:103FE8007FF481A83B9D3A9BE3E7109B0022129443
:103FF8000024149223EAE3739DF80F210A9318947E
:10400800FFF715B912990C6804311291E517FFF7FB
:10401800C3B8129900250C6804311291FFF7B8BA99
:10402800089810F0400F00F00C8112990F9A0B6855
:10403800043112911A80FEF798BF119839AA0C9989
:1040480004F0DAFE00287FF44EA83B9D534638E47E
:10405800B7F1FF3F00F05181169CA4F1670EDEF125
:10406800000343EB0E03472C08BF43F0010313B1D1
:10407800002F08BF01271B9B0898002B40F4807075
:104088000890C0F20182DDF86C9000221492169B11
:10409800A3F16604D4F1000B4BEB040B462B08BFCD
:1040A8004BF0010BBBF1000F40F0BB81452B02D058
:1040B800652B40F0E68107F1010802231A9C42A90A
:1040C800CDF82C9000930A94DDE90A231198029107
:1040D80041A9CDF80480039140A9049101F0E2FBC5
:1040E800169AB2F1670318BF0123472A0CBF0023B1
:1040F80003F00103139023B9089B13F0010F00F09C
:10410800E181139800EB0804BBF1000F05D0037898
:10411800302B00F0E281429BE4181A980022002319
:10412800494607F0CFFE002800F0858123464094D9
:104138001699139CA1F167004242C4EB030342EBBA
:1041480000020E93472914BF134642F00103002BC7
:1041580000F04881429B13F1030F109302DB9F424A
:1041680080F27481169802381690013B169A002B3B
:1041780042938DF8F820C0F2C3812B228DF8F920E4
:10418800092B40F3868146F267640DF1F600C6F20A
:10419800666484FB0321DA170546C2EBA10202EB31
:1041A8008201A3EB410113463031092A00F80119B5
:1041B800EFDC30336A1E05F8013C0DF1F7039A4233
:1041C80080F0C4810DF1FA0312F8011B03F8011BFA
:1041D8001946079C9442F7D83EAB0E98CB1A0E9915
:1041E80018181D930129109040F36E81109B00242C
:1041F800189401331093149B002B40F00781109CF6
:104208009DF80F2124EAE4740A94FFF710B8129875
:1042180000250268043012901446003A18BF0122A3
:10422800FFF78EB940211198FCF77AFF0C990860C6
:104238000861002800F082810C9840234361FEF752
:1042480082BE129C0F982368043412941860FEF7FB
:104258008CBE119839AA0C9904F0CEFD00287EF482
:1042680042AF3B9D0DF184093A9CD346FFF7D6BA7D
:10427800119839AA0C9904F0BFFD00287EF433AFD9
:10428800429ED1463B9D002E7FF46EAE65E6A04669
:104298001C460134C9F80080072CC9F8046035446D
:1042A8003A943B95D8BF09F108090ADD119839AA53
:1042B8000C9904F0A1FD00287EF415AF3B9DD14672
:1042C8003A9C01340E9B139A072C1D44C9F80430FC
:1042D800C9F800203A943B957FF778A8FFF7ABBA66
:1042E800119839AA0C9904F087FD00287EF4FBAEDA
:1042F800429ED1463B9D3A9C47E60627BBE64B4685
:10430800A4E52D228DF80F21FFF7E1B813980021BD
:104318001491FEF7FDF9149B1294189320EAE072A9
:1043280010900A929DF80F21FEF781BF42F6583887
:1043380006F108033B9DC0F603083A9CFEF7C2BF8E
:10434800119839AA0C9904F057FD00287EF4CBAED9
:104358003B9DD146FFF7E3BB119839AA0C9904F0AD
:104368004BFD00287EF4BFAE429A53463B9D75E54F
:10437800119839AA0C9904F03FFD00287EF4B3AED9
:10438800429A53460E983B9D821A7EE5139B0BF189
:10439800280BC3EB0B031093FEF73FBF42F65838C8
:1043A8003A9CC0F60308FFF74BB8119839AA0C9944
:1043B80004F022FD00287EF496AE53463B9D45E569
:1043C800062F28BF062744F2183027EAE771C0F6FF
:1043D80003001A4610970A91129414931893139095
:1043E800FEF725BF1699662940F08F80429B002B67
:1043F800109340F398801FB9089810F0010F02D06D
:104408005A1CD219109218931695F4E610982D227A
:1044180000218DF80F2120EAE07014910A90FEF730
:1044280007BFB846032349E633463A9C0836DFF807
:104438002481FFF7BEBA409B9C427FF679AE3022BA
:1044480003F8012BA3424093FAD171E60E9A9342E6
:104458002EDB089C14F0010F3DD0581C67251090E6
:10446800D1E727EAE77214900A9212949DF80F2177
:1044780010971890FEF7DBBE002747EAE777FEF7AC
:10448800B9BDB846022319E62D2103F1004914915C
:10449800FDE5303330223FA98DF8FA208DF8FB3046
:1044A8009AE603F108093A9CDFF8A880FFF7E6BB13
:1044B800002B0E99D4BFC3F10202012252186725BE
:1044C8001092A0E7409B33E6089A12F001037FF4AC
:1044D8008DAE18938FE6672595E71A98002200237A
:1044E800494607F0EFFC00287FF415AEC8F1010338
:1044F800429310E609F108033A9CDFF858809AE4E1
:104508002D225B428DF8F9203AE6429B2DE612985F
:1045180007680430002FBFF643A913784FF0FF3720
:104528001290FEF766BD1FB9089911F0010F02D06D
:104538000237109767E70122109264E7119C4FF049
:10454800FF320C230F922360FEF7D6BD0DF1FA015E
:1045580042E600BF682B03082DE9F04FADF52F7D2B
:104568000C46174680469B46FCF71AFCA38948F67A
:10457800B12113F4005FC0F6000102BF43F40053F9
:10458800A381626E0B9104BF22F40053636600207E
:1045980065AA0546033206900A90079004923A7875
:1045A800AD923AB340F2AC560137C2F20006336816
:1045B800991891F801A01AF0080A22D063680DE052
:1045C800236831685A1C1B78CB185B7813F0080FE6
:1045D800E5D0636801352260013B6360002BEFDCA6
:1045E8004046214605F042FA0028E9D03A78AD92D3
:1045F800002AD7D1FCF7D6FB07980DF52F7DBDE82B
:10460800F08F252A10D06368002B40F30B812368B4
:1046180017F8012C19789142ECD162680133013501
:104628002360531E6360BAE73A78D1460A210137FE
:10463800782A00F20C850FF2080C5CF822F000BF13
:104648007D50000857500008575000085750000880
:104658005750000857500008575000085750000896
:104668005750000857500008575000085750000886
:104678005750000857500008575000085750000876
:104688005750000857500008575000085750000866
:104698005750000857500008575000085750000856
:1046A8005750000857500008575000085750000846
:1046B8005750000857500008575000085750000836
:1046C8005750000857500008575000085750000826
:1046D800575000080F460008575000085750000868
:1046E80057500008575000088B50000857500008D2
:1046F80057500008575000085750000857500008F6
:10470800D14F0008D14F0008D14F0008D14F000801
:10471800D14F0008D14F0008D14F0008D14F0008F1
:10472800D14F0008D14F00085750000857500008D3
:1047380057500008575000085750000857500008B5
:1047480057500008575000085750000857500008A5
:1047580059480008E14F000857500008E14F000889
:104768005750000857500008575000085750000885
:10477800E74F00085750000857500008F14F00084D
:104788005750000857500008575000085750000865
:104798005750000857500008575000085750000855
:1047A80009500008575000085750000821500008C9
:1047B8005750000857500008575000085750000835
:1047C8005750000857500008575000083950000843
:1047D8005D480008E14F0008E14F0008E14F00087C
:1047E800674F0008714F00085750000857500008DD
:1047F800894F0008575000089F4F0008BD4F000818
:10480800955000085750000857500008AF5000084E
:1048180057500008435000085750000857500008E8
:10482800095000084046214605F020F900283FF4C9
:10483800EEAEFCF7B7FA079A002A00F03884A3898D
:1048480003F04003002B18BF4FF0FF320792D3E666
:104858004AF0010A42F6A5530A20C0F600030321D4
:104868000A90069305916368002B40F3E9811AF0DA
:10487800400F17D1236831681A7801338A185278A3
:1048880012F0080F0ED06268013A6260002AC8BFB1
:10489800236012DD01351A7801338A18527812F034
:1048A800080FF0D1059A531E032B00F22581DFE88B
:1048B80013F0D80083000E0045014046214605F05C
:1048C800D5F80028B5D1316801352368E3E709F147
:1048D800FF33B3F5AE7F00F23C8300230DF1440CA7
:1048E80042F67832CDF824C0C0F60302CDF830C0C5
:1048F8006646AC460A9D08974AF4586A1F465B46C6
:10490800934600200590D4F800E09EF80000A0F13E
:104918002B014D2900F2D782DFE811F01503D502EB
:104928001503D502D502B8021003100310031003B3
:1049380010031003100304030403D502D502D502A3
:10494800D502D502D502D5020B030B030B030B03CB
:104958000B030B03D502D502D502D502D502D50229
:10496800D502D502D502D502D502D502D502D50287
:10497800D502D502D502F902D502D502D502D50253
:10498800D502D502D502D5020B030B030B030B038B
:104998000B030B03D502D502D502D502D502D502E9
:1049A800D502D502D502D502D502D502D502D50247
:1049B800D502D502D502F902B9F1000F08BF4FF0B0
:1049C800FF391AF0010340F0F1831AF0100F1EBFEF
:1049D8009A463168236830D1DBF800A00BF1040354
:1049E8002268D346D144117830684118497811F0CB
:1049F800080F40F0B78361680139616012F8011B44
:104A08000BF8011BCB45226000F0AC8361680029DC
:104A1800E9DC40462146029305F028F8029B00286D
:104A280040F0A0832268DEE74046214605F01EF8E4
:104A3800002840F00381316823681A7801338A1806
:104A4800527812F0080F40F0F98062680AF1010A02
:104A58002360013ACA45626000F0F080002AECDC6D
:104A6800E2E7B9F1000F08BF4FF0FF391AF0100F55
:104A78001CBF4FF0000A23682BD1DBF800A0236885
:104A88005646D1441A780DF5D27C1CF80220002A2B
:104A980000F0C9806268013A626013F8012B06F8D9
:104AA800012B4E45236000F0BE806268002AE9DCD5
:104AB8004046214604F0DAFF002840F0B180236820
:104AC800E0E74046214604F0D1FF002840F0B680D8
:104AD80023681A7869AE0133B25C002A00F03F847B
:104AE80062680AF1010A2360013ACA45626000F06F
:104AF800A580002AEDDCE4E7B9F1000F08BF4FF00C
:104B080001091AF0010640F0B6831AF0100F00F000
:104B1800DE826368404621464B4580F24C84226819
:104B2800F618C3EB0909D318236004F09FFF002887
:104B3800EFD0002E3FF47DAE751930E509F1FF3353
:104B4800B3F5AE7F00F29B8100210C91002611AADB
:104B58004AF4F06C09929246CDF820B03A464346A2
:104B68006746B346B0460D960F9605960E96D4F84E
:104B780000E09EF80000A0F12B014E297ED8DFE866
:104B880011F009017D00090100017D00EF006700B7
:104B980067006700670067006700670067006700D5
:104BA8007D007D007D007D007D007D007D00500141
:104BB8007D007D007D00310157017D007D001001E1
:104BC8007D007D007D007D0061017D007D007D0010
:104BD8007D007D005C017D007D007D007D00790108
:104BE8007D007D007D007D007D007D007D00500101
:104BF8007D007D007D00310157017D007D001001A1
:104C08007D007D007D007D0061017D007D007D00CF
:104C18007D007D005C017D007D007D007D007901C7
:104C2800B2453FF406AEB6EB0A0A3FF4E3AC079888
:104C38000BF1040B00230130079033705544AEE4A8
:104C48004046214604F012FF00283FF410AEF0E57C
:104C580006EB0B0191B927F4C0770AF8010B6168DC
:104C68000135013961600029C4BF0EF101012160DD
:104C780040F35782B9F101097FF479AFCDF8148078
:104C8800BC461746059A98465B46DDF820B00AB13F
:104C98002CF4807C013B012B40F21282731E062B00
:104CA8001CD8022E40F22A82032E17D0043E0AF1A5
:104CB800FF33D146CDF830C0F6B208969E1B19F8DE
:104CC800011D4046224604F08BFEB145F7D1089EEF
:104CD800013DDDF830C0F343AD1B9A441CF4807FDE
:104CE80011D01CF4806F40F014821AF8011D013DA8
:104CF800452940F04B8340462246CDF80CC004F0CD
:104D08006FFEDDF80CC01CF010027FF448AC0CF408
:104D1800C0638AF80020B3F5806F00F057830F9BBB
:104D2800002B40F08C83002240460999CDF80CC036
:104D380002F09AFDDDF80CC01CF0010F02460B468C
:104D480003D11CF0020F00F09C83DBF800100BF17C
:104D58000406C1E900230799B346013107911EE40F
:104D680017F4807F3FF474AF0C9827F0800708F1A0
:104D7800010800283FF473AF013809F101090C90CC
:104D88006DE717F4007F3FF479AF27F42077CDF86B
:104D9800388062E717F0800F3FF470AF27F0800784
:104DA8005BE7D6F1010138BF0021B8F1000F14BF4D
:104DB800002101F0010129B107F4E061B1F5E06FCC
:104DC80000F0F382A6F1030CDCF1000141EB0C01C9
:104DD800052E08BF41F0010100293FF44FAF01360D
:104DE800F6B23AE707F4A061B1F5806F07D017F47F
:104DF800806F3FF443AFB8F1000F3FF43FAF17F4B3
:104E0800007F27F4F06708BFCDF834A047F4C077D7
:104E180004BF0E99C1EB08014FF0000808BF0F91BD
:104E28001BE7BBF1010F7FF429AF4FF0020B14E72A
:104E3800022E7FF423AF03260FE7062E7FF41EAF62
:104E480007260AE7DBF1010138BF0021B8F1000F9E
:104E580014BF002101F00101002900F07C8107F452
:104E6800E061B1F5E06F00F0E382042EB7D0012EC7
:104E7800B5D003E7072E7FF401AF0826EDE6A9F5C4
:104E8800AE7040F25D1901380C905FE61AF4006FBD
:104E980009D015B94AF4007A08351AF4806F00F081
:104EA80065822AF4B06A06F8010B6168013961600D
:104EB8000029C4BF0EF10101216040F33E81B9F120
:104EC80001097FF420AD1AF4807F0A950C96654697
:104ED800089F9B460ED009998E4206D916F8011DE7
:104EE800404622460C9604F07BFD0C9A099B9A4298
:104EF8003FF480AB1AF0100200F04081099B059E38
:104F0800ED1ADDF830C0AD196544FFF748BB0AF467
:104F1800C061B1F5007FD6D12AF4007A10254AF491
:104F2800A06AC0E73BF91550082DCCDD2AF4386A91
:104F3800B9E70A2DC7DD2AF4386AB4E73BF91550FA
:104F48002AF4386AAFE71AF0800FBCD02AF0800A3A
:104F5800A9E7A9F5AE7340F25D19013BBEE44AF03A
:104F6800040A3A78FFF763BB42F6A5520023C0F65D
:104F780000024FF0030C0A930692CDF814C072E4B5
:104F88003A786C2A0ABF4AF0020A4AF0010A17F86E
:104F9800012FFFF74CBB1AF0100F7FF400AB1AF08B
:104FA800040F00F02E82DBF800300BF1040B1D809B
:104FB800FFF7F5BA48F6B1200821C0F60000032231
:104FC8000A91069005924EE401FB09F9A9F130090E
:104FD80091443A78FFF72BBB0422059243E44AF048
:104FE800020A3A78FFF723BB48F6B1200821C0F639
:104FF800000003224AF0010A06900A91059232E461
:1050080048F6B1231020C0F6000303214AF4007AC1
:1050180006930A90059126E4394669A802F0CCFB6C
:105028004AF0400A4FF0010CCDF814C007461AE4C4
:1050380000204AF0400A059015E448F6B1230A20FA
:10504800C0F6000303210A90069305910BE49B1810
:1050580042F6A550C0F600005B78069003F0030303
:10506800012B08BF4AF0010A0A2103220A9105927E
:10507800FFF7F9BBFBF796FE4FF0FF360796FFF7F1
:10508800BBBA4AF0100A3A78FFF7D1BA48F6B1210C
:105098001022C0F6000103234AF4087A06910A9206
:1050A8000593FFF7E0BB02230593FFF7DCBB4FF046
:1050B800FF330793FFF7A0BA1AF8011D04F090FC1C
:1050C800099B404622465345F6D3FFF793BA00940E
:1050D8004046DBF8001001224B4604F0E5FC0028AE
:1050E8003FF4A7AB079B0BF1040B4519013307935A
:1050F800FFF755BA1AF8011D04F072FC099F4046E3
:1051080022465745F6D3FFF775BA1AF8011D04F081
:1051180067FCDDF824C040462246D445F5D3FFF7A6
:1051280069BA184621460392029304F09FFC039A39
:10513800029B00283FF49EADA0E54046214602931D
:10514800CDF80CC004F092FC029BDDF80CC00028DE
:105158003FF4B5AEB7E6BBF1020F7FF486AE4FF071
:10516800030B7AE500228BF80020079ECAEB0505A1
:105178005D449B4601360796FFF711BA0C9E4046E0
:10518800327009990A9B069EB0471AF0200F40F02A
:10519800F7801AF0040F00F08781DBF800300BF17C
:1051A800040B1880079A01320792A7E6082200210B
:1051B800A9A8FCF7EDFB1AF010014FF0000A12BF86
:1051C800ADABDBF800200BF1040B0DF1440C08919A
:1051D800CDF830C009970CBF05920593B9F1000FBF
:1051E8000BD1099F089900297FF4D9A9059A079B33
:1051F800116001330793FFF7D2B9236832681B782F
:10520800D3185B7813F0080FEBD101F007FB50457A
:105218003FF40FAB236811AA67684046059913F855
:1052280001EB013F6760A9AF009702F80AE00AF1B5
:10523800010A2360534601F023FBB0F1FF3F3FF41E
:10524800F8AA002840F00881DDF814C0CCF8000066
:105258000599086801F0A0FA002840F03D81089FF0
:10526800554409F1FF39002F40F04C810598BA46A2
:1052780004300590F4E000210822ABA8FCF788FB75
:105288001AF0100005900DF1440A06BFDBF8003053
:105298000BF1040B0023CDF824B0DDF814B0002680
:1052A8000C954D460897994601F0B8FAB0423FF47C
:1052B800C0AA2368ABAFD4F804C04046494652465A
:1052C80013F801EB0CF1FF3CC4F804C000970AF88E
:1052D80006E001362360334601F0D2FAB0F1FF3F11
:1052E8003FF4A7AA00282ED1BBF1000F01D1C9F8BD
:1052F80000B00C98013D80190C90BBF1000F2CD127
:1053080009F104095E466368002B0EDD002DCBD140
:105318000C9D089FDDF824B0059900297FF43FA96A
:10532800079A01320792FFF73AB94046214604F03E
:105338009DFB0028EAD00C9D089FDDF824B0002EC4
:10534800EAD0FFF776BA10F1020FDCD00C98013DD5
:1053580080190C90BBF1000FD2D00026D3E7BAF128
:10536800000F3FF447A95544FFF719B92AF4607AAA
:1053780017B1013F09F1010905980130059094E53D
:10538800DBF800300BF1040B18600BE765293FF4DC
:10539800B2AC40462246CDF80CC0013D04F020FBDB
:1053A8001AF8011DDDF80CC0A5E427F4F067012602
:1053B8004FF0000851E422684E44C9EB0303751905
:1053C800636002EB09032360FFF7E9B805980E99BB
:1053D800421A3FF4A8AC5242CDF834A00D9B44F2D7
:1053E8003831049EC0F60301CDF80CC0B34224BF87
:1053F8000DF5CB700D900D98FAF704FFDDF80CC091
:1054080091E41AF0010F0CD11AF0020F09D0DBF861
:1054180000102A46EB170BF1040BC1E90023FFF734
:10542800BEB8DBF800300BF1040B1D60FFF7B7B80E
:1054380027F4F0674FF0010B4FF000080DE40D9EC4
:1054480040460A23CDF80CC0711CFDF7A7FC0F9944
:10545800DDF80CC0421AC1E710F1020F7FF4F8AE74
:105468006368002B3FF7BAAE4046214604F0FEFAC7
:1054780000283FF4B3AE099FBAF1000F7FF4D9A911
:10548800B0E6DBF800900BF104060390029102F0FD
:105498004BF9039A029B00282FD01046194606F0B4
:1054A8008BFDC9F8000056E41AF001027FF468AFDA
:1054B8001AF0020F3FF464AF06980B99884223D084
:1054C800404609990A9B03F007FADBF800300BF114
:1054D800040B1860596065E6099FBAF1000F3FF4A4
:1054E80081AE11AA92441AF8011D4046224604F0E2
:1054F80077FA0C9B9A45F6D174E602F099F9C9F847
:10550800000028E48246ABE7404609990A9B03F06D
:105518008BFBDAE740F2A4030022C2F2000310B5C5
:1055280082B004466946186801F01AF90028B8BF25
:105538004FF0FF3002DB1CB10098206002B010BDB4
:105548000098FBE7704700BF704700BFF0B5141E16
:105558009BB0054620DB4FF402720091ADF80C2099
:105568001A4604916946209B08BF26464FF0FF372C
:1055780018BF661EADF80E7002960596FDF7CCFCB6
:10558800B0F1FF3F05DB14B1009B00221A701BB07D
:10559800F0BD8B232B60F6E78B234FF0FF302B6099
:1055A800F5E700BFF0B540F2A40483B0C2F20004EE
:1055B80007460E46154600932068394632462B4664
:1055C800FFF7C4FF03B0F0BD2DE9F0410C4686B0EB
:1055D800054690461E46B1B140F2A853C2F20003F8
:1055E8001F6801F015F900962146424603462846F1
:1055F800B847B0F1FF3F03D1002333608A232B6003
:1056080006B0BDE8F08140F2A853C2F200031F685B
:1056180001F0FEF8009603A9224603462846B8473B
:10562800E7E700BF2DE9F043074687B088461546EF
:10563800E8B140F2A40440F2A853C2F20003C2F257
:1056480000041E68D4F8009001F0E2F8009539468D
:10565800424603464846B047B0F1FF3F04D12368AD
:1056680000222A608A221A6007B0BDE8F08340F25F
:10567800A40440F2A853C2F20003C2F200041E6858
:10568800D4F8008001F0C4F8009503A93A4603460F
:105698004046B047E0E700BF10B582B0049C0093D5
:1056A8004FF0FF33019405F077F802B010BD00BF4A
:1056B80030B540F2A40483B0C2F200040D4601469E
:1056C80000922A4601934FF0FF33206805F064F8F2
:1056D80003B030BD034621B1FF2A04D80A70012067
:1056E8007047084670478A224FF0FF301A607047AB
:1056F8002DE9F04140F2A854C2F2000482B01E46DF
:10570800054688461746246801F082F80096414607
:105718003A4603462846A04702B0BDE8F08100BFDC
:1057280038B545F68C24C2F20004054608461146F1
:105738001A46002323602AF0F5F9B0F1FF3F00D0A4
:1057480038BD2368002BFBD02B6038BD38B545F633
:105758008C24C2F2000405460846002323600CF09E
:105768000FF9B0F1FF3F00D038BD2368002BFBD004
:105778002B6038BD000000002DE9F04F83B00369AD
:1057880081460D6901919D4200F38980EA1C01F16F
:10579800140400F11408013D92008B1882181F1D93
:1057A80059685068013105F0D7FC064600283CD0FE
:1057B800002042462346864653F804CB11681FFA58
:1057C8008CFB4FEA1C4C1FFA81FA0BFB060BD644E4
:1057D8000CFB06F000EB1B401FFA8BFBCBEB0E0A11
:1057E8001FFA80FE000CCEEB114E9F420EEB2A4EA4
:1057F8001FFA8AFC4CEA0E414FEA2E4E42F8041B6F
:10580800DAD22A1D09EB8203596871B998450AD280
:1058180059F822203AB9043B02E053F8042912B996
:10582800013D9845F9D3C9F810504846019901F04F
:105838003FFB00282FDB013643464FF0000C54F89D
:10584800040B19681FFA80FA000C8AB2C0EB1141E8
:10585800CAEB0202A742944401EB2C421FFA8CFCCB
:105868004CEA02414FEA224C43F8041BE7D22A1DB6
:1058780009EB8203596871B998450AD259F8222070
:105888003AB9043B02E053F8042912B9013D98459E
:10589800F9D3C9F81050304603B0BDE8F08F0020A6
:1058A800FAE700BF2DE9F04F9FB0456A04469046DD
:1058B80099462B9E002D00F090832B6853B16A689F
:1058C8000125194695409D605A6001F0AFF8636A5A
:1058D80000221A60B9F10005C0F2D38000233360BA
:1058E80000231A46C7F6F073C7F6F07205EA0303F9
:1058F800934200F0AF800022002340464946CDE99C
:105908000289012606F0DEFA88B916F0FF0F12D1D7
:105918002A9801232C99036044F23430C0F603001E
:1059280011B17B4B581E0B601FB0BDE8F08F0026ED
:1059380016F0FF0FECD02046DDE902231CA90091E8
:105948001DA9019101F0C8FBC5F30A568246002E35
:1059580000F0AC800398A6F57E761D9F073E20F0E8
:105968007F43002123F47003169143F07E5343F4E0
:10597800E00303930023DDE902010022C3F6F87374
:1059880005F084FE5CA3D3E9002306F033F85CA39A
:10599800D3E9002305F07CFECDE90201304605F08D
:1059A800C3FF59A3D3E9002306F024F802460B46A7
:1059B800DDE9020105F06CFECDE9020106F0B4FA5A
:1059C800002200230546DDE9020106F085FA40B110
:1059D800284605F0A9FFDDE9022306F073FA00B9AD
:1059E800013D162D00F2558242F6B0414246C0F6FE
:1059F80003014B4601EBC501D1E9000106F08AFA23
:105A0800002800F00083013D00201590013FBE1BD7
:105A180000F1F48200200B960D90002DC0F2E68272
:105A28000B990022119549190F920B91289A092A6E
:105A380070D8052A40F390860027043A28922898BF
:105A4800831E032B00F20A84DFE813F00204EC0340
:105A5800CC0305042A9842F20F73036044F24C30D9
:105A6800C0F60300B8F1000F11D02C9900293FF4BB
:105A78005BAFC278C31C0AB100F108032C9A13600B
:105A880052E725F000450123A946336028E744F290
:105A9800403244F24C33C5F31300C0F60302C0F69B
:105AA800030300280CBF10461846DEE71D9F1C9B09
:105AB800FB1803F586639E1C202EDCBFC6F1200070
:105AC80008FA00F007DDC6F140001E3B854028FAC1
:105AD80003F345EA03000122169205F015FFA6F527
:105AE8008666033E0B460246CDE90223039BA3F1DB
:105AF800F87303933EE700BF61436F63A787D23F04
:105B0800B3C8608B288AC63FFB799F501344D33FA4
:105B18003543030800204FF0FF3107460122289043
:105B28000E9110920A912990666A002373602046AC
:105B3800716800F047FF636A30601B680C93002FA0
:105B480000F0DE80002D40464946CDE90889CDE9C0
:105B5800020140F32E8442F6B04305F00F02C0F66E
:105B680003032E1103EBC20316F0100F08BF4FF00A
:105B78000208D3E90001CDE9120140F04782BEB125
:105B880042F67857DDE91223C0F6030716F0010F35
:105B98001046194607D0D7E9002308F1010805F097
:105BA80029FF02460B4608377610EFD1CDE91223BC
:105BB800DDE90801DDE9122306F046F8CDE9080120
:105BC8001599002938D00023DDE908010022C3F621
:105BD800F073012606F080F9002800F001830A9A84
:105BE800002AD4BF002606F001062EB30E9B002B18
:105BF80040F3828000230022C4F22403DDE9080177
:105C080005F0F8FECDE9080108F10100691E1291BE
:105C180005F08AFE02460B46DDE9080105F0EAFEBA
:105C280000230022C4F21C0305F032FDDDF838B071
:105C38008046A1F150793CE2404605F075FEDDE969
:105C4800082305F0D7FE00230022C4F21C0305F048
:105C58001FFD0A9AA1F150768046B146002A40F00D
:105C6800258200230022C4F21403DDE9080105F0AF
:105C78000DFD42463346CDE9080106F04BF90028F0
:105C880040F00F824246DDE9080106F1004306F0C4
:105C980023F9002830D0DDF828B0CDF820B0299BB2
:105CA80000270C9EDD435946204600F0BFFE0899A8
:105CB80071B13B1E18BF01238F420CBF002303F0B4
:105CC8000103002B40F05E832046089900F0AEFEE9
:105CD8002046514600F0AAFE0023337001352A9A67
:105CE8002C9B1560002B00F018841E600C981BE696
:105CF800189DDDF85CA0089CDDE902018046894614
:105D08001C9BDF43FF0F0E2DCCBF002707F00107B8
:105D1800002F00F0C18042F6B0432999C0F6030372
:105D28000A9A03EBC503CF0FD3E90001002ACCBFC1
:105D3800002707F00107CDE90201002F40F09E81FE
:105D480002460B4640464946CDE9048905F07CFFEA
:105D580006F0EAF80C9E814605F0E6FDDDE902232F
:105D680005F048FE02460B46DDE9040105F08EFC0D
:105D780009F13003CDE9040106F8013B0A9A012A2A
:105D880056D000230022C4F224034FF0010805F086
:105D980031FE00220023CDE9040106F093F800B19A
:105DA800B84618F0FF0F93D00A9937460C98A046CA
:105DB800079500EB010BCDF828A05D46DDE904ABA3
:105DC8000DE005F017FE0022002382468B4606F000
:105DD80079F800B1002414F0FF0F00F00F84DDE91A
:105DE800022350465946012405F02EFF06F09CF880
:105DF800814605F099FDDDE9022309F1300605F039
:105E0800F9FD02460B465046594605F03FFC002373
:105E180007F8016B0022AF42C4F224033E468246D3
:105E28008B46CED1CDE904AB4446079DDDF828A0CA
:105E3800DDE9040102460B4605F02AFCCDE9040120
:105E4800DDE90423DDE9020106F046F860B9DDE981
:105E58000201DDE9042306F035F800283FF438AFE5
:105E680019F0010F3FF434AF12950C98334613F82C
:105E7800011C5A1E1E461346392940F0E18383420D
:105E8800F5D10C983121129B5D1C302303701170E1
:105E98001EE701211591B9E51099002940F0C78046
:105EA800109B0F9F0D9E0893002E0B98D4BF0023C4
:105EB80001230028D4BF002303F001034BB103469C
:105EC8000D99B342A8BF3346F61AC91AC01A0D91E4
:105ED8000B900F9A002A1ADD109B002B00F0948378
:105EE800002F10DD08993A46204600F039FF524647
:105EF80008902046089900F09FFE514683462046A8
:105F080000F094FDDA460F98C21B40F0848301210B
:105F1800204600F087FE11990029834605DD594681
:105F28002046119A00F01CFF8346289A012A40F364
:105F38009E8100271199002940F0F28201230B9AD3
:105F48009B1813F01F0300F02282C3F12003042BD7
:105F580040F3F683043B0D98F618D218C0180B923C
:105F68000D900D9B002B05DD514620461A4600F08A
:105F780049FF82460B98002805DD594620460B9AB2
:105F880000F040FF83461599002940F0D3822899F4
:105F98000A9A0229D4BF00230123002ACCBF002378
:105FA80003F00103002B00F07C81002A7FF477AE18
:105FB800594605220A9B204600F054FD8346504668
:105FC800594600F075FF00287FF769AE0C9E312313
:105FD8000135002706F8013B65E61020FBF790F82D
:105FE8006062456085600560C56073E40D9B68422A
:105FF80000210F905B1B11910D9317E5764200234A
:106008000D960B9309E500221592FFE442F67853AA
:106018004046C0F60303494606F00F064FF0030852
:10602800D3E9082305F010FECDE90801A7E5289A71
:10603800012A40F3F6820A990F9A4B1E9A42A8BF8A
:10604800C3EB02070A9ABFBF0F981199C0EB03036D
:10605800C918BEBFC01811910F90002AC0F2F9826A
:106068000D9E0A9B0D9A20460121D2180D920B9A7B
:10607800D2180B9200F0D6FD089015E70A9B002B6A
:1060880040F0D88200230022C4F21403DDE90201A3
:1060980005F0B0FC42464B4605F032FF00287FF47D
:1060A800FAADDDF828B0CDF820B08FE7DDF828B0DC
:1060B8001295109B002B00F0AF8142F6B0430021EF
:1060C800C0F60303002003EBCB03C3F6E0710C9E7C
:1060D80053E9022305F0B8FD42464B4605F0D6FACF
:1060E80080468946DDE9080105F01EFF074605F0F0
:1060F8001BFC02460B46DDE9080105F0C7FA07F16B
:106108003003CDE90801404606F8013B4946DDE980
:10611800082305F0FFFE002840F0FC810021DDE99E
:1061280008230020C3F6F07105F0B0FA02460B46CA
:106138004046494605F0EEFE00287FF496AEBBF1D6
:10614800010F7FF7D9AD0C98374618958344CDF8E1
:106158005CA05D46DDE908AB08940FE00021002053
:10616800C3F6F07105F092FA42464B4605F0B4FECC
:10617800002840F06A82AF423FF4BAAD0023002203
:10618800C4F224034046494605F034FC00230022AB
:10619800C4F22403804689465046594605F02AFC35
:1061A8008B46824605F0C0FE044605F0BDFB303440
:1061B80002460B465046594605F068FA42464B4699
:1061C80007F8014B3E4682468B4605F085FE52464F
:1061D8005B460028C2D0DDF85CA0089C129D77E5DC
:1061E8000026FCE40123109329990029C2BF8B469D
:1061F8000E910A9140F3B481666A0022BBF1170F31
:10620800726040F2A18204235B00013203F11401A1
:106218005945F9D90A9B72600E2B8CBF002707F0ED
:10622800010784E400231093299828180E9000F1A0
:10623800010BBBF1000FC8BFCDF828B0DCDCBBF107
:106248000E0F8CBF002707F00107CDF828B06BE4CC
:1062580000201090C8E701221092E5E74FF0FF33C5
:10626800002701200E9310900A9329975CE4B8F157
:10627800000F7FF45EAEC9F313034746002B7FF48B
:1062880059AEC7F6F07309EA03031F46002B3FF423
:1062980051AE0D9B01270B9801330D9301300B90E4
:1062A80048E61098002800F06181002E05DD2046A0
:1062B8000899324600F0A6FD0890002F40F0ED81C5
:1062C800089802900A9908F001020C9E089F71181C
:1062D8000A920B91089559465046FFF74DFA3946F0
:1062E8004FF0010930300790504600F0E1FD594663
:1062F800029A0546204600F0F9FDC3688046002B47
:106308003AD02046414600F091FB289B59EA030306
:1063180003D10A98002800F0F381002DC0F29D8176
:106328002898284303D10A99002900F09681B9F1E9
:10633800000F00F3D281079A06F8012BB0460B9B99
:106348009E4200F0C68151460A220023204600F0F2
:1063580089FB82460298874222D039460A220023C6
:10636800204600F07FFB02990A22002307462046B8
:1063780000F078FB0290AEE75046414600F098FDE9
:106388008146BEE72046394600F050FB9CE41C23BA
:106398000D99F6180B9AC9180D91D2180B92E0E5D1
:1063A800394620460A22002300F05CFB074602908B
:1063B80091E76E42002E00F01D8106F00F0342F6B1
:1063C800B042C0F60302DDE9080102EBC303D3E9DA
:1063D800002305F00FFB3611CDE9080100F00A8112
:1063E80042F678574FF00208C0F6030702460B46FC
:1063F80016F0010F1046194607D0D7E9002308F117
:10640800010805F0F7FA02460B4608377610EFD177
:10641800CDE90823FFF7D4BB0BF1FF321792179889
:1064280042F6B041C0F6030142464B460C9E01EBD2
:10643800C001D1E9000105F0DDFACDE91801DDE977
:10644800080105F071FD074605F06EFA0B46024695
:10645800DDE9080105F01AF9BBF1010F07F1300376
:10646800CDE9080106F8013B2BD00C991B9501F1E9
:10647800FF390F46D944DDE90801D3464D46B246F7
:10648800264600230022C4F2240305F0B3FA894605
:10649800804605F049FD044605F046FA30340246C8
:1064A8000B464046494605F0F1F807F8014FAF4260
:1064B800E7D1179A34461B9D5646B618DA46CDE9F9
:1064C800080100230022C3F6E073DDE9180105F096
:1064D800DFF802460B46DDE9080105F01BFD002840
:1064E8007FF4C3AC0021DDE918230020C3F6E07176
:1064F80005F0CCF802460B46DDE9080105F0ECFC96
:1065080000283FF4F9AB33461E46013B16F8012C30
:10651800302AF9D0129DFFF7DBBB0C98FFF704BABD
:10652800DBF810300BEB8303186900F029FBC0F18E
:10653800200304E55046594600F0BAFC0028BFF68F
:1065480026AD51460A222046002300F08BFA109A05
:10655800013D8246002A40F0E9800E980A9016E52F
:1065680001220E920A922992FFF7DEBA0C9E0127A9
:10657800DDF82890029502E000F074FA8246594648
:106588005046FFF7F9F80A2200234F45514607F114
:10659800010700F13005204606F8015BB046EBDB49
:1065A80007950027029D51460122204600F02AFC4B
:1065B8005946824600F07CFC00280FDD0C9A4646BE
:1065C80008F1FF3816F8013C392B61D19045F6D116
:1065D8000C98312301350370FFF765BB03D1079A87
:1065E80012F0010FEAD1464618F8013D302BFAD0D7
:1065F800FFF759BB4FF00208FFF7E2BA079D444680
:10660800DDF828A0FFF764BB514620460F9A00F03A
:10661800A7FB82467BE45146204600F0A1FB824658
:1066280075E4169800284ED003F586630F9F033350
:106638000D9E17E54FF0000BCDF820B0FFF72FBBEC
:106648000131129D1170FFF743BBDDF85CA0089C77
:106658000BE40D9B9E1A002304E5B9F1000F089D79
:106668000FDD51460122204600F0CCFB59468246F8
:1066780000F01EFC002853DD079B392B39D001336D
:10668800079302980799089006F8011BFFF70BBBC0
:10669800013388F80030FFF706BB089A2046516896
:1066A80000F090F9089B03F10C011A69023292007C
:1066B80006460C30FBF76AF820463146012200F006
:1066C800A1FB0290FEE51D9B0F9F0D9EC3F13603B3
:1066D800C8E40299089D089165E7079A089D392A38
:1066E80007D0029907980891431C06F8013BFFF769
:1066F800DABA029BB0460893392308F8013B5DE7F4
:1067080007992B46089D3929F3D0002B01DD01316B
:106718000791029A079B089206F8013BFFF7C3BA54
:10672800AFD1079A12F0010FABD0A5E7002320469E
:1067380008990A2200F096F90E9B0A93089026E41D
:106748003FF40FAC1C3323E60A990E298CBF0027AF
:1067580007F00107FFF7EBB90127FFF770B900BF92
:1067680038B545F68C24C2F20004054608461146A1
:10677800002323600BF02AF9B0F1FF3F00D038BDA9
:106788002368002BFBD02B6038BD00BF40F2B0500F
:10679800C2F20000704700BFFF289FBF40F2AC5311
:1067A800C2F200031B6818189ABF407800F008006E
:1067B8000020704710B514463AB144F250311046E3
:1067C800C0F60301FBF758FE20B944F22030C0F6AA
:1067D800030010BD44F220312046C0F60301FBF748
:1067E8004BFE20B944F22030C0F6030010BD44F23D
:1067F800F8212046C0F60301FBF73EFE44F22033A1
:10680800C0F6030300280CBF1846002010BD00BFC7
:1068180040F2F050C2F20000704700BF40F2F0535F
:10682800C2F20003186A7047004870471406002037
:1068380000207047004870473406002040F2A40347
:106848000A46C2F2000301461868B3E700487047D9
:106858003406002038B545F68C24C2F200040546FB
:10686800084611461A46002323600BF07BF8B0F166
:10687800FF3F00D038BD2368002BFBD02B6038BD0C
:106888002DE9F04383B014460546894698460A9E8A
:10689800BAB140F26C63C2F200031F68FFF7B8FF99
:1068A800019649462246434600902846B847B0F12B
:1068B800FF3F03D1002333608A232B6003B0BDE878
:1068C800F08340F26C63C2F200031F68FFF7A0FF79
:1068D80044F2F82201962146C0F6030201230090F3
:1068E8002846B847E3E700BF2DE9F0470D4682B0D8
:1068F800814617461E46F9B140F26C6340F2A40483
:10690800C2F20003C2F20004D3F800A0D4F8008059
:10691800FFF77EFF019649462A463B4600904046CF
:10692800D047B0F1FF3F04D12368002232608A22A9
:106938001A6002B0BDE8F08740F26C6340F2A4042C
:10694800C2F20003C2F20004D3F800802768FFF700
:106958005FFF44F2F82201962946C0F6030201239C
:1069680000903846C047DCE782B071B110460AB9DA
:1069780002B070476FF00100002BF9D013780B605C
:106988001078003818BF0120F2E701A9EEE700BF30
:106998002DE9F04140F26C64C2F2000482B01E4658
:1069A8000546884617462468FFF732FF089B41468C
:1069B8003A460193334600902846A04702B0BDE806
:1069C800F08100BF70B50646446A0D465CB1E368C5
:1069D8009BB153F82500E0B1026843F82520002355
:1069E8000361C36070BD1020FAF78AFB00230446D8
:1069F8007062436083600360C360304604212122D3
:106A080003F054FF736AE060DB68002BE1D118469D
:106A180070BD012430462146AC40621D920003F04F
:106A280045FF0028F4D045608460D8E730B50446B7
:106A3800456A83B055B139B1636A4A68DB6853F86F
:106A48002200086043F8221003B030BD10200191E5
:106A5800FAF756FB01996062456085600560C5607C
:106A6800E9E700BF2DE9F0410C4605460E6901F142
:106A7800140082B00021076801311FFA87FC3F0C1F
:106A88000CFB023307FB02F707EB13471FFA83FCE3
:106A98003B0C8E424FEA074808EB0C0740F8047B92
:106AA800E9DC3BB1A268964208DA04EB86020136BB
:106AB80026615361204602B0BDE8F081616828462E
:106AC80001930131FFF77EFF226904F10C010232C4
:106AD800920007460C30FAF759FE214628463C46F4
:106AE800FFF7A4FF019BE0E72DE9F84348F6396575
:106AF8001F46C3F6E30508330E460446904685FB59
:106B08000315DB17C3EB6503012B37DD01220021D9
:106B1800520001319342FBDC2046FFF753FF089BEC
:106B280043610123B8F1090F0146036122DD06F133
:106B3800090946444D4615F8013B0A222046303BD8
:106B4800FFF790FFB5420146F5D109EB0806083E6C
:106B580047450CDDF719C8EB070716F8013B0A2271
:106B68002046303BFFF77EFFBE420146F5D108467E
:106B7800BDE8F8830A364FF00908E9E70021CBE7BA
:106B8800020C034619D10304102013F07F4F01D1E2
:106B980008301B0213F0704F01D104301B0113F0B1
:106BA800404F01D102309B00002B05DB13F0804FD2
:106BB80001D001307047202070470020E5E700BF72
:106BC8000368024613F0070009D013F0010F21D122
:106BD80013F0020F22D19B0802201360704799B26C
:106BE80009B91B0C102013F0FF0F01D108301B0A44
:106BF80013F00F0F01D104301B0913F0030F01D15B
:106C080002309B0813F0010F02D15B0804D0013059
:106C18001360704700207047202070475B080120F0
:106C28001360704710B50C460121FFF7CBFE012217
:106C38004461026110BD00BF2DE9F04F90460F6915
:106C48000D46166985B0B742BFBF45463A46374636
:106C58001646AB68B8BF8846F41969689C42C8BF35
:106C68000131FFF7AFFE00EB840300F1140C14337D
:106C780001909C45029306D202996346002243F88C
:106C8800042B9942FBD808EB860605EB870708F129
:106C98001408143614351437B04500954DD20394B2
:106CA80058F8044BA0B2F0B1009A6346002452F899
:106CB800045B19681FFA85FA2D0C1FFA81F9090C73
:106CC80000FB0A9900FB0511A14401EB19411FFAC9
:106CD80089F90C0C974249EA014543F8045BE6D868
:106CE8001C6058F8044C240C21D0DCF800206046C5
:106CF800009BE14611460025B3F800A01FFA82FB6D
:106D08000AFB045505EB11454BEA054240F8042BF4
:106D180053F8042B59F8041F120C1FFA81FA02FBCE
:106D280004A202EB1542150C9F42E5D802604645C5
:106D380002D90CF1040CB3E7039C002C0ADD02997C
:106D48000B1F51F8042C1AB104E053F8042D0AB9AA
:106D5800013CFAD1019A1046146105B0BDE8F08FE4
:106D680012F003032DE9F04115460446884628D160
:106D7800AD101AD0666A002E2FD0B7682FB936E04A
:106D88006D1012D03E689EB1374615F0010FF7D04E
:106D980041463A462046FFF74FFF41460646204601
:106DA800FFF744FE6D10B046ECD14046BDE8F081D7
:106DB80039463A462046FFF73FFF386007460660E7
:106DC800E3E742F6A0425E1EC0F60302002352F833
:106DD8002620FFF747FE8046CAE71020FAF790F909
:106DE800002306466062436083600360C3602046F8
:106DF80040F27121FFF716FF0023B06007460360D9
:106E0800C3E700BF2DE9F84356110D690C468B689E
:106E1800904601358146AD1949689D4203DD5B0006
:106E280001319D42FBDC4846FFF7CCFD002E0746AA
:106E380000F114020ADD00231946013342F8041B4D
:106E4800B342FAD107EB830303F11402266904F174
:106E5800140104EB8606143618F01F081AD0C8F17E
:106E6800200E00200B6803FA08F3184342F8040BBD
:106E780051F8040B8E4220FA0EF0F3D8106000B1DE
:106E880001354846013D21463D61FFF7CFFD3846B3
:106E9800BDE8F88351F8043B8E4242F8043BF0D930
:106EA80051F8043B8E4242F8043BF3D8E9E700BFAF
:106EB80003460A69006930B4801A0FD1043203F11D
:106EC800140592009B1889180433043153F8044DB3
:106ED80051F8042D944203D19D42F7D330BC70473A
:106EE80038BF4FF0FF30F9D30120F7E72DE9F84F0D
:106EF80089460446114648469046FFF7D9FF051EC5
:106F080064D0BCBF4B46C1462046B8BF9846D9F8A6
:106F18000410ACBF4FF0000A4FF0010AFFF752FD12
:106F2800D9F8106009F11405D8F8103008F11407E1
:106F3800002409EB860909F1140983461430CBF8BB
:106F48000CA008EB830A0AF1140A55F8041B03463F
:106F580057F8040B2A461FFA81F81FFA80FC000C28
:106F6800CCEB080CC0EB1140644400EB2440A4B205
:106F780044EA00410414BA4543F8041B1846E4D80F
:106F8800A9451F4614D952F8041B88B2090C2418C5
:106F980001EB2441A4B244EA01400C14914543F8A2
:106FA800040BF0D8EB434B4423F003030433FB18E2
:106FB80053F8042C043B22B953F8042D013E002A4F
:106FC800FAD0CBF810605846BDE8F88F204629461D
:106FD800FFF7F8FC01238346456103615846BDE885
:106FE800F88F00BF0023C7F6F07301EA0303A3F18B
:106FF8005073002B02DD1946002070475B421B15B9
:10700800132B0DDD143B00211E2B02DD0123184636
:1070180070470122C3F11F0312FA03F318467047A1
:107028004FF40022002052FA03F170472DE9F04195
:1070380000F1140604690F46043450F8245000EB9C
:107048008404A0462846FFF79BFD0A28C0F12003C8
:107058003B6015DCC0F10B0135FA01F7A64247F099
:107068007E5747F4E00333D254F8044C34FA01F164
:107078001530854041EA050210461946BDE8F08101
:10708800A64221D300210B3802BF45F07E550A469F
:1070980045F4E003F0D08540C0F1200745F07E5567
:1070A800B44221FA07FC45F4E00545EA0C0311D97E
:1070B80054F8044C34FA07F711FA00F0194647EA75
:1070C80000021046BDE8F081043C58F8041CDAE7D9
:1070D8000021CDE70027EFE72DE9F04383B0012138
:1070E8001D4614460A9F0B9EFFF76CFCC5F30A5910
:1070F80025F07F4323F4700300938046B9F1000F15
:1071080002D043F480130093002C25D002A840F845
:10711800044DFFF755FD002836D1019A009BC8F8A9
:107128001420002B0CBF01240224C8F81830C8F81A
:107138001040B9F1000F1DD108EB8403A0F586605B
:107148000238386018696401FFF71AFD241A3460A0
:10715800404603B0BDE8F0836846FFF731FD0123E0
:107168001C46C8F81030009BC8F814302030B9F11C
:10717800000FE1D0A9F58669C0F13503A9F103092B
:10718800484438603360E3E7009BC0F1200201996E
:1071980013FA02F2C3400A430093C8F81420C0E768
:1071A8002DE9F04182B0884601A90646FFF73EFF67
:1071B8000D46044669464046FFF738FFD8F810E008
:1071C800D6F810C0DDF80480CEEB0C0CDDF800E03A
:1071D8004FEA4C1CCEEB080EE644BEF1000F4FEA16
:1071E8000E5EC4BF0EEB05073D460B46D8BFCEEB7F
:1071F80001010246DCBF0B4602462946204604F040
:1072080023FD02B0BDE8F081172810B504460CDD57
:1072180000210020C3F6F07100230022C4F22403E9
:1072280004F0E8FB013CF7D110BD42F6A043C0F6DC
:10723800030303EBC003D3E9040110BD70B40139A3
:10724800166902F114034911013102EB860614365E
:1072580000EB8101B3420CD2044653F8045B9E4212
:1072680044F8045BF9D8B31A153B23F0030304333D
:10727800C018814204D9002340F8043B8142FBD85E
:1072880070BC704702694B1110B49A4211DB0FDDD4
:1072980011F01F010CD01A4600EB83035B6933FA27
:1072A80001F414FA01F1994203D0012010BC70478F
:1072B8001A46043200F1140100EB82031C1DA1429E
:1072C8000BD250F82220002AEFD1994205D253F868
:1072D800042D002AE9D19942F9D30020E6E700BF3E
:1072E80038B545F68C24C2F2000405460846114616
:1072F8001A46002323600AF027FBB0F1FF3F00D0B5
:1073080038BD2368002BFBD02B6038BD2DE9F04F2A
:107318000D4683B007469046002900F0558108F1D4
:107328000B04A1F1080AFAF717FE162CDAF8043054
:1073380000F29780102200201446444538BF40F0E0
:107348000100002840F0468123F0030B9345A4BFB9
:107358000AF108085E466EDA40F298190AEB0B014A
:10736800C2F20009D9F808E08E4500F038814E686D
:1073780026F0010C8C44DCF804C01CF0010F18BF87
:10738800014673D013F0010F40F0928055F8083C85
:10739800C3EB0A0CDCF8043023F00303002900F0E7
:1073A800D180714500F04F815B44C618B24200F3AA
:1073B800CA80CB68E0468968ABF10402242ACB6016
:1073C8009960DCF80C3058F8081FCB60996000F21F
:1073D8009681132A414621D92B460CF1100153F806
:1073E800040BCCF8080068681D1D1B2ACCF80C009B
:1073F80014D958682B1D0CF11801CCF810006868D6
:107408000835242ACCF8140008D15B680CF1200157
:10741800CCF818306B680835CCF81C302A460B4677
:10742800E24652F8040B43F8040B68684860526857
:107438005A60DCF80430301B0F2824D80AEB060207
:1074480003F0010343EA0606CAF80460536843F0F0
:10745800010353603846FAF781FD404603B0BDE8A2
:10746800F08F24F007042246E00F66E726F00300B9
:1074780000EB0B06B24285DCCA680AF10808896885
:10748800CA609160D7E70AEB040103F001030A1808
:1074980043EA040440F00100CAF804404860384652
:1074A8005368083143F001035360F9F7EDFCD1E765
:1074B80041463846F9F734FE80460028CAD0DAF843
:1074C8000430A0F1080223F0010151448A4200F07F
:1074D8000E81ABF10402242A00F2B180132A294656
:1074E80003461DD92C4654F8043B211D40F8043BA3
:1074F800031D6E681B2AC8F8046011D9D4F804E08B
:107508000E1D1C1DC0F804E0486808315860083397
:10751800242A05D1726862604A6808315A600833C3
:1075280008461A4650F8044B42F8044B496859601B
:107538004368536038462946F9F7A6FC3846FAF7F7
:107548000DFD8AE75B449A42B2DCE046DCF80C1099
:10755800ABF1040258F8080F242AC16088605FD88C
:10756800132A404621D929460CF1100051F8046B22
:10757800CCF808606E680D1D1B2ACCF80C6014D975
:107588004E68291D0CF11800CCF810606E6808359B
:10759800242ACCF8146008D14A680CF12000CCF8F1
:1075A80018206A680835CCF81C2029461E46024671
:1075B800E24651F8043B42F8043B6B6843604B6871
:1075C8005360DCF8043036E7114603B0BDE8F04FED
:1075D800F9F7A6BD0C234FF000083B603DE7DEF845
:1075E800040004F1100C20F0030000EB0B016145CE
:1075F800B8BF7146FFF6C6AE0AEB04030A1B42F099
:107608000102C9F808305A603846DAF80420A8465A
:1076180002F001031C43CAF80440FAF79FFC1CE778
:10762800404629460193CDF800C0FAF757F9DDF82E
:1076380000C0019BE2461E46DCF80430FBE6294602
:10764800FAF74CF976E75B4404F11001C6188E424C
:10765800FFF679AFE046DCF80C30ABF1040258F8DD
:10766800081F242ACB60996055D8132A414621D98E
:107678002B460CF1100153F8040BCCF8080068688D
:107688001D1D1B2ACCF80C0014D958682B1D0CF1B1
:107698001801CCF8100068680835242ACCF81400C2
:1076A80008D15B680CF12001CCF818306B680835FC
:1076B800CCF81C302A460B4652F8040B43F8040B4E
:1076C8006868486052685A600CEB0403321B42F049
:1076D8000102C9F808305A603846DCF8042002F084
:1076E80001031C43CCF80440FAF738FCB5E650F81F
:1076F800046C0AF1080826F003065E449BE640463F
:107708002946CDF800C0FAF7E9F8DDF800C0E246EE
:10771800DCF804308FE640462946CDF800C0FAF779
:10772800DDF8DDF800C0CFE750EA010310B43CD023
:10773800D0F1010238BF0022B1F1004F14BF00237D
:1077480002F00103002B30D14FF6FF73A1F5801032
:10775800C7F6DF7301F1FE44984204F570048CBF4C
:10776800002001209C428CBF034640F00103002BFF
:1077780020D1B1F5801F01F100402CBF0023012367
:10778800B0F5801F38BF43F001038BB911F5801F96
:10779800C7F6F07314BF00200120994214BF0146B8
:1077A80040F0010102EA010000E0022010BC70472D
:1077B8000320FBE70420F9E702460846F0B410F876
:1077C800015B5E2D2FD0002421460023D4540133C1
:1077D800B3F5807FFAD17DB181F001045455034699
:1077E80013F8011B2D290BD05D2907D009B9F0BC6E
:1077F80070470D461846F1E70138F8E71846F6E7EE
:107808004678A6F15D0CDCF1000747EB0C07AE42A9
:10781800B8BF47F00107002FEBD102300135AE4267
:107828005455FBDCDBE701244D7800192146CCE7F1
:107838000020C7F6C070704710B40346046808E01B
:1078480014F8012F402A02DD5A2AD8BF203282427A
:1078580008D111F8010B0028F2D1012001341C6075
:1078680010BC70470020FBE72DE9F04F9BB08A461B
:1078780004460A925346524600200021CDF85CA0E7
:10788800CDE904011F4613F8010B2D2800F21481DD
:10789800DFE810F0F90012011201120112011201C1
:1078A8001201120112011001100110011001100142
:1078B8001201120112011201120112011201120128
:1078C8001201120112011201120112011201120118
:1078D800120112011001120112011201120112010A
:1078E800120112011201120112010D0112012E00E2
:1078F80001230C93013717973878002800F0C380CC
:10790800302800F0DF80002206922F28804640F3BE
:10791800DB85392800F3D88500267B1C3546B1461F
:1079280002E0B8F1390F1BDC05EB8502B9F1080F4D
:1079380008EB4202D8BFA2F1300508DD06EB86024B
:10794800B9F10F0F08EB4208D8BFA8F130069B46E3
:10795800013309F101099BF80080B8F12F0FE0DC31
:10796800CDF85CB02046FEF765FF0168204603911C
:10797800FEF760FF0068FAF7CBFE03990246584607
:10798800FAF7F6FE8346002800F05B81CC4600201B
:1079980008900990A8F16502534243EB0203B8F13D
:1079A800450F08BF43F00103002B61D0069A4CEA4B
:1079B80000031A4367D0DDF85CA00AF101021792B0
:1079C8009AF80180B8F12B0F00F08485B8F12D0FDB
:1079D80000F0AD8400210B91A8F13003092B00F2CF
:1079E8000A85B8F1300F07D1179B0133179313F8A5
:1079F800018BB8F1300FF9D0A8F13103082B00F250
:107A0800BD851799A8F1300201F1010BCDF85CB0E2
:107A18000D9191F80180B8F12F0F14DDB8F1390FED
:107A280011DC8B1C02E0B8F1390F0CDCA8F1300135
:107A380017939B4613F8018B02EB8202B8F12F0FC4
:107A480001EB4202EFDC0D9B44F61F618A42C3EB57
:107A58000B0BD4BF00230123BBF1080FC8BF43F0B1
:107A68000103002B0CBF13460B460B9901B15B4277
:107A7800BCF1000F3DD1069A024340F0DE80099B1D
:107A8800002B00F09183DDF810800025059BCDF8D0
:107A98005CA00C950A9909B1179A0A600C9A0AB168
:107AA80003F10043404619461BB0BDE8F08F0022A1
:107AB8000C921FE71A46E5E6002530280C95179228
:107AC8007FF421AF7B780137582B00F09D84782B09
:107AD80018BF3B4600F098841F4601333878302899
:107AE800FAD01797804603460028D3D00121069183
:107AF8000BE708992846BCF1100FB4BFE0464FF0D9
:107B08001008B9F1000F14BFCA46E2465B1ACDF857
:107B18000CC0099303F0F8FEB8F1090FDDF80CC0AA
:107B280002460B46CDE904231ADD42F6B043C0F6FF
:107B3800030303EBC80353E9122303F05BFFCDE90A
:107B48000401304603F0E0FE02460B46DDE904017D
:107B580003F09EFDDDF80CC002460B46CDE9042378
:107B6800BCF10F0F00F3BB80099B002B65D040F3DD
:107B7800C9850998162800F39A8542F6B041DDE9CF
:107B88000423C0F6030101EBC001D1E9000103F0B1
:107B980031FF80460B467DE70899002900F0A7854C
:107BA80005994FF6FF72C0F20F0221F07F4323F4CC
:107BB8007003934200F0C685049800F001037BB17E
:107BC8000899002900F0F683DDE90601FFF70AFAB3
:107BD800DDE9062303F05CFD02460B46CDE90423EC
:107BE800BBF1000F15D0002310931A46DDE90401FC
:107BF800C3F650121192DDE9102303F0FBFE0B4689
:107C08000246CDE90423059B1BB9049808B9222331
:107C1800236020461699FEF709FF20463946FEF7ED
:107C280005FF20462946FEF701FF20460B99FEF77F
:107C3800FDFE20464146FEF7F9FEDDF81080059B63
:107C480028E72046DDF85C80FEF7F4FD0068FAF7C7
:107C58005FFD08EB0003179318F80080B9F1000FD7
:107C680040F06382B8F1300F18BF484608D101339D
:107C780048461793013013F8018BB8F1300FF8D04C
:107C8800A8F13103082B00F2E582179F4FF0000C92
:107C98000890A8F1300B01200997BBF1000F00F004
:107CA8002884089B0128034408BF6046089300F015
:107CB80016840CEB0008634608F1FF3803E04D001A
:107CC800434500F00A84013305EB85015A1E082A52
:107CD800F5DD06EB8602102BD8BF5600F0E70998B1
:107CE800C8EB0C0B8344BBF1000F40F36B841BF013
:107CF8000F0013D042F6B041DDE90423C0F60301BA
:107D0800CDF80CC001EBC001D1E9000103F072FE0F
:107D1800DDF80CC002460B46CDE904233BF00F0BFF
:107D280040F0A08239462046524663460095FEF749
:107D3800DBFE0B90DDE90401CDE906010B990C315E
:107D48000D910B9A204619AD5168FEF73BFE0B9B2F
:107D58000D991A690232920007460C30F9F716FDA0
:107D6800DDE90623204618A900950191FFF7B4F92B
:107D7800012116902046FEF755FF099A002A05466C
:107D8800C0F26581DDF82490002219996FF47F70A4
:107D9800189B0029ACBF02EB010AC1EB090CCBEB25
:107DA8000101B8BF924601EB030EA8BFCC46864539
:107DB8000CEB0B06AEBFC3F1360301F58663033344
:107DC80003EB0A08F618B045B4BF4346334653459B
:107DD800A8BF5346002BC2BFC3EB0808C3EB060677
:107DE800C3EB0A0A8AB129462046FEF7B9FF169A5C
:107DF800054620462946FEF71FFF169903462046EA
:107E08000393FEF713FE039B1693B8F1000F05DDED
:107E1800204616994246FEF7F5FF1690B9F1000F75
:107E280005D0394620464A46FEF79AFF0746002EF7
:107E380005DD394620463246FEF7E4FF0746BAF12B
:107E4800000F05DD294620465246FEF7DBFF0546B2
:107E580016993A462046FFF749F800222946C36892
:107E68008046C2600893FFF723F80028C0F24783D2
:107E78003FF492AE40462946FFF792F900224FF0B0
:107E88008043CDE9060104F031F800287FD0089836
:107E9800002800F0E0804FF00009DDF814C0CA4661
:107EA800C3F6F07900230022C3F6F073CDE9062368
:107EB80000263346C7F6F076C7F6E0730CEA0606E6
:107EC8009E4200F08380BBF1000318BF0123B6F186
:107ED800D46F8CBF002303F0010313B35046A2A351
:107EE800D3E90023494604F001F8A8B150464946B1
:107EF80004F042F84FF00009C3F6F079824618B151
:107F080003F002FD82468946089909F1004301B150
:107F18004B465246CDE90623079800F1D6639B1BD2
:107F28000793DDE9042310461946FFF75BF802467C
:107F38000B46DDE9060103F05DFD02460B46DDE96F
:107F4800040103F0A5FB02460B46CDE90423DDF846
:107F580014C0CDE90601BBF1000F07D10023C7F615
:107F6800F0730CEA03039E4200F0AA80204616999B
:107F7800FEF75CFD20463946FEF758FD20462946A7
:107F8800FEF754FD20464146FEF750FDD9E6002392
:107F9800DDE90601C3F6E073002203F02BFD089B20
:107FA80082468946002B75D101F10043DDF814C0E3
:107FB80052460026CDE906233346C7F6F076C7F6C3
:107FC800E0730CEA06069E427FF47DAFDDE904010A
:107FD800ACF1547CCDF814C0DDE90423CDE91001DF
:107FE80010461946FEF7FEFF02460B46DDE906017C
:107FF80003F000FD02460B46DDE9040103F048FBEF
:1080080002460B46CDE904230023DDF814C0C7F669
:10801800F0734FF6FF720CEA0303C7F69F429342D0
:108028007AD94FF6FF731198C7F6EF73984200F0AC
:10803800AC824FF6FF724FF0FF3013460490C7F63C
:10804800EF730593DDE90423CDE906238EE7524259
:108058004FF0000999E6049BF3B9DDF814C0CCF39E
:108068001303FBB90023DDE906010022C3F6F07310
:10807800CDF80CC003F030FFDDF80CC0002800F08C
:108088008380002399461A46CA46CBF6E073C3F6A6
:10809800E0798EE70B4689E7012B03D10599002982
:1080A80000F0A2814FF0000900230022CBF6F07304
:1080B800CA46CDE90623DDF814C0C3F6F079F7E621
:1080C80049465046CDF80CC003F02EFF03F02CFCB7
:1080D8000B4602464946504603F0D8FA089BDDF89D
:1080E8000CC0CDE90E0113B9049A002A2DD0DDE9A0
:1080F8000E011FA3D3E9002303F0EEFE00287FF44E
:1081080088ADDDE90E011CA3D3E9002303F002FFCB
:1081180000283FF42BAF7CE50CF1547CCDF814C05B
:10812800DDE90401CDE9060115E75846CC46CDF84E
:1081380020B0A8F1300BBBF1090F03D8179A013012
:108148000992AAE50121099124E4CCF31303002B39
:10815800CDD10BA3D3E9002303F0BEFE00283FF4E2
:1081680005AF56E5AFF300800000C0FFFFFFDF4119
:108178009535A094FFFFDF3F35E5AF350000E03FC0
:108188009535A094FFFFCF3F00230022C3F6E0738C
:10819800DDE9060103F02EFCDDF80CC082468946B5
:1081A800024601F1004304E7A8F14908B8F1250F98
:1081B8003FF669AC01A555F828F000BF798300089F
:1081C8008F7A00088F7A00088F7A00088F7A000863
:1081D800478300088F7A00088F7A00088F7A000892
:1081E8008F7A00088F7A00088F7A00088F7A000843
:1081F8008F7A00088F7A00088F7A00088F7A000833
:108208008F7A00088F7A00088F7A00088F7A000822
:108218008F7A00088F7A00088F7A00088F7A000812
:108228008F7A00088F7A00088F7A00088F7A000802
:108238008F7A00088F7A00088F7A000879830008FF
:108248008F7A00088F7A00088F7A00088F7A0008E2
:10825800478300084FF0000C0123CDF820C0099394
:10826800FFF798BBBBF59A7F00F39F814FEA2B1667
:10827800012E40F3998242F6785B4FF00009C0F670
:10828800030BDDE90423D846CDF810C016F0010F22
:10829800104619464FEA660609F1010905D0D8E9E2
:1082A800002303F0A7FB02460B46012E08F108083D
:1082B800ECDCDDF810C010461946CDE9040105993B
:1082C8000BEBC909CDF80CC0A1F154710591DDE99A
:1082D8000423D9E9000103F08DFBDDF80CC00B463F
:1082E8000246CDE90423002305990022C7F6F0735E
:1082F800C7F6A04201EA0303934200F25681002226
:10830800C7F69042934283BF4FF6FF734FF0FF3199
:10831800184601F1547183BFC7F6EF704FF0000B98
:1083280005904FF0000B8CBF04910591FAE40123EE
:108338000B93531C179392F80180FFF74DBB44F23F
:10834800683117A8C0F60301FFF776FA00283FF452
:108358009AAB179B1B78282B00F02D8200200490E5
:1083680001468046CFF6F87105910B46FFF792BBA0
:1083780044F25C3117A8C0F60301FFF75DFA002844
:108388003FF481AB179B44F2603117A8C0F6030194
:10839800013B1793FFF750FA10B9179B0133179356
:1083A8000020049001468046C7F6F07105910B46FF
:1083B800FFF770BBDDE906010126FEF713FE024652
:1083C8000B46DDE9060103F061F902460B46CDE9EB
:1083D80004230022002303F075FD08B1089B1E4604
:1083E80016F0FF0F7FF4FCAB00230022CDE9042335
:1083F800222323600DE4CDF85CA00023BCF1000F1C
:108408007FF477ABFFF737BB0C9D40F27066C2F282
:10841800000615AB204617A93246019516AD009502
:1084280002F0EAFA10F00708054608BF43463FF491
:1084380031ABB8F1060F02BF17974FF0000843465B
:108448003FF428AB169A3AB1316813A8FEF7F6FE46
:1084580020461699FEF7EAFA159BB8F1060F0BD8D5
:10846800DFE808F02E221D1604222E006FF00041CE
:108478004FF0FF320591049215F0080F3FF4DDAB81
:10848800059DDDF8108045F000430593FFF702BB1A
:10849800002204921346C7F6F0730593ECE7139B8A
:1084A800149804930590E7E703F586631399149AE3
:1084B800033322F48012049142EA03520592DBE767
:1084C800002105910491D7E70026BB463546B14601
:1084D800FFF748BA00230B932BE7604401380828BC
:1084E80000F1010C00F3248105EB850500200BEB5E
:1084F800450509994B1C179391F8018019E6089BCB
:10850800002B7FF46DAB049800287FF469AB059AC3
:10851800C2F31303002B7FF463ABC7F6F07302EAD0
:108528000303B3F1D66F7FF65BABD8F8143023B9E9
:10853800D8F81030012B7FF753AB41460122204673
:10854800FEF760FC29468046FEF7B2FC00287FF75C
:1085580047ABBBF1000F40F01981059A22F00043A8
:108568001B0D1B05A3F580134FF0FF3204926FEA31
:1085780013536FEA03510591FFF732BB0023BCF197
:10858800000F7FF4B6AAFFF776BA1099B1F1FF3F52
:108598007FF44FAD0023002118460491C7F6F07010
:1085A800223305902360FFF734BB002300201D46CB
:1085B8000490C7F6F07522230595804623602B4664
:1085C800FFF768BA3FF4AEABCBF1000616F00F0226
:1085D80013D042F6B043DDE90401C0F60303CDF839
:1085E8000CC003EBC203D3E9002303F02DFBDDF835
:1085F8000CC002460B46CDE90423361108BFB3462A
:108608003FF490AB1F2E4BDC16F0100B18BF4FF049
:108618006A0B002E1ADD42F6C858DDE90423C0F6BD
:108628000308E14616F0010F1046194605D0D8E9AF
:10863800002303F0DFF902460B46761008F108081C
:10864800F0D1CC4610461946CDE90401BBF1000F24
:1086580015D00023059AC7F6F07302EA03031B0D31
:10866800C3F16B03002B0ADD1F2B40F3B7800021F9
:10867800342B049140F3BB804FF05C720592DDE926
:10868800040100220023CDF80CC003F01BFC0126D6
:10869800DDF80CC000B1002616F0FF0F7FF442ABE6
:1086A8004FF00008222243462260FFF7F3B9CCF1CD
:1086B8000F06099906F1160399423FF710AB42F6E7
:1086C800B044DDE90423C0F6030404EBC601D1E994
:1086D800000103F08FF9099A961B04EBC604D4E94C
:1086E800002303F087F980460B46FFF7D3B90598B6
:1086F800C0F31303002B7FF45FAA049900297FF4C9
:108708005BAA26E7099B13F1160FFFF6E8AA42F6C3
:10871800B043099DC0F60303DDE90401A3EBC503DB
:10872800D3E9002303F090FA80460B46FFF7B2B96D
:10873800BCF1100F04DC0A23002003FB06B6D8E6C0
:108748000020D6E60498BBF1000F1CD00023C7F622
:10875800F07301EA0303B3F1D46F14D81B0DC3F10E
:108768006B024FF0FF33934098427FF425AA002311
:108778000022C7F6F073049201EA030303F580139D
:108788000593FFF72DBA4FF0FF33EDE7059820F07A
:1087980000431B0D1B05B3F1D66F3FF6E3AEB3F1F3
:1087A8005C7F3FF620AA1FE642F6785B4FF000098F
:1087B800C0F6030B83E517A8114913AA02F0E4FBDE
:1087C80005287FF4CBAD139D149BA84643F0FE43C8
:1087D800049543F470030593FFF75CB94FF0FF323B
:1087E800049812FA03F303EA0000049047E7A3F1A0
:1087F80020014FF0FF338B40134005933FE700BF44
:108808008406002040F2A4030A46C2F2000301468F
:108818001868FFF729B800BF2DE9704340F2A40497
:10882800C2F200040A46014601262068FFF71CF838
:108838008946804603F0C0FB0021054603F050FC42
:1088480000B1002616F0FF0F0CD140464946002221
:10885800002303F037FB28B9236822221A60284630
:10886800BDE870834FF6FF712846C7F67F7103F0A5
:108878005FFC70B14FF6FF73404649464FF0FF3238
:10888800C7F6EF73012603F045FBC8B116F0FF0FDA
:10889800E2D028466FF4000103F02CFC0028DED05B
:1088A800404649464FF0FF326FF48013012603F02B
:1088B80013FB50B116F0FF0FCED02846BDE87083E9
:1088C800002616F0FF0FC7D0E3E7002616F0FF0FCB
:1088D800C2D0F2E7AFF300802DE9F04F40F2AC547C
:1088E800C2F2000487B01F468B4626680B460590E7
:1088F800049213F8014B32191D46527812F00802FF
:10890800F7D12D2C00F09D802B2C08BF15F8014BBA
:108918000392D7F1010338BF0023102F14BF1A4662
:1089280043F0010272B1302C00F09D80002B00F062
:10893800B680302C00F0AD800A2000210A27CDE94E
:10894800000103E03A46FB17CDE9002303994FF0F5
:1089580000084FF0004919B94FF0FF386FF000498F
:1089680040464946DDE9002303F0ECFB4046494612
:108978009246DDE9002303F0E5FB002200234FF0D7
:10898800000C894631198046497811F0040F30D01F
:10899800303CA74237DD904579EB03002CBF00211E
:1089A800012151EADC7C40D183EA090182EA08000E
:1089B80050EA010C14BF002101215445D4BF002105
:1089C80001F00101002930D101984FF0010C02FBA0
:1089D80000F1009800FB0311A2FB0023CB18121929
:1089E80043EBE47315F8014B3119497811F0040F82
:1089F800CED111F0030106D0012914BF5721372128
:108A0800641AA742C7DCBCF1FF3F1FD00399A1B984
:108A1800049828B1BCF1000F0CD10499C1F800B03A
:108A28001046194607B0BDE8F08F4FF0FF3C15F827
:108A3800014BD9E705F1FF3BEFE7524263EB4303F4
:108A4800E6E715F8014B0120039062E703994FF020
:108A5800FF326FF0004311B100224FF00043059838
:108A680022210160D4E72A78A2F17800414241EB43
:108A78000001582A14BF0A4641F00102002A3FF4B7
:108A880055AF6C78102200230235CDE9002310275A
:108A98005CE7082200230827CDE9002356E738467B
:108AA800F917CDE9000151E72DE9F04F40F2AC5636
:108AB800C2F2000683B09A460C46D6F800801546E6
:108AC8000B46019013F8016B08EB06021F4692F85B
:108AD80001B01BF0080BF5D12D2E74D02B2E08BF3A
:108AE80017F8016BDAF1010338BF0023BAF1100F50
:108AF80014BF1A4643F001026AB1302E68D053B150
:108B0800302E7BD049F699194FF00A0A0521C1F693
:108B18009919D4460BE051464FF0FF3002F01CFB88
:108B2800514681464FF0FF3002F044FCD44608EB32
:108B38000603002210465B7813F0040F1FD0303E66
:108B4800B24526DD484594BF0023012353EAD2727B
:108B58002BD1C9EB0002534243EB02038E42D4BF30
:108B6800002303F0010303BB0CFB006017F8016B43
:108B7800012208EB06035B7813F0040FDFD113F032
:108B8800030306D0012B14BF57233723F61AB24527
:108B9800D8DCB2F1FF3F11D0BBF1000F0CD10DB101
:108BA80042B92C6003B0BDE8F08F4FF0FF3217F8E0
:108BB800016BDEE77C1EF4E74042F0E701992223CF
:108BC80010460B60EBE717F8016B4FF0010B89E7D4
:108BD8003A78A2F17800414241EB0001582A14BFCB
:108BE8000A4641F00102002A89D04FF0100A7E7827
:108BF8000F2102376FF07049D44698E74FF0080A02
:108C080007216FF06049D44691E700BF30B440F2C5
:108C1800A404C2F200040D46134601462A46206801
:108C280030BC41E7000000002DE9F04F40F2AC54A1
:108C3800C2F2000487B01F460B46266802910590D1
:108C4800039213F8014B32191D46527812F00802AC
:108C5800F7D12D2C00F09F802B2C08BF15F8014B65
:108C68000492D7F1010338BF0023102F14BF1A460E
:108C780043F0010292B1302C00F0928073B1302C95
:108C880000F0AA800FF26819D9E900894FF0050CA5
:108C98004FF00A0A4FF0000B0A2715E04FEAE77B6E
:108CA8003A465B464FF0FF304FF0FF31BA4603F0CB
:108CB80049FA3A465B46804689464FF0FF304FF006
:108CC800FF3103F03FFA94463019CDF804C0002173
:108CD80000224078002310F0040F2ED0303CA74229
:108CE80035DD904579EB030C2CBF0020012050EABC
:108CF800D1713CD182EA080083EA090150EA010CEB
:108D0800019814BF002101218442D4BF002101F041
:108D1800010100292BD102FB0BF001210AFB030002
:108D2800A2FB0A23C318121943EBE47315F8014B8D
:108D38003019407810F0040FD0D110F0030006D09D
:108D4800012814BF57203720241AA742C9DCB1F1E3
:108D5800FF3F18D0049890B9039C1CB161B90298E0
:108D6800039908601046194607B0BDE8F08F4FF028
:108D7800FF3115F8014BDBE7013D0295EFE7524261
:108D880063EB4303E8E7059C22204FF0FF324FF0E6
:108D9800FF332060E0E715F8014B0120049060E7FD
:108DA8002A78A2F17800414241EB0001582A14BF09
:108DB8000A4641F00102002A3FF460AF6C784FF098
:108DC8000F0C02354FF0FF386FF070494FF0100A62
:108DD8004FF0000B102777E74FF0070C4FF0FF38E4
:108DE8006FF060494FF0080A4FF0000B08276BE757
:108DF80099999999999999192DE9F04F83B09146C4
:108E08000D46019090681768002877D04FF0000A47
:108E180008688B685446002C4CD09C421E469846E5
:108E28003CBF2646A04635D3AB8913F4906F31D0AA
:108E38006A6904F1010E296902EB420B461A0EEB2E
:108E480006000BEBDB7B4FEA6B0B83455A463CBFB6
:108E58008346024613F4806F31D001981146F8F723
:108E68005FF98046002834D029693246F8F78EFC2D
:108E7800AB8923F4906343F08003AB8108EB0600D1
:108E8800C6EB0B03C5F810802646A0462860C5F837
:108E980014B0AB6042465146F8F720FDD9F80820D7
:108EA800AB682868141B9B1BAB6040442860C9F85A
:108EB8000840ECB1D7F800A07C680837ABE7019808
:108EC800FEF724FA80460028D8D101982969F7F7D7
:108ED800DBFF019A0C234FF0FF3013600023AA89AF
:108EE80042F04002AA81C9F80830C9F8043002E00B
:108EF8002046C9F8044003B0BDE8F08F5060FAE797
:108F08002DE9F04FABB08946834606938B8913F061
:108F1800800F03D00B69002B00F01585174600233E
:108F28000CAE089305932696289327933B78B3F1C4
:108F3800250218BF0122002B0CBF002302F00103F9
:108F4800002B00F060837A1C144601322378191E26
:108F580018BF0121252B0CBF002301F00103002BB2
:108F6800F2D1E51B0ED0279B289A01333760072BD7
:108F780075602A442793289200F3BC830836059924
:108F8800491905912378002B00F03F830022002324
:108F98000492671C8DF8A7304FF0FF38637892462B
:108FA8004FF0200C2B240137A3F12002582A00F29D
:108FB8004E82DFE812F05A024C024C02FB014C02CE
:108FC8004C024C024C024C024C02FE0014024C02B1
:108FD8000A0118024C021002FF01FF01FF01FF0104
:108FE800FF01FF01FF01FF01FF014C024C024C028F
:108FF8004C024C024C024C024C024C024C02C70080
:109008004C024C024C024C024C024C024C024C02E8
:109018004C024C02BD004C024C024C024C024C0269
:1090280059004C024C026D014C024C024C024C029D
:109038004C024C024C024C024C024C029201C900F8
:109048004C024C024C026901C9004C024C025F01FF
:109058004C024C01BF00340130014C020E014C029D
:109068005B004C024C0235024AF0100A1AF0200F3D
:1090780000F0BF83069BDA1D012322F0070202F1EC
:1090880008050695D2E9004554EA05000CBF002200
:10909800012200218DF8A710B8F1000FA8BF2AF00F
:1090A800800AB8F1000F18BF42F00102002A70D000
:1090B800012B00F04883022B00F06F831CAAB446F2
:1090C80002F1270302920397EA08E70847EA45777F
:1090D80004F00704114604F130020D463C461E46D2
:1090E8001A70013B54EA0500EED11AF0010F0996F7
:1090F800039F664600F0AB83302A00F0658309932E
:109108000299099A01F128039B1A039330231370DB
:10911800CDF81C80039807999DF8A7308842B8BFFE
:1091280008460290002B00F0E88001300290E4E04D
:109138004AF0100A1AF0200300F06683069BDA1D35
:1091480000239AE74AF0100A1AF0200F00F0438330
:109158000698C31D23F0070303F108010691D3E91C
:109168000045002C75F10000C0F2AB8354EA0501FC
:109178004FF001030CBF00220122B8F1000FA8BF75
:109188002AF0800AB8F1000F18BF42F00102002A45
:109198008ED1002B40F0AA821AF0010F00F0F9825C
:1091A800012130230DF1970203918DF89730099230
:1091B800AEE70698069900680A1D0028049080F218
:1091C8003883049B06925B4204934AF0040A3B7876
:1091D800E9E6069B00258DF8A750181D06901B6828
:1091E8000993002B00F0CE83B8F1000FC0F27B8307
:1091F800099800214246F8F751FA002800F0D48374
:10920800099D401B0390404540F37F830025CDF81E
:109218000C8007957EE74AF0200A3B78C3E6069B58
:1092280044F2D4210025C0F603014AF0020A1A6864
:1092380004330693302314468DF8A4307823003A7B
:109248008DF8A53018BF01220891022321E71AF0F2
:10925800200F40F00C831AF0100F40F04B831AF0E7
:10926800400F00F04783069D05982B680435069546
:1092780018805BE63B786C2B0ABF4AF0200A4AF05C
:10928800100A17F8013F8EE64AF0400A3B788AE652
:109298001AF0200F44F2E822C0F60302089200F008
:1092A800C880069DEA1D22F0070202F10800069018
:1092B800D2E9004554EA05000CBF002201221AEA4F
:1092C800020F00F0B4828DF8A5304AF0020A30236C
:1092D80001228DF8A4300223DBE6069B01201CAA9C
:1092E8000025191D02901B680691039009928DF8BC
:1092F800A7508DF87030002107911AF002020A92E7
:1093080002D0029B023302931AF084050B9540F0B9
:10931800B58004980299441A002C40F3AF80102CB1
:1093280040F3218342F6F055289A279BC0F603059F
:109338004FF0100802E0103C102C1CDD01333560A2
:10934800C6F8048010320836072B279306F1080C5C
:109358002892F0DD26AA584649460CAEFFF74CFD88
:109368000CAA02F1080C002840F05681103C289AFB
:10937800102C279BE2DC01333560072B74602244F4
:1093880027932892DCBF0CF1080166467ADD58461F
:10939800494626AAFFF730FD002840F03D810CAB76
:1093A800289A03F108010CAE279B6BE04AF0010AEA
:1093B8003B78F8E539460022A3F1300511F8013B66
:1093C80002EB8202A3F130000F46092805EB4202A6
:1093D800F2D90492E8E54AF0800A3B78E3E58DF893
:1093E800A7403B78DFE517F8013B2A2B00F0E18224
:1093F800A3F13002092A88BF4FF000080DD839467A
:109408004FF0000811F8013B08EB880802EB480808
:10941800A3F13002092A0F46F4D948EAE878C3E5EF
:109428001AF0200F44F2D421C0F6030108917FF40A
:1094380038AF1AF0100F40F026821AF0400F00F0F3
:109448007882069A002514880432069232E7002BA7
:1094580000F0DB80012000211CAA02908DF87030FA
:109468008DF8A7100390099245E79DF8A730002BC7
:1094780040F01A828DF8A7C03B7894E5289A06F147
:109488000801279B9DF8A70068B101330DF1A700DB
:1094980030600120072B706002442793289200F364
:1094A80032810E4608310A9860B1013329A830602C
:1094B8000220072B706002442793289200F334811E
:1094C8000E4608310B9D802D00F0B3800798039D50
:1094D800441B002C3EDD102C40F31482914D4FF0BC
:1094E800100802E0103C102C1BDD01333560C6F873
:1094F800048010320836072B279306F1080C2892AF
:10950800F0DD4946584626AA0CAEFFF775FC0CA9B3
:1095180001F1080C00287FD1103C289A102C279BB9
:10952800E3DC01333560072B7460224427932892CB
:10953800DCBF0CF1080166460CDD5846494626AAF0
:10954800FFF75AFC002867D10CAB289A03F10801F1
:10955800279B0CAE01330398099D072B02447060CA
:1095680035602793289200F3AE801AF0040F30D0AC
:10957800049B029D5C1B002C2BDD102C40F3FC810E
:1095880042F6F055279BC0F60305102602E0103C72
:10959800102C15DD01330D604E6010320831072B99
:1095A80027932892F3DD4946584626AAFFF724FC5C
:1095B8000CA9002830D1103C289A102C279BE9DCF4
:1095C80001330D60072B4C6022442793289200F347
:1095D80034810598029B04998B42ACBFC01840188F
:1095E8000590002A79D1002527953B780CAEB3F178
:1095F800250218BF0122002B0CBF002302F0010333
:10960800002B7FF4A0AC3C46BCE4289B23B1584611
:10961800494626AAFFF7F0FBB9F80C30059813F075
:10962800400F18BF4FF0FF30059005982BB0BDE8EC
:10963800F08F0498029D441B002CD8BF06F1080146
:109648007FF744AF102C40F3AC81364D4FF0100833
:1096580002E0103C102C1BDD01333560C6F8048095
:1096680010320836072B279306F1080C2892F0DDF4
:109678004946584626AA0CAEFFF7BEFB0CA901F1D5
:10968800080C0028C8D1103C289A102C279BE3DC32
:1096980001333560072B7460224427932892DCBF7E
:1096A8000CF1080166467FF711AF5846494626AACD
:1096B800FFF7A2FB0028AFD10CAB289A03F10801F1
:1096C8000CAE279B02E75846494626AAFFF794FBAB
:1096D8000028A1D1289A0CA947E75846494626AA46
:1096E800FFF78AFB00283FF47EAF95E726AB03928D
:1096F80009930DE55846494626AAFFF77DFB002841
:109708008AD10CAE3BE45846494626AAFFF774FBBB
:10971800002881D10CAD289A05F10801279B2E4617
:10972800C1E600BF002E03085846494626AAFFF79F
:1097380063FB00287FF470AF0CAB289A03F1080193
:109748000CAE279BBEE60A2C75F10003C0F086809C
:109758001CA9039701F1270302911F46079620468B
:1097680029460A22002302F0EDFC3E4620462946FF
:109778000023013F02F130040A22347002F0E2FCB7
:1097880004460D4654EA0502E9D10996039F079E4F
:109798001AE026AD03930995BAE41CA9DDF820C0A8
:1097A80001F12700029104F00F02230943EA05732F
:1097B80029091CF802201C4603460D4601381A7078
:1097C80054EA0502EFD10993029D099805F128038F
:1097D8001B1A03939CE41AF0100F68D11AF0400F7B
:1097E80000F09680069BB3F9004004330693E51712
:1097F800B7E41AF0100F72D11AF0400F00F09F80F2
:10980800069B1A88012309E01AF0100141D11AF0C9
:10981800400300F08380069B1A880B46069D144679
:10982800043506950025003A18BF012231E40223C9
:109838002FE43B780692FFF7B6BB5846494626AA5E
:10984800FFF7DAFA00287FF4E7AE289AC1E6029912
:10985800099A01F128039B1A039359E4303401252E
:109868000DF1970003958DF89740099050E4069BF9
:10987800059D069819682A46EB1704300690C1E939
:109888000023FFF753BB069900250C6804310691A5
:1098980010E506990A68043114460025003A069135
:1098A80018BF0122FFF7F5BB3B78FFF77CBB069A90
:1098B800146804320692E517002C75F10000BFF613
:1098C80055AC644265EB45052D2354EA05028DF835
:1098D800A7300CBF002201220123FFF7DDBB069948
:1098E80001230A68D7E7099800210791F8F710FFC4
:1098F80003900FE40699059A0B68043106911A60E3
:10990800FFF714BB354D8C460BE60023079301E4A3
:10991800069D2C6804350695E51722E4069802682A
:10992800043014460025003A069018BF0122FFF7BC
:10993800B0BB069D2C68043506950025BAE4069848
:1099480001230268ECE740210192F7F7E9FB019A4D
:10995800C9F80000C9F81000002838D04023C9F819
:109968001430FFF7DBBA42F6F05506F1080C289AD6
:10997800C0F60305279BFEE442F6F055279BC0F688
:1099880003051DE6B8F1060F34BF4146062144F22F
:10999800183221EAE173C0F6030203910293099297
:1099A800A9E40E4D8C4673E6CDF80C800790FFF7BE
:1099B800B1BB069D2A1DD5F80080B8F1000FBFF68F
:1099C80038AF3B784FF0FF380692FFF7ECBA013812
:1099D8000C230590CBF8003027E600BF002E0308C3
:1099E800B1F1FF3F30B50C4683B012D09189E4B293
:1099F800536B21F02001918173B15168936B9942A7
:109A08002ADA1368591E116003F8014C53680133B0
:109A18005360204603B030BD1369DBB111688B4237
:109A280004D211F8013C481EA3420ED055681346D3
:109A380002F14400D16303F8464F03211360012368
:109A48001564506391635360E3E753681060013312
:109A58005360DEE71168E9E71146019200F0C6FDA0
:109A6800019A0028CDD04FF0FF34D2E710B50C464C
:109A7800496B69B104F14403994201D0F7F704FA3C
:109A8800236C00206063636013B1E36B236010BD37
:109A980022690021A3894FF0FF30616043F0200361
:109AA8002260A38110BD00BF2DE9F04F83B002FBF7
:109AB80003FB01929A4680460C9CBBF1000F22D012
:109AC8000F465E464FF0000965683846AE422A46A2
:109AD8001BD92168761BF7F759FE2368C4F8049050
:109AE80040465B19214623607F19FFF7BFFF002816
:109AF800EAD0C6EB0B00019901F02EFB82465046D6
:109B080003B0BDE8F08FDA46F9E732462168F7F787
:109B18003DFE62682368921B62609E192660EEE72C
:109B28002DE9F04FE1B00C46174680469B46F7F703
:109B380037F9A38948F6B12113F4005FC0F6000194
:109B480002BF43F40053A381626E0D9104BF22F457
:109B580000536366002051AA054609900C900A90AC
:109B680008923A785F923AB340F2AC560137C2F2A3
:109B780000063368991891F801A01AF0080A21D054
:109B880063680DE0236831685A1C1B78CB185B7832
:109B980013F0080FE5D0636801352260013B63606C
:109BA800002BEFDC40462146FFF760FF0028E9D094
:109BB8003A785F92002AD7D1F7F7F4F80A9861B09B
:109BC800BDE8F08F252A10D06368002B40F30A8186
:109BD800236817F8012C19789142EDD16268013396
:109BE80001352360531E6360BBE73A78D1460A21EA
:109BF8000137782A00F2228301A050F822F000BF32
:109C080067A2000845A2000845A2000845A200086E
:109C180045A2000845A2000845A2000845A2000880
:109C280045A2000845A2000845A2000845A2000870
:109C380045A2000845A2000845A2000845A2000860
:109C480045A2000845A2000845A2000845A2000850
:109C580045A2000845A2000845A2000845A2000840
:109C680045A2000845A2000845A2000845A2000830
:109C780045A2000845A2000845A2000845A2000820
:109C880045A2000845A2000845A2000845A2000810
:109C980045A20008D19B000845A2000845A200087B
:109CA80045A2000845A2000873A2000845A20008C2
:109CB80045A2000845A2000845A2000845A20008E0
:109CC8007BA200087BA200087BA200087BA20008F8
:109CD8007BA200087BA200087BA200087BA20008E8
:109CE8007BA200087BA2000845A2000845A2000844
:109CF80045A2000845A2000845A2000845A20008A0
:109D080045A2000845A2000845A2000845A200088F
:109D1800199E000845A2000845A2000845A20008AF
:109D280045A2000845A2000845A2000845A200086F
:109D380089A2000845A2000845A2000891A20008CF
:109D480045A2000845A2000845A2000845A200084F
:109D580045A2000845A2000845A2000845A200083F
:109D6800A7A2000845A2000845A20008BDA2000855
:109D780045A2000845A2000845A2000845A200081F
:109D880045A2000845A2000845A20008CFA2000885
:109D98001D9E000845A2000845A2000845A200082B
:109DA800BDA10008F3A1000845A2000845A20008CB
:109DB80005A2000845A20008C5A10008E1A1000805
:109DC80019A2000845A2000845A200082FA2000811
:109DD80045A2000833A2000845A2000845A20008D1
:109DE800A7A2000840462146FFF740FE00283FF49E
:109DF800EFAEF6F7D7FF0A99002900F06882A38929
:109E080003F04003002B18BF4FF0FF310A91D5E64D
:109E18004AF0010A42F6A5530A20C0F60003099346
:109E280003230C906268002A40F37B811AF0400FEC
:109E380019D122680B93306813780132C3185B7804
:109E480013F0080F0ED06368013B6360002BC8BF96
:109E5800226030DD013513780132C3185B7813F0C6
:109E6800080FF0D10B9B022B00F00681032B57D073
:109E7800012B2AD0B9F1000F08BF4FF001091AF0E1
:109E8800010640F0BC821AF0100F00F028836368C6
:109E9800404621464B4580F23E832268F618C3EBC4
:109EA8000909D3182360FFF7E1FD0028EFD0002E41
:109EB8009FD0AD1955E640462146FFF7D7FD00284B
:109EC80097D1306801352268C5E7B9F1000F08BF9E
:109ED8004FF0FF391AF0100F00F03B81236800267D
:109EE8001A7811A80133825CAAB16268013623602E
:109EF800013A4E456260DCD0002AF1DC404621463A
:109F0800FFF7B4FD0028D4D1236811A81A780133CB
:109F1800825C002AE9D1002E3FF44EAEAD1920E64E
:109F280009F1FF3351A9262B42F6106386BFA9F128
:109F380027024FF0270900220E91C0F603030E46B0
:109F4800DDF830C011460F972A464AF4586A1F4672
:109F58000D4600200B90D4F800E09EF80000A0F118
:109F68002B014D2947D8DFE801F081468146462775
:109F78007C7C7C7C7C7C7C747446464646464646A3
:109F88006E6E6E6E6E6E4646464646464646464679
:109F9800464646464646466246464646464646463D
:109FA8006E6E6E6E6E6E4646464646464646464659
:109FB80046464646464646621AF4006F0CD0BCF147
:109FC800000F03D14AF4007A0CF1080C1AF4806FE0
:109FD80000F07B822AF4B06A06F8010B6168013947
:109FE80061600029C4BF0EF10101216040F3A38024
:109FF800B9F10109AFD11AF4807F0E961546CDF854
:10A0080030C00F9F08D008998E4200F264810E9AE2
:10A01800089B9A423FF4D0AD1AF0100200F0D781A5
:10A02800089B0B9EED1A0E98AD19451999E50AF48F
:10A03800C061B1F5007FDED12AF4007A4FF0100C30
:10A048004AF4A06AC8E7BCF10A0FD4DD2AF4386ADA
:10A05800C2E737F91CC0BCF1080FCCDD2AF4386A16
:10A06800BAE737F91CC02AF4386AB5E71AF0800F46
:10A07800C1D02AF0800AAFE7B9F1000F08BF4FF04E
:10A08800FF391AF0010340F03B811AF0100F1EBF90
:10A098009A463168236830D1DBF800A00BF104033D
:10A0A8002268D346D144117830684118497811F0B4
:10A0B800080F40F0188161680139616012F8011BCE
:10A0C8000BF8011BCB45226000F00D816168002967
:10A0D800E9DC404621460793FFF7C8FC079B0028A8
:10A0E80040F001812268DEE740462146FFF7BEFCCA
:10A0F800002840F00381316823681A7801338A18F0
:10A10800527812F0080F40F0F98062680AF1010AEB
:10A118002360013ACA45626000F0F080002AECDC56
:10A12800E2E7404621460793FFF7A0FC079B00287B
:10A138003FF47CAE5DE6404621460792CDF818C054
:10A14800FFF794FC079ADDF818C000283FF450AFD9
:10A1580051E7DBF800602368B246B1441A7811A9C8
:10A168008A5CCAB16268013A626013F8012B0AF886
:10A17800012BCA4523600FD06268002AEEDC4046F6
:10A188002146FFF773FC002840F01982236811A9C3
:10A198001A788A5C002AE5D1BAEB06063FF40CADC2
:10A1A8000A9A00230BF1040BAD1901320A928AF8BE
:10A1B8000030D6E44AF0040A3A7819E51AF0100F8C
:10A1C8007FF4CFAC1AF0040F00F0BA81DBF800304E
:10A1D8000BF1040B1D80C4E448F6B1210822C0F637
:10A1E80000010C92099103231CE642F6A5510022B6
:10A1F800C0F600010C920991032313E63A786C2A01
:10A208000ABF4AF0020A4AF0010A17F8012FEFE4E0
:10A2180048F6B1231020C0F600034AF4087A0993DF
:10A2280003230C90FEE50223FCE548F6B1200A2141
:10A23800C0F600000C9109900323F3E59B1842F641
:10A24800A552C0F600025B78099203F00303012BC4
:10A2580008BF4AF0010A0A230C93073BE2E5F6F728
:10A26800A1FD4FF0FF310A91A8E44AF0100A3A78AC
:10A27800BEE401FB09F9A9F1300991443A78B7E441
:10A288004AF0020A3A78B3E448F6B1230820C0F647
:10A2980000034AF0010A099303230C90C2E548F62B
:10A2A800B1211022C0F600014AF4007A0991032373
:10A2B8000C92B7E5394611A8FDF77EFA4AF0400A34
:10A2C80001230746AEE54AF0400A0023AAE54FF00D
:10A2D800FF320A9272E416F8011D404622460E9695
:10A2E800FFF77EFB93E600228BF800200A9ECAEB5C
:10A2F80005055D449B4601360A9632E4554430E430
:10A30800002108225BA8F7F743FB1AF010034FF06F
:10A31800000A12BF5FA9DBF800000BF1040B0E93D3
:10A328000F9703960CBF0B900B91B9F1000F0AD150
:10A338000F9F0E9800287FF414AC0B9908600A9AB6
:10A3480001320A920DE42368039E1B783268D31801
:10A358005B7813F0080FEBD1FCF760FA50453FF437
:10A3680048AD276860AA636802EB0A0C0AF1010A83
:10A37800404617F801EB013B0B9951AA63605BAEAD
:10A388005346009627600CF83CECFCF779FAB0F1DC
:10A39800FF3F3FF42EAD002840F0FC800B99086089
:10A3A8000B9A1068FCF7F8F9002800F00C810F9F51
:10A3B800BAF1000FBDD051AB9A441AF8011D4046BE
:10A3C8002246FFF70DFB089EB245F6D1B1E70E9E77
:10A3D800404651A932700C9B099EB0471AF0200FD5
:10A3E80040F093801AF0040F00F08C80DBF8003006
:10A3F8000BF1040B18800A9A01320A9210E6002128
:10A4080008225DA8F7F7C4FA1AF0100243460B9227
:10A418000ABFDBF800A04FF0000A0BF1040BCDF8DF
:10A428000C90CDF83CB000260E97A846DDF82CB06D
:10A43800994614E0BBF1000F01D1CAF800B0B0444E
:10A44800039E013E0396BBF1000F3CD10AF1040ABA
:10A458005E466368002B28DD0398002866D0FCF769
:10A46800DDF9B0423FF4C5AC276860AB03EB060CDE
:10A4780063680136484617F801EB013B51466360B3
:10A4880051AA33465DAD009527600CF83CECFCF70B
:10A49800F7F9B0F1FF3F3FF4ACAC0028CAD010F197
:10A4A800020FCCD16368002BD6DC48462146FFF763
:10A4B800DDFA0028D0D045460E9FDDF83CB0C846EE
:10A4C800002E38D095E40026C3E72AF4607A15B147
:10A4D800013D09F101090B9801300B907EE50094CC
:10A4E8004046DBF8001001224B46FFF7DDFA002852
:10A4F8003FF47FAC0A9B0BF1040B451901330A9317
:10A50800FFF72FBB1AF0010231D0DBF800300BF156
:10A51800040B18606FE722684E44C9EB0303AD19BA
:10A52800636002EB09032360FFF71BBB0E9F4546E0
:10A53800DDF83CB0C8460B9900297FF412ABFEE663
:10A548001AF0010F0CD11AF0020F09D0DBF8001035
:10A558002A46EB170BF1040BC1E90023FFF701BBF7
:10A56800DBF800300BF1040B1D60FFF7FABA1AF0A4
:10A57800020FCAD009980D99884230D0404651A997
:10A588000C9BFEF7A9F9DBF800300BF1040B1860FF
:10A59800596030E710F1020F7FF402AF6368002BB7
:10A5A8003FF7C3AE40462146FFF760FA00283FF464
:10A5B800BCAE0F9FBAF1000F7FF41BACB9E656454D
:10A5C8007FF4EAAD15E40E99554409F1FF3921B934
:10A5D8000B9A8A4604320B92E0E78246DEE7404651
:10A5E80051A90C9BFEF720FBCDE700BF01F1440306
:10A5F8002DE9F0410C46496B994218D0A66B7700BB
:10A608003A46FCF783FE054668B100EB06080146AA
:10A6180032464046F7F7BAF8C4F800806563002070
:10A62800A763BDE8F0814FF0FF30BDE8F0814FF43B
:10A638008061F6F775FD0246B0B194F8461000F552
:10A648007E7360634FF48060A063053382F8FF1364
:10A65800002094F8451082F8FE1394F8441082F80C
:10A66800FD132360BDE8F0814FF0FF30BDE8F081B5
:10A67800B1F1FF3F70B50C46054616463CD010B107
:10A688008369002B3AD042F68C23C0F603039E421E
:10A6980008BF6E680ED042F6AC23C0F603039E4294
:10A6A80008BFAE6806D042F6CC23C0F603039E422C
:10A6B80008BFEE68B28912F4005F01BF42F400528D
:10A6C800736E23F4005373664FF6DF7302EA0303D5
:10A6D800B3819AB212F0040F33D0736BE4B283B132
:10A6E8007268B36B9A4236DA33685A1E326003F8DE
:10A6F800014C736801337360204670BDF6F788FA21
:10A70800C1E73369002B2FD03268934204D212F884
:10A71800013C511EA3420FD07068334606F1440134
:10A72800F26303F8464F0322306420463360012366
:10A738007163B263736070BD7368316001337360B5
:10A74800DAE712F0100F0CD012F0080F0ED143F018
:10A758000403B381C1E728463146FFF747FF0028C5
:10A76800C2D04FF0FF34C7E73268D5E728463146F4
:10A77800F6F730F90028F4D1B389B06023F0080364
:10A78800B0611B041B0CE2E740F2A4030A46C2F2C4
:10A798000003014618686BE72DE9F04F8FB0099167
:10A7A800079008920693199E002956D018991368A5
:10A7B800002964D0069A002A5ED00027099D984691
:10A7C800B9460BAC40F2A851C2F200010591059AB6
:10A7D8003368716858F804ABD2F800B00493039159
:10A7E800FCF716F800962146524603460798D847C4
:10A7F800B0F1FF3F28D0189900EB090399421BD309
:10A80800099A62B1002806DD0022A15CA954013230
:10A818008242FAD1AD1808990A6804320A6058F8D9
:10A82800042C002A1FD01899994214D9069A013786
:10A83800974210D09946CAE7049A039B3260736026
:10A8480048460FB0BDE8F08F079A8A238146136007
:10A8580000233360F4E79946F2E708994FF0FF3296
:10A868000B681892A6E7099909B108990A6003F1DB
:10A87800FF3900233360E3E7DDF81890E0E7DDF8FF
:10A888006090DDE7F0B540F2A40483B0C2F20004A2
:10A8980007460E4620681546089C394600933246FE
:10A8A8002B460194FFF778FF03B0F0BD38B501FBE4
:10A8B80002F1F6F735FC0446F8B150F8042C22F002
:10A8C8000302043A242A1AD8132A03460FD900216E
:10A8D80040F8041B031D1B2A616008D91D1D416037
:10A8E80059600833242A02BF6960596008331A4640
:10A8F800002142F8041B59605160204638BD0021F0
:10A90800F7F746F8204638BD2DE9F0014A110469E9
:10A9180000F114073B46A24226DA043200EB840415
:10A92800143411F01F0100EB820202F1040C23D051
:10A9380055680CF10402C1F12008CD40944211D9A8
:10A94800166806FA08F6354343F8045B52F8045BC8
:10A95800CD409442F4D8CCEB0403053B23F0030329
:10A96800C31818331D60CDB9DB1B9B10036103B9F5
:10A978004361BDE8F0017047644588BF6246F3D97A
:10A9880052F8041B944243F8041BF9D86FEA0C03ED
:10A998001B1923F00303C3181833E5E70433E3E76F
:10A9A80044F27C3045F69021C0F603001022302393
:10A9B800C2F20001CA54013210F8013FD2B2002B92
:10A9C800F8D144F274301A22C0F603006123CA5445
:10A9D800013210F8013FD2B2002BF8D144F26C30AA
:10A9E8001A22C0F603004123CA54013210F8013F6D
:10A9F800D2B2002BF8D170472DE9F04F8BB045F655
:10AA080090270391C2F20007069209930890FBF77A
:10AA180011FF00680490F7F77BFE049997F830302F
:10AA28000A18834612F801AC002B00F02E81039A15
:10AA380013689E1C9A78302A40F02B820333002535
:10AA48001E4613F8012B0135302AF9D017F8029069
:10AA580045F69028C2F20008B9F1000F00F01881FD
:10AA680033784FF0000918F80330344633B1721CBC
:10AA7800144601322378FB5C002BF9D1079320465A
:10AA880004995A46F7F774FED0B1B9F1000F2DD0EA
:10AA9800C4EB090923784FEA89020592502B2AD082
:10AAA800702B28D003992046079A0860002A5ED0A8
:10AAB800002D0CBF0625002528460BB0BDE8F08FF9
:10AAC800B9F1000FE4D114F80B3004EB0B094C4634
:10AAD800FB5C002BD9D009F101031C460133227815
:10AAE800BA5C002AF9D1B9F1000FD1D12378CDF899
:10AAF8001490502BD4D16378611C2B2B00F0C080AC
:10AB08002D2B08BF4FF0010900F0BC804FF0000961
:10AB1800FA5C45F69023C2F20003002AC2D0192A33
:10AB2800C0DC91F801C0103A481C13F80C3093B1FE
:10AB3800192B10DC023101E0192B0CDC084611F846
:10AB4800018BA3F1100C02EB820217F808300CEB12
:10AB58004202002BF0D1B9F1000F00D05242059B00
:10AB680003999B18079A05930860002AA0D1631ED1
:10AB78009B1B072BD8BF079904DD07995B10013190
:10AB8800072BFBDC0898FBF71DFFA64200F1140316
:10AB98008446039380F09D814FF000081A46B94619
:10ABA8005B464546474693460FE0202D2A4605F169
:10ABB80004055FD0217819F8011001F00F0111FA8E
:10ABC80002F2A64247EA020718D214F8012D5245AC
:10ABD800EBD1C3F10108A0444645E6D81A464046E1
:10ABE80004990293CDF804C0F7F7C2FD029BDDF883
:10ABF80004C00028D9D14446A642E6D3B8465B46ED
:10AC08000399404643F8048B5B1A9D10CCF810500A
:10AC1800CDF804C0FBF7B4FF069A6D01DDF804C057
:10AC280014682D1AA54200F3F880C0F2238100268B
:10AC38000699059A8B689A4200F3D180069A05997D
:10AC48005368994280F2DB805D1AAC4243DCD268DB
:10AC5800022A00F02C81032A00F05B81012A00F00F
:10AC6800458161460898FBF7E1FE149900235025B9
:10AC78000B6021E74BF8047B00273A46042599E747
:10AC88004FF0000911F8013F42E7FFF789FECEE6D1
:10AC9800304604995A46F7F76BFD002840F0A88023
:10ACA80016F80B3006EB0B0418F80320002A00F006
:10ACB800F280302B40F0F580631C1E4613F8012B00
:10ACC800302AFAD0BB5C002B40F0EC80A14601256D
:10ACD80034460795D3E66F1E002E40F0E080002F23
:10ACE80008DD60463946CDF804C0FCF7CBFADDF83C
:10ACF80004C00646039A7B1107F01F0760462946E1
:10AD0800641B52F823300122CDF804C0BA401A421D
:10AD180018BF46F00206FFF7F7FD069B0225DDF88F
:10AD280004C05B680593002E70D00699CB68022B8F
:10AD380000F0D380032B64D0012B65D116F0020FED
:10AD480062D0039A13681E4316F0010F5CD0DCF83A
:10AD580010700020039B0CEB870114311E4653F83A
:10AD6800042BB2F1FF3F40F0E080994243F8040C15
:10AD7800F4D8DCF808309F42B8BF3B4680F2D88050
:10AD88000CEB83020133CCF8103001235361022D00
:10AD980000F0C480DCF810309F4211DB14F01F046F
:10ADA80000F095800CEB8707C4F120043869CDF8D2
:10ADB80004C0FBF7E5FEDDF804C0A04280F28780FE
:10ADC80001216046CDF804C0FFF79EFD0699059A5B
:10ADD800DDF804C08B68013205929A4277DD61463E
:10ADE8000898FBF723FE14990023A3250B6063E65C
:10ADF800337801213446CDF8149007914EE60125A9
:10AE080091E7159B002BA2D145F01005149B0599DD
:10AE1800099AC3F800C011604EE62D1B604629460A
:10AE2800FCF730FADDF804C00646B8B1691E012601
:10AE380001F01F024B1116FA02F20CEB83035B6957
:10AE48001A420BD0B1424FDD6046A91EFCF71AFA30
:10AE5800DDF804C0002814BF0326022660462946F0
:10AE6800CDF804C0FFF750FD059BDDF804C05B1961
:10AE78000593DDE6651B61462A460898FBF7C2FF85
:10AE880005990026491B059100F114028446039296
:10AE9800CEE60025DAE5012105920791FEE50126B7
:10AEA80028E726463378A1460125FB5CDDE51599A0
:10AEB80000297FF4D6AE09996225039A0B60012315
:10AEC800CCF810301360149BC3F800C0F4E52125BA
:10AED8009CE7039B4FF0000892E61599C1F1010326
:10AEE800002B7FF434AF8FE70226B7E7A5427FF443
:10AEF800B8AE012CDFDD6046611ECDF804C0FCF75A
:10AF0800C1F9DDF804C000283FF4ABAE069A5368D7
:10AF1800D1E7159A002A3FF4A4AECCE7069A136845
:10AF2800013BA34223D0222570E7013232602EE78D
:10AF3800DCF8041008980131CDF804C0FBF742FD95
:10AF4800DDF804C00CF10C01DCF81020023292008C
:10AF580006460C30F6F71AFCDDF804C0089861467E
:10AF68000196FBF763FD3369DDF804C008E7631158
:10AF7800012204F01F040CEB8303A2405B691A4210
:10AF880014BF2125222541E72DE9F04F45F69024ED
:10AF9800C2F2000485B00D46924694F83030029013
:10AFA800002B00F0B6802A680298531112F01F0295
:10AFB80001680AEB8303039218BF04330022181FA9
:10AFC800914601318046064693461746019043F85C
:10AFD800042C084611F8013B002B38D0E25C002A0B
:10AFE8007AD1202B00F28F805F45F2DD46452CBFD9
:10AFF80000230123B9F1070FCCBF002303F001039D
:10B00800ABB1C9F1080C3068324633464FEA8C0CB4
:10B01800CCF12009556805FA09F5284342F8040BD4
:10B02800586820FA0CF043F8040F9845F2D85645B2
:10B0380098BF4FF00809CCD90022084646F8042DDD
:10B04800BB4611F8013BB0469146002BC6D1002FF4
:10B058005BD0B04594BF00230123B9F1070FCCBFE3
:10B06800002303F00103A3B1C9F10809316832468E
:10B0780033464FEA8909C9F12000546884402143C6
:10B0880042F8041B596821FA09F143F8041F98454E
:10B09800F3D8B24540D20198524656F8041B1346DD
:10B0A800B04243F8041B1A46F7D20199002243F82C
:10B0B800042B9942FBD2019803685BB9019A924527
:10B0C80018BF134602D136E09A4535D053F8042DFF
:10B0D800002AF9D0052019E009F101090137B9F171
:10B0E800080F07DC33681B0102F00F0243EA020273
:10B0F80032606EE756457FF66CAF00234FF00109CA
:10B1080046F8043DF0E7292B1DD0042005B0BDE822
:10B11800F08FFFF745FC46E7039989B10399019839
:10B12800C1F120024FF0FF31036831FA02F202EA5E
:10B1380003030360C1E75346012205201A60E5E7CF
:10B14800019A1368B9E7029B01301860002F80D17B
:10B15800DBE700BF000000004A1E08BF7047C0F0D0
:10B168002481884240F21681114200F01781B0FA1A
:10B1780080F3B1FA81F2A2EB0303C3F11F0304A227
:10B1880002EB03134FF000029F4600BFAFF30080AD
:10B19800B0EBC17F00BF42EB020228BFA0EBC17039
:10B1A800B0EB817F00BF42EB020228BFA0EB8170A9
:10B1B800B0EB417F00BF42EB020228BFA0EB417019
:10B1C800B0EB017F00BF42EB020228BFA0EB017089
:10B1D800B0EBC16F00BF42EB020228BFA0EBC16019
:10B1E800B0EB816F00BF42EB020228BFA0EB816089
:10B1F800B0EB416F00BF42EB020228BFA0EB4160F9
:10B20800B0EB016F00BF42EB020228BFA0EB016068
:10B21800B0EBC15F00BF42EB020228BFA0EBC150F8
:10B22800B0EB815F00BF42EB020228BFA0EB815068
:10B23800B0EB415F00BF42EB020228BFA0EB4150D8
:10B24800B0EB015F00BF42EB020228BFA0EB015048
:10B25800B0EBC14F00BF42EB020228BFA0EBC140D8
:10B26800B0EB814F00BF42EB020228BFA0EB814048
:10B27800B0EB414F00BF42EB020228BFA0EB4140B8
:10B28800B0EB014F00BF42EB020228BFA0EB014028
:10B29800B0EBC13F00BF42EB020228BFA0EBC130B8
:10B2A800B0EB813F00BF42EB020228BFA0EB813028
:10B2B800B0EB413F00BF42EB020228BFA0EB413098
:10B2C800B0EB013F00BF42EB020228BFA0EB013008
:10B2D800B0EBC12F00BF42EB020228BFA0EBC12098
:10B2E800B0EB812F00BF42EB020228BFA0EB812008
:10B2F800B0EB412F00BF42EB020228BFA0EB412078
:10B30800B0EB012F00BF42EB020228BFA0EB0120E7
:10B31800B0EBC11F00BF42EB020228BFA0EBC11077
:10B32800B0EB811F00BF42EB020228BFA0EB8110E7
:10B33800B0EB411F00BF42EB020228BFA0EB411057
:10B34800B0EB011F00BF42EB020228BFA0EB0110C7
:10B35800B0EBC10F00BF42EB020228BFA0EBC10057
:10B36800B0EB810F00BF42EB020228BFA0EB8100C7
:10B37800B0EB410F00BF42EB020228BFA0EB410037
:10B38800B0EB010F00BF42EB020228BFA0EB0100A7
:10B39800104670470CBF012000207047B1FA81F2B7
:10B3A800C2F11F0220FA02F0704708B14FF0FF30D7
:10B3B80000F066B90029F8D02DE90340FFF7CCFE6C
:10B3C800BDE8064002FB00F3A1EB0301704700BF94
:10B3D800002900F03E8180EA010C48BF49424A1E1C
:10B3E80000F01F81030048BF43428B4240F21E8198
:10B3F800114200F02381B3FA83F2B1FA81F0A0EB95
:10B408000202C2F11F0204A000EB02124FF000007A
:10B41800974600BFAFF30080B3EBC17F00BF40EB9E
:10B42800000028BFA3EBC173B3EB817F00BF40EBE3
:10B43800000028BFA3EB8173B3EB417F00BF40EB53
:10B44800000028BFA3EB4173B3EB017F00BF40EBC3
:10B45800000028BFA3EB0173B3EBC16F00BF40EB43
:10B46800000028BFA3EBC163B3EB816F00BF40EBC3
:10B47800000028BFA3EB8163B3EB416F00BF40EB33
:10B48800000028BFA3EB4163B3EB016F00BF40EBA3
:10B49800000028BFA3EB0163B3EBC15F00BF40EB23
:10B4A800000028BFA3EBC153B3EB815F00BF40EBA3
:10B4B800000028BFA3EB8153B3EB415F00BF40EB13
:10B4C800000028BFA3EB4153B3EB015F00BF40EB83
:10B4D800000028BFA3EB0153B3EBC14F00BF40EB03
:10B4E800000028BFA3EBC143B3EB814F00BF40EB83
:10B4F800000028BFA3EB8143B3EB414F00BF40EBF3
:10B50800000028BFA3EB4143B3EB014F00BF40EB62
:10B51800000028BFA3EB0143B3EBC13F00BF40EBE2
:10B52800000028BFA3EBC133B3EB813F00BF40EB62
:10B53800000028BFA3EB8133B3EB413F00BF40EBD2
:10B54800000028BFA3EB4133B3EB013F00BF40EB42
:10B55800000028BFA3EB0133B3EBC12F00BF40EBC2
:10B56800000028BFA3EBC123B3EB812F00BF40EB42
:10B57800000028BFA3EB8123B3EB412F00BF40EBB2
:10B58800000028BFA3EB4123B3EB012F00BF40EB22
:10B59800000028BFA3EB0123B3EBC11F00BF40EBA2
:10B5A800000028BFA3EBC113B3EB811F00BF40EB22
:10B5B800000028BFA3EB8113B3EB411F00BF40EB92
:10B5C800000028BFA3EB4113B3EB011F00BF40EB02
:10B5D800000028BFA3EB0113B3EBC10F00BF40EB82
:10B5E800000028BFA3EBC103B3EB810F00BF40EB02
:10B5F800000028BFA3EB8103B3EB410F00BF40EB72
:10B60800000028BFA3EB4103B3EB010F00BF40EBE1
:10B61800000028BFA3EB0103BCF1000F48BF404264
:10B6280070479CEA000F48BF4042704738BF00206F
:10B6380004BF4FEAEC7040F001007047B1FA81F2A4
:10B64800C2F11F02BCF1000F23FA02F048BF4042CA
:10B6580070470028C8BF6FF00040B8BF4FF00040E7
:10B6680000F00EB80029F4D02DE90340FFF7B3FE2F
:10B67800BDE8064002FB00F3A1EB0301704700BFE1
:10B68800704700BF81F0004102E000BF83F0004333
:10B6980030B54FEA41044FEA430594EA050F08BF65
:10B6A80090EA020F1FBF54EA000C55EA020C7FEA29
:10B6B800645C7FEA655C00F0E2804FEA5454D4EBA6
:10B6C8005555B8BF6D420CDD2C4480EA020281EA70
:10B6D800030382EA000083EA010180EA020281EAA8
:10B6E8000303362D88BF30BD11F0004F4FEA0131FA
:10B6F8004FF4801C4CEA113102D0404261EB410109
:10B7080013F0004F4FEA03334CEA133302D052428E
:10B7180063EB430394EA050F00F0A780A4F101044A
:10B72800D5F1200E0DDB02FA0EFC22FA05F2801884
:10B7380041F1000103FA0EF2801843FA05F359416A
:10B748000EE0A5F120050EF1200E012A03FA0EFCE9
:10B7580028BF4CF0020C43FA05F3C01851EBE37113
:10B7680001F0004507D54FF0000EDCF1000C7EEB30
:10B7780000006EEB0101B1F5801F1BD3B1F5001F6E
:10B788000CD349085FEA30004FEA3C0C04F101048D
:10B798004FEA445212F5800F80F09A80BCF1004FB6
:10B7A80008BF5FEA500C50F1000041EB045141EA38
:10B7B800050130BD5FEA4C0C404141EB010111F439
:10B7C800801FA4F10104E9D191F0000F04BF0146E4
:10B7D8000020B1FA81F308BF2033A3F10B03B3F1C2
:10B7E80020020CDA0C3208DD02F1140CC2F10C0252
:10B7F80001FA0CF021FA02F10CE002F11402D8BFB0
:10B80800C2F1200C01FA02F120FA0CFCDCBF41EA7B
:10B818000C019040E41AA2BF01EB0451294330BD4A
:10B828006FEA04041F3C1CDA0C340EDC04F1140427
:10B83800C4F1200220FA04F001FA02F340EA0300FE
:10B8480021FA04F345EA030130BDC4F10C04C4F144
:10B85800200220FA02F001FA04F340EA0300294624
:10B8680030BD21FA04F0294630BD94F0000F83F46E
:10B87800801306BF81F480110134013D4EE77FEA51
:10B88800645C18BF7FEA655C29D094EA050F08BF9D
:10B8980090EA020F05D054EA000C04BF194610467E
:10B8A80030BD91EA030F1EBF0021002030BD5FEAC2
:10B8B800545C05D14000494128BF41F0004130BDEA
:10B8C80014F580043CBF01F5801130BD01F000453E
:10B8D80045F0FE4141F470014FF0000030BD7FEAB1
:10B8E800645C1ABF194610467FEA655C1CBF0B46AC
:10B8F800024650EA013406BF52EA033591EA030FC3
:10B9080041F4002130BD00BF90F0000F04BF0021BA
:10B91800704730B54FF4806404F132044FF00005ED
:10B928004FF0000150E700BF90F0000F04BF002166
:10B93800704730B54FF4806404F1320410F00045CC
:10B9480048BF40424FF000013EE700BF42004FEAC7
:10B95800E2014FEA31014FEA02701FBF12F07F4344
:10B9680093F07F4F81F06051704792F0000F14BF41
:10B9780093F07F4F704730B54FF4607401F0004585
:10B9880021F0004120E700BF50EA010208BF7047DC
:10B9980030B54FF000050AE050EA010208BF7047D1
:10B9A80030B511F0004502D5404261EB41014FF43A
:10B9B800806404F132045FEA915C3FF4DCAE4FF03E
:10B9C80003025FEADC0C18BF03325FEADC0C18BF25
:10B9D800033202EBDC02C2F1200300FA03FC20FA76
:10B9E80002F001FA03FE40EA0E0021FA02F11444C3
:10B9F800C1E600BF70B54FF0FF0C4CF4E06C1CEAD8
:10BA080011541DBF1CEA135594EA0C0F95EA0C0F4C
:10BA180000F0DEF82C4481EA030621EA4C5123EABF
:10BA28004C5350EA013518BF52EA033541F48011EE
:10BA380043F4801338D0A0FB02CE4FF00005E1FBA1
:10BA480002E506F00042E0FB03E54FF00006E1FBEB
:10BA580003569CF0000F18BF4EF0010EA4F1FF042E
:10BA6800B6F5007F64F5407404D25FEA4E0E6D416E
:10BA780046EB060642EAC62141EA55514FEAC5207F
:10BA880040EA5E504FEACE2EB4F1FD0C88BFBCF5FB
:10BA9800E06F1ED8BEF1004F08BF5FEA500E50F1AC
:10BAA800000041EB045170BD06F0004646EA010172
:10BAB80040EA020081EA0301B4EB5C04C2BFD4EBA4
:10BAC8000C0541EA045170BD41F480114FF0000E9D
:10BAD800013C00F3AB8014F1360FDEBF002001F00B
:10BAE800004170BDC4F10004203C35DA0C341BDC85
:10BAF80004F11404C4F1200500FA05F320FA04F057
:10BB080001FA05F240EA020001F0004221F000418A
:10BB180010EBD37021FA04F642EB06015EEA430EFD
:10BB280008BF20EAD37070BDC4F10C04C4F120052D
:10BB380000FA04F320FA05F001FA04F240EA0200E0
:10BB480001F0004110EBD37041F100015EEA430EB1
:10BB580008BF20EAD37070BDC4F1200500FA05F2D1
:10BB68004EEA020E20FA04F301FA05F243EA020350
:10BB780021FA04F001F0004121FA04F220EA02005F
:10BB880000EBD3705EEA430E08BF20EAD37070BDA5
:10BB980094F0000F0FD101F00046400041EB010185
:10BBA80011F4801F08BF013CF7D041EA060195F067
:10BBB800000F18BF704703F00046520043EB030321
:10BBC80013F4801F08BF013DF7D043EA060370470E
:10BBD80094EA0C0F0CEA135518BF95EA0C0F0CD019
:10BBE80050EA410618BF52EA4306D1D181EA03015F
:10BBF80001F000414FF0000070BD50EA410606BF59
:10BC08001046194652EA430619D094EA0C0F02D19D
:10BC180050EA013613D195EA0C0F05D152EA0336E2
:10BC28001CBF104619460AD181EA030101F0004100
:10BC380041F0FE4141F470014FF0000070BD41F049
:10BC4800FE4141F4780170BD70B54FF0FF0C4CF423
:10BC5800E06C1CEA11541DBF1CEA135594EA0C0F42
:10BC680095EA0C0F00F0A7F8A4EB050481EA030E8F
:10BC780052EA03354FEA013100F088804FEA033376
:10BC88004FF0805545EA131343EA12634FEA022244
:10BC980045EA111545EA10654FEA00260EF0004105
:10BCA8009D4208BF964244F1FD0404F5407402D257
:10BCB8005B084FEA3202B61A65EB03055B084FEAE8
:10BCC80032024FF480104FF4002CB6EB020E75EBE5
:10BCD800030E22BFB61A754640EA0C005B084FEA0D
:10BCE8003202B6EB020E75EB030E22BFB61A75468A
:10BCF80040EA5C005B084FEA3202B6EB020E75EBD5
:10BD0800030E22BFB61A754640EA9C005B084FEA4C
:10BD18003202B6EB020E75EB030E22BFB61A754659
:10BD280040EADC0055EA060E18D04FEA051545EA48
:10BD380016754FEA06164FEAC30343EA52734FEAF1
:10BD4800C2025FEA1C1CC0D111F4801F0BD141EA6A
:10BD580000014FF000004FF0004CB6E711F4801FCF
:10BD680004BF01430020B4F1FD0C88BFBCF5E06FAF
:10BD78003FF6AFAEB5EB030C04BFB6EB020C5FEABF
:10BD8800500C50F1000041EB045170BD0EF0004E14
:10BD98004EEA113114EB5C04C2BFD4EB0C0541EA46
:10BDA800045170BD41F480114FF0000E013C90E643
:10BDB80045EA060E8DE60CEA135594EA0C0F08BF07
:10BDC80095EA0C0F3FF43BAF94EA0C0F0AD150EA06
:10BDD80001347FF434AF95EA0C0F7FF425AF104699
:10BDE80019462CE795EA0C0F06D152EA03353FF4C1
:10BDF800FDAE1046194622E750EA410618BF52EA3E
:10BE080043067FF4C5AE50EA41047FF40DAF52EA11
:10BE180043057FF4EBAE12E74FF0FF3C06E000BFAE
:10BE28004FF0010C02E000BF4FF0010C4DF804CDBB
:10BE38004FEA410C7FEA6C5C4FEA430C18BF7FEA7B
:10BE48006C5C1BD001B050EA410C0CBF52EA430CA9
:10BE580091EA030F02BF90EA020F0020704710F129
:10BE6800000F91EA030F58BF994208BF90422CBFB8
:10BE7800D8176FEAE37040F0010070474FEA410CB1
:10BE88007FEA6C5C02D150EA013C07D14FEA430CCF
:10BE98007FEA6C5CD6D152EA033CD3D05DF8040B40
:10BEA800704700BF8446104662468C461946634672
:10BEB80000E000BF01B5FFF7B7FF002848BF10F149
:10BEC800000F01BD4DF808EDFFF7F4FF0CBF01208E
:10BED80000205DF808FB00BF4DF808EDFFF7EAFF0A
:10BEE80034BF012000205DF808FB00BF4DF808EDC5
:10BEF800FFF7E0FF94BF012000205DF808FB00BFBA
:10BF08004DF808EDFFF7CEFF94BF012000205DF843
:10BF180008FB00BF4DF808EDFFF7C4FF34BF012050
:10BF280000205DF808FB00BF4FEA410212F500123D
:10BF380015D211D56FF47873B3EB625212D94FEA68
:10BF4800C12343F0004343EA505311F0004F23FA52
:10BF580002F018BF404270474FF00000704750EAA7
:10BF6800013005D111F0004008BF6FF00040704764
:10BF78004FF00000704700BF4A0011D212F50012BE
:10BF880011D20DD56FF47873B3EB62520ED44FEA29
:10BF9800C12343F0004343EA505323FA02F07047A9
:10BFA8004FF00000704750EA013002D14FF0FF30E7
:10BFB80070474FF0000070474FEA4102B2F1E0438A
:10BFC80024BFB3F5001CDCF1FE5C0DD901F0004C78
:10BFD8004FEAC0024CEA5070B2F1004F40EB8300C8
:10BFE80008BF20F00100704711F0804F21D113F1F4
:10BFF8003872BCBF01F00040704741F480114FEA2D
:10C008005252C2F11802C2F1200C10FA0CF320FAB5
:10C0180002F018BF40F001004FEAC1234FEAD323D2
:10C0280003FA0CFC40EA0C0023FA02F34FEA43033C
:10C03800CCE77FEA625307D150EA01331EBF4FF0C5
:10C04800FE4040F44000704701F0004040F0FE40E0
:10C0580040F40000704700BF4FF0FF3C06E000BF0F
:10C068004FF0010C02E000BF4FF0010C4DF804CD79
:10C078004FEA40024FEA41037FEA226C18BF7FEA89
:10C08800236C11D001B052EA530C18BF90EA010F8B
:10C0980058BFB2EB030088BFC81738BF6FEAE1701A
:10C0A80018BF40F0010070477FEA226C02D15FEAB6
:10C0B800402C05D17FEA236CE4D15FEA412CE1D022
:10C0C8005DF8040B704700BF844608466146FFE7E9
:10C0D8000FB5FFF7C9FF002848BF10F1000F0FBDCB
:10C0E8004DF808EDFFF7F4FF0CBF012000205DF8C4
:10C0F80008FB00BF4DF808EDFFF7EAFF34BF012049
:10C1080000205DF808FB00BF4DF808EDFFF7E0FFE1
:10C1180094BF012000205DF808FB00BF4DF808ED32
:10C12800FFF7D2FF94BF012000205DF808FB00BF95
:10C138004DF808EDFFF7C8FF34BF012000205DF877
:10C1480008FB00BF4BB942B9002908BF002802D03C
:10C158004FF0FF310846FFF793BA82B0EC462DE95D
:10C16800005000F01DF8DDF804E002B00CBC704788
:10C178002DE970431646804689461D4600F028F88A
:10C1880000FB05F3A0FB064506FB0136069B751967
:10C19800B8EB040469EB0505C3E90045BDE8708305
:10C1A8002DE970431646804689461D4600F0C0F9C1
:10C1B80000FB05F3A0FB064506FB0136069B751937
:10C1C800B8EB040469EB0505C3E90045BDE87083D5
:10C1D80000292DE9F04F1C4685B0C0F2CB8000261F
:10C1E800002CC0F2C2808C46174614460546884685
:10C1F8009A46002B4AD18A426ED9B2FA82F35BB1D1
:10C20800C3F1200401FA03F830FA04F210FA03F536
:10C2180017FA03F442EA08084FEA144A404651461E
:10C228001FFA84FBFEF798FF514681464046FFF708
:10C23800C1F8280C0BFB09F340EA0148434509D92A
:10C2480018EB040809F1FF3904D2434584BF09F10A
:10C25800FF39A044C3EB080851464046ADB2FEF78B
:10C268007BFF514607464046FFF7A4F80BFB07FB48
:10C2780045EA0145AB4505D9013F2D1902D2AB4529
:10C2880088BF013F47EA0949002403E08B420CD9E3
:10C298000024A1464A46234616B1524263EB4303A3
:10C2A8001046194605B0BDE8F08FB3FA83F4002CA8
:10C2B80040F0B3808B424FF001092CBF4FF0000CC7
:10C2C8004FF0010C82428CBF67464CF00107002FEB
:10C2D800E0D13C46B946DDE722B901201146FEF718
:10C2E8003BFF0446B4FA84F3002B49D1C4EB080899
:10C2F800270C1FFA84FA0121029139464046FEF7BD
:10C308002BFF394681464046FFF754F82A0C0AFBB2
:10C3180009F342EA014B5B4509D91BEB040B09F110
:10C32800FF3904D25B4584BF09F1FF39A344C3EB4D
:10C338000B0B39465846ADB2FEF70EFF394680461C
:10C348005846FFF737F80AFB08FA45EA0145AA45B7
:10C3580007D92D1908F1FF3803D2AA4588BF08F17B
:10C36800FF3848EA0949029C94E7F643524263EBD6
:10C37800430338E7404261EB41014FF0FF362FE7B6
:10C388009C40C3F1200728FA07FA35FA07F2270C70
:10C3980008FA03FB3946504642EA0B029D400292D6
:10C3A800FEF7DAFE394683465046FFF703F8029B4C
:10C3B8001FFA84FA4FEA13490AFB0BF349EA0148CA
:10C3C800434505D918EB04080BF1FF3BC0F0AA80E0
:10C3D800C3EB080839464046FEF7BEFE394681469B
:10C3E8004046FEF7E7FF02980AFB09F31FFA80FCB4
:10C3F8004CEA0148434509D918EB040809F1FF390B
:10C4080004D2434584BF09F1FF39A04449EA0B4EE1
:10C41800C3EB0808CDF808E06FE7C4F120030AFA77
:10C4280004FADA4021FA03F842EA0A0A01FA04F99E
:10C4380030FA03F240464FEA1A4B42EA09010391E7
:10C44800594617FA04F30293FEF786FE59468146C9
:10C458004046FEF7AFFF1FFA8AF3039803FB09F281
:10C46800070C47EA0148424504D918EB0A0809F1C4
:10C47800FF3951D3C2EB0808594640460193FEF7ED
:10C488006BFE594607464046FEF794FF019B03980A
:10C4980003FB07F31FFA80FC4CEA014C634507D9FC
:10C4A800013F1CEB0A0C03D2634501D9013FD44478
:10C4B80047EA0949029FC3EB0C0C1FFA89FE4FEAB1
:10C4C8001943B8B23F0C00FB0EF800FB03F107FB61
:10C4D8000E1207FB03F002EB1842914288BF00F5E9
:10C4E800803000EB124EF44512D34FEA02421FFA95
:10C4F80088F814BF0021012102EB080C15FA04F496
:10C5080064452CBF002401F00104002C3FF4C2AEA6
:10C5180009F1FF390024BDE6424584BF09F1FF391E
:10C52800D044A7E7434584BF0BF1FF3BA0444FE746
:10C538002DE9F04F054683B00C46174680460E4657
:10C54800002B4DD18A4261D9B2FA82F353B1C3F1BB
:10C55800200411FA03F630FA04F29F4042EA060674
:10C5680000FA03F83C0C304621461FFA87FAFEF71A
:10C57800F3FD214681463046FEF71CFF4FEA18407E
:10C588000AFB09F340EA0146B34208D9F61909F152
:10C59800FF3904D2B34284BF09F1FF39F619F61AFC
:10C5A800214630461FFA88F8FEF7D6FD2146054693
:10C5B8003046FEF7FFFE0AFB05FA48EA0148C24585
:10C5C80006D9013D18EB070802D2C24588BF013DD4
:10C5D80045EA094A00263146504603B0BDE8F08FC7
:10C5E8008B425BD8B3FA83F6002E5AD18B424FF0B8
:10C5F800010A2CBF0024012482428CBF254644F046
:10C608000105002DE7D12E46AA46E4E722B901200C
:10C618001146FEF7A1FD0746B7FA87F3002B40F055
:10C62800B680E41B4FEA174BBDB201265946204697
:10C63800FEF792FD59464FEA184982462046FEF712
:10C64800B9FE05FB0AF349EA0144A34208D9E419F3
:10C658000AF1FF3A04D2A34284BF0AF1FF3AE4196F
:10C66800E41A59462046FEF777FD5946814620468A
:10C67800FEF7A0FE1FFA88F305FB09F543EA014817
:10C68800454508D918EB070809F1FF3903D2454594
:10C6980088BF09F1FF3949EA0A4A9CE70026B246F1
:10C6A80099E7C6F12001B34032FA01F724FA01F9FB
:10C6B8001F43B44030FA01F348464FEA174843EAAB
:10C6C800040101914146B2400092FEF745FD414602
:10C6D800BCB282464846FEF76DFE019804FB0AF399
:10C6E8004FEA104B4BEA014B5B4505D91BEB070B97
:10C6F8000AF1FF3AC0F09380C3EB0B0B4146584652
:10C70800FEF72AFD414681465846FEF753FE01983A
:10C7180004FB09F41FFA80FC4CEA01439C4203D94C
:10C72800DB1909F1FF3974D3009F49EA0A4A1C1B37
:10C738001FFA8AFEB8B23A0C4FEA1A4700FB0EFC01
:10C7480000FB07F302FB0E3102FB07F201EB1C4171
:10C758008B4288BF02F5803202EB114E744512D32A
:10C768004FEA01411FFA8CF214BF0023012301EBA9
:10C77800020C15FA06F666452CBF002603F00106E2
:10C78800002E3FF428AF0AF1FF3A002623E79F4026
:10C79800C3F1200134FA01F614FA03F24FEA174BF9
:10C7A80025FA01FA3046594605FA03F84AEA020A18
:10C7B800FEF7D2FC5946BDB281463046FEF7FAFD77
:10C7C8004FEA1A4C05FB09F34CEA0144A34203D98A
:10C7D800E41909F1FF3928D3E41A59462046FEF72F
:10C7E800BBFC594606462046FEF7E4FD1FFA8AF4CC
:10C7F80005FB06F344EA0144A34206D9013EE419C5
:10C8080003D2A34201D9013EE419E41A46EA0946D3
:10C818000CE79C4284BF09F1FF39DB1984E75B45CB
:10C8280084BF0AF1FF3ABB4466E7A34284BF09F11B
:10C83800FF39E419D0E700BF80B500AF134B134AA6
:10C84800126842F001021A60104B4FF000029A6021
:10C858000E4A0E4B1B6823F0847323F48033136055
:10C868000A4B0B4A5A60094B084A126822F4802284
:10C878001A60064B4FF00002DA6000F07FF800F013
:10C888000BF8044B4FF000629A6080BD00380240FC
:10C898001030002400ED00E080B483B000AF4FF00A
:10C8A80000037B604FF000033B60314B304A126855
:10C8B80042F480321A602E4B1B6803F400333B604D
:10C8C8007B6803F101037B603B68002B03D17B6825
:10C8D800B3F5A06FEFD1264B1B6803F40033002B90
:10C8E80003D04FF001033B6002E04FF000033B60D0
:10C8F8003B68012B36D11E4B1D4A926842F08002DC
:10C908009A601B4B1A4A92689A60194B184A9268A7
:10C9180042F480529A60164B164A5A60144B144AD5
:10C92800126842F080721A6000BF114B1B6803F056
:10C938000073002BF9D0104B40F203721A600C4BB5
:10C948000B4A926822F003029A60094B084A9268DF
:10C9580042F002029A6000BF054B9B6803F00C038B
:10C96800082BF9D107F10C07BD4680BC704700BF02
:10C9780000380240193C4005003C024080B5A0B098
:10C9880000AF4FF001004FF0010106F007F84FF03B
:10C998001A004FF0010105F0BDFF4FF6FF73BB67AA
:10C9A8004FF0020387F87C304FF0020387F87F309E
:10C9B8004FF0030387F87D304FF0000387F87E308F
:10C9C80007F17803CA48194605F0D0FDC8484FF06A
:10C9D80000014FF00C0205F089FEC5484FF0010137
:10C9E8004FF00C0205F082FEC1484FF002014FF0F3
:10C9F8000C0205F07BFEBE484FF003014FF00C021D
:10CA080005F074FEBA484FF004014FF00C0205F02F
:10CA18006DFEB7484FF005014FF00C0205F066FEB9
:10CA2800B3484FF006014FF00C0205F05FFEB04826
:10CA38004FF007014FF00C0205F058FEAC484FF0DC
:10CA480008014FF00C0205F051FEA9484FF009010A
:10CA58004FF00C0205F04AFEA5484FF00A014FF0CE
:10CA68000C0205F043FEA2484FF00B014FF00C02F8
:10CA780005F03CFE9E484FF00C014FF00C0205F00B
:10CA880035FE9B484FF00D014FF00C0205F02EFECD
:10CA980097484FF00E014FF00C0205F027FE94481E
:10CAA8004FF00F014FF00C0205F020FE4FF6CB734C
:10CAB800BB674FF0020387F87C304FF0020387F81A
:10CAC8007F304FF0030387F87D304FF0000387F87D
:10CAD8007E3007F178038748194605F047FD8548F9
:10CAE8004FF000014FF00C0205F000FE81484FF0B6
:10CAF80001014FF00C0205F0F9FD7E484FF00301EB
:10CB08004FF00C0205F0F2FD7A484FF006014FF0A5
:10CB18000C0205F0EBFD77484FF008014FF00C02CE
:10CB280005F0E4FD73484FF009014FF00C0205F0E1
:10CB3800DDFD70484FF00A014FF00C0205F0D6FDFC
:10CB48006C484FF00B014FF00C0205F0CFFD69481F
:10CB58004FF00C014FF00C0205F0C8FD65484FF08E
:10CB68000D014FF00C0205F0C1FD62484FF00E01B7
:10CB78004FF00C0205F0BAFD5E484FF00F014FF080
:10CB88000C0205F0B3FD4FF03003BB674FF0020312
:10CB980087F87C304FF0010387F87F304FF00003AF
:10CBA80087F87D304FF0000387F87E3007F178036F
:10CBB8005048194605F0DAFC4E484FF004014FF092
:10CBC8000C0205F093FD4B484FF005014FF00C02A5
:10CBD80005F08CFD47484FF007014FF00C0205F0B7
:10CBE80085FD4FF08003BB674FF0020387F87C3068
:10CBF8004FF0020387F87F304FF0030387F87D304A
:10CC08004FF0000387F87E3007F178033A48194659
:10CC180005F0ACFC38484FF007014FF00C0205F066
:10CC280065FD4FF00003BB664FF00003FB634FF058
:10CC380002033B644FF004037B644FF01003BB64B2
:10CC48004FF00003FB644FF000033B654FF0000317
:10CC58007B654FF00003BB654FF00003FB654FF4A5
:10CC680080533B664FF00003BB664FF000037B66C2
:10CC78004FF00003FB664FF001033B624FF00103E6
:10CC88007B624FF00403BB624FF00003FB624FF07E
:10CC98000F033B634FF000037B634FF00003BB635C
:10CCA8004FF001037B604FF00103BB604FF00403BA
:10CCB800FB604FF000033B614FF00F037B614FF0C7
:10CCC8000003BB614FF00003FB6107F120033B67E2
:10CCD80007F104037B6707F13C03184605F074FB72
:10CCE8004FF000004FF0010105F016FC06E000BF10
:10CCF80000100240000C02400004024007F18007C7
:10CD0800BD4680BD80B400AFBFF34F8FBD4680BC29
:10CD1800704700BF80B500AF054A054BDB6803F4D8
:10CD2800E061044B41EA0303D360FFF7EBFFFEE742
:10CD380000ED00E00400FA0590B585B004AF00F0FE
:10CD4800AFF900F0FFFEAD4B4FF002021A70AB4B8B
:10CD58004FF000025A70A94B4FF001029A70A74B8E
:10CD68004FF00002DA70A54B4FF065021A71A34B21
:10CD78004FF003025A71A14B4FF000029A719F4B7A
:10CD88004FF00002DA719D4B4FF003021A724FF018
:10CD9800C0404FF000014FF40022F4F7F9FD40F6CF
:10CDA800782022F0A5FD03461A46954B1A60944B4D
:10CDB8001B68184602F03EF9924B4FF400421A8362
:10CDC800914B4FF010021A838E4B4FF400621A8376
:10CDD8008C4B4FF480521A83894B1A6892F8B039F9
:10CDE8006FF3000382F8B039854B1A6892F8B039AE
:10CDF8006FF3410382F8B039814B1A6892F8B03961
:10CE08006FF3820382F8B0397D4B1A6892F8B03913
:10CE18006FF3C30382F8B039794B1A6892F8B039C6
:10CE28006FF3041382F8B039754B1A6892F8B03969
:10CE38006FF3451382F8B039714B1A6892F8B0391C
:10CE480043F0400382F8B0396D4B1A6892F8B03954
:10CE58006FF3C71382F8B039694B1B684FF00002B3
:10CE6800C3F83C2A664B1B684FF00002C3F84C2AF3
:10CE7800634B1B684FF00002C3F8502A604B1B68D5
:10CE88004FF00002C3F8402A5D4B1B684FF00002C8
:10CE9800C3F8442A5A4B1B684FF00002C3F8542ABF
:10CEA800574B1B684FF00002C3F8582A544B1B68B5
:10CEB8004FF00002C3F8482A514B1B68184604F08B
:10CEC800E3FB4F4B1B68184603F07EFC4C4B1B687A
:10CED800184604F0A3FB4A4B1B68494A1268D2F86B
:10CEE800402A4FF00301009101924FF00002029294
:10CEF8004FF000020392454845494FF4807221F0F3
:10CF080013FD3F4B1B683E4A1268D2F8442A4FF083
:10CF18000301009101924FF0000202924FF00002CB
:10CF280003923C483C494FF4807221F0FDFC344B9D
:10CF38001B68334A1268D2F8542A4FF00201009154
:10CF480001924FF0000202924FF000020392334820
:10CF580033494FF4007221F0E7FC294B1B68284A3B
:10CF68001268D2F83C2A4FF00201009101924FF06A
:10CF7800000202924FF0000203922A482A494FF415
:10CF8800486221F0D1FC1E4B1B684FF00002C3F829
:10CF98005C2A1B4B1B684FF00002C3F8602A184B31
:10CFA8001B684FF00002C3F8642A154B1B684FF04A
:10CFB8000002C3F8682A124B1B684FF00002C3F83E
:10CFC8006C2A0F4B1B684FF00002C3F8702A0C4BF9
:10CFD8001B684FF00002C3F8742A144B4FF000028C
:10CFE8001A60074B1C684FF001004FF000014FF02A
:10CFF800030221F0B5F803461AE000BFE83200202A
:10D00800E032002000000240000402409D170108A1
:10D0180030FB020809F3000838FB020875D1000844
:10D0280040FB0208B1E6000848FB0208E432002091
:10D03800C4F8743A194B1B68D3F8743A002B0CD017
:10D04800164B1B68D3F8743A18464FF000014FF09E
:10D0580000024FF0000321F0E1F8104B1B68D3F8F1
:10D06800743A18464FF000014FF000024FF00003E9
:10D0780021F0D4F845F2555005F062FE4FF0030058
:10D0880005F06EFE4FF4006005F07AFE05F088FEAC
:10D0980005F092FE21F080FDFEE700BFE03200209F
:10D0A80080B500AF4FF040004FF0010105F054FC8F
:10D0B8004FF0010005F056FD4FF010004FF0010150
:10D0C80005F04AFC4FF020004FF0010105F044FC48
:10D0D80080BD00BF80B582B000AF78607B68DBB2EE
:10D0E8001148194604F07EFD00BF0F484FF040017B
:10D0F80004F0B2FD0346002BF7D07B680A2B0DD154
:10D1080009484FF00D0104F06DFD00BF06484FF0CF
:10D11800400104F0A1FD0346002BF7D07B681846B8
:10D1280007F10807BD4680BD004C004080B582B0BD
:10D1380000AF78603960FFF7EDFDFEE780B483B09B
:10D1480000AF0346FB71FB79092B04D9FB7903F186
:10D158003703DBB203E0FB7903F13003DBB2184697
:10D1680007F10C07BD4680BC704700BF80B592B080
:10D1780000AF78604FF0000387F847307B683B6466
:10D188003B6C4FF0030283F8AE293B6C4FF064020E
:10D19800A3F8AC293B6C4FF0010283F8AA293B6C39
:10D1A800D3F8743A18464FF000014FF096024FF04A
:10D1B800000321F00DF90346012B40F0DE803B6CA3
:10D1C80093F87C34052B00F2CD8001A252F823F0AD
:10D1D800F1D10008FDD10008DFD200080DD3000806
:10D1E80015D3000857D300083B6C4FF0030283F8AF
:10D1F8007C24B7E069486A4904F030FF0346012BF4
:10D2080017D16648664904F06BFF664B4FF0000281
:10D218001A703B6C4FF06402A3F8AC293B6C4FF0DA
:10D22800030283F8AE293B6C4FF0020283F87C249A
:10D2380098E03B6CB3F8AC39002B14BF00220122F4
:10D24800D2B203F1FF3399B23B6CA3F8AC19002AB0
:10D258003CD03B6C4FF06402A3F8AC293B6C93F8CC
:10D26800AE39002B14BF00220122D2B203F1FF33E2
:10D27800D9B23B6C83F8AE19002A22D03B6C4FF030
:10D288006402A3F8AC293B6C4FF0030283F8AE2983
:10D298003B6C4FF0050283F87C243B6C4FF0010295
:10D2A80083F8AA293A6C92F8B0396FF3C30382F86D
:10D2B800B0393A6C92F8B03943F0800382F8B0394B
:10D2C80004E03B6C4FF0000283F87C244FF00A0026
:10D2D80021F036FC46E03A6C92F8B03943F0080386
:10D2E80082F8B0393A6C92F8B0396FF3C71382F804
:10D2F800B0393B6C4FF0000283F8AA29386C00F073
:10D308007FF82FE0386C00F081FB2BE026484FF0C7
:10D31800205104F0A3FE0346012B0DD122484FF003
:10D32800205104F0DDFE214B4FF000021A703B6CD7
:10D338004FF0000283F87C243B6C4FF06402A3F8A2
:10D34800AC293B6C4FF0030283F8AE290AE03B6C32
:10D358004FF0000283F87C243B6C4FF0030283F803
:10D368007D2400BF3B6C93F87C34002B05D03B6CCC
:10D3780093F87C34052B7FF422AF3B6CD3F8743AD6
:10D3880018464FF000014FF000024FF0000320F064
:10D3980045FF4FF0320021F0D3FB00E788640240DC
:10D3A8000008002098060020B86402409906002072
:10D3B80080B487B000AFF860B9607A604FF00003BE
:10D3C8007B6110E07B69FA68D3181A787B69B968C1
:10D3D800CB181B789A4202D04FF0010309E07B6911
:10D3E80003F101037B617A697B689A42EADB4FF0BB
:10D3F8000003184607F11C07BD4680BC704700BFF4
:10D4080090B587B000AF78607B68FB604FF0000391
:10D418003B61FB6893F89937022B31D1FB6893F88D
:10D428009B3703F107039BB2FA68D31893F899372F
:10D43800032B25D1FB6803F5B06202F10B02FB68F0
:10D4480003F5F26303F109031046194640F2071287
:10D45800F4F79CF9FB6893F88F25FB6883F8A829F3
:10D46800FB684FF0010283F87E24FB684FF000024E
:10D4780083F87C24FB6893F8A839662B06D05AE217
:10D48800FB684FF0050283F87C245AE2FB6893F8A6
:10D498008E3503F07F03002B03D0012B00F0A28010
:10D4A8003EE2FB6803F18102FB6803F5B2631046B4
:10D4B80019464FF02002FFF77BFF03461A46484BF8
:10D4C8001B7842EA0303DAB2454B1A70444B1B78C7
:10D4D800002B0FD0FB6803F18102FB6803F5B063F2
:10D4E80003F10B0303F10503104619464FF0200220
:10D4F800F4F74CF9FB6803F16102FB6803F5B663C6
:10D50800104619464FF02002FFF752FF03461A460D
:10D51800334B1B7842EA0303DAB2314B1A70304BB3
:10D528001B78002B0FD0FB6803F16102FB6803F541
:10D53800B06303F10B0303F12503104619464FF0BE
:10D548002002F4F723F94FF000037B6135E07A6994
:10D558003B69D4187B6903F14503FA68D31893F83B
:10D568008B354FEA1313DBB21846FFF7E7FD034686
:10D578001A46FB681B1983F822227A693B69D3187B
:10D5880003F101047B6903F14503FA68D31893F8A2
:10D598008B3503F00F03DBB21846FFF7CFFD0346C8
:10D5A8001A46FB681B1983F822223B6903F1010321
:10D5B8003B617B6903F101037B617B690F2BC6DD4E
:10D5C800FB684FF0000283F84222FB684FF000022C
:10D5D80083F84322FB684FF0000283F87C249FE124
:10D5E800A0060020FB6803F5107303F106031A4632
:10D5F800FB6803F5B263104619464FF00402FFF7C3
:10D60800D7FE03461A46A84B1B7842EA0303DAB250
:10D61800A54B1A70A44B1B78002B11D0FB6803F59F
:10D62800107303F10603FA6802F5B06202F10B0207
:10D6380002F10502184611464FF00402F4F7A6F865
:10D64800FB6803F5127303F102031A46FB6803F53E
:10D65800B26303F10403104619464FF00402FFF7C2
:10D66800A7FE03461A46904B1B7842EA0303DAB238
:10D678008D4B1A708C4B1B78002B11D0FB6803F56F
:10D68800127303F10203FA6802F5B06202F10B02A9
:10D6980002F10902184611464FF00402F4F776F831
:10D6A800FB6803F5127303F106031A46FB6803F5DA
:10D6B800B363104619464FF00402FFF779FE03469C
:10D6C8001A46794B1B7842EA0303DAB2764B1A7092
:10D6D800754B1B78002B11D0FB6803F5127303F10F
:10D6E8000603FA6802F5B06202F10B0202F10D02BC
:10D6F800184611464FF00402F4F748F8FB6803F5A2
:10D70800147303F102031A46FB6803F5B26303F1CD
:10D718000C03104619464FF00402FFF749FE034672
:10D728001A46614B1B7842EA0303DAB25E4B1A7061
:10D738005D4B1B78002B11D0FB6803F5147303F1C4
:10D748000203FA6802F5B06202F10B0202F111025B
:10D75800184611464FF00402F4F718F8FB6803F571
:10D76800147303F106031A46FB6803F5B463104605
:10D7780019464FF00402FFF71BFE03461A464A4BB0
:10D788001B7842EA0303DAB2474B1A70464B1B7800
:10D79800002B11D0FB6803F5147303F10603FA6834
:10D7A80002F5B06202F10B0202F1150218461146A9
:10D7B8004FF00402F3F7EAFFFB6803F5087202F181
:10D7C8000102FB6803F5B46303F10403104619462C
:10D7D8004FF00102FFF7ECFD03461A46324B1B7867
:10D7E80042EA0303DAB2304B1A702F4B1B78002B36
:10D7F80011D0FB6803F5087303F10103FA6802F519
:10D80800B06202F10B0202F11902184611464FF0FC
:10D818000102F3F7BBFFFB6803F1E102FB6803F5C4
:10D82800B46303F10503104619464FF04002FFF7B1
:10D83800BFFD03461A461C4B1B7842EA0303DAB2C3
:10D84800194B1A70184B1B78002B0FD0FB6803F18B
:10D85800E102FB6803F5B06303F10B0303F11A035C
:10D86800104619464FF04002F3F790FFFB6803F5A6
:10D87800B07202F10102FB6803F5BC6303F1050312
:10D88800104619464FF04002FFF792FD03461A462C
:10D89800054B1B7842EA0303DAB2034B1A70024BBA
:10D8A8001B78002B14D001E0A0060020FB6803F5CC
:10D8B800B07303F10103FA6802F5B06202F10B02DA
:10D8C80002F15A02184611464FF04002F3F75EFF84
:10D8D8001E4B1B78002B1DD0FB6803F1380318463C
:10D8E8004FF0000140F222224FF0000301F074FFD4
:10D8F800FB68D3F82C3A5B79012B08D102F09EF92A
:10D908000346134819464FF006021FF09FF9FFF728
:10D9180001FA05E0FB684FF0010283F8A92900BF6E
:10D92800FB684FF0000283F87C24FB684FF000028C
:10D9380083F87E2405E0FB684FF0010283F8A729ED
:10D9480000BF07F11C07BD4690BD00BFA006002020
:10D958005C33002080B586B000AFF860B9607A60AB
:10D968003B6078684FF0AA013A68F4F711F8234849
:10D978004FF0000104F056FB21484FF0000104F07D
:10D9880051FB20484FF0C0014FF0000204F03EF96F
:10D998001C4B9B88FB821B4B1B88FB8219484FF052
:10D9A800400104F079F915484FF0305104F098FB24
:10D9B8001348154904F094FB104BFA68DA600F4BD2
:10D9C800BA685A600E4B7A68DA600D4B3A685A604A
:10D9D8000C484FF0C0014FF0010204F017F9084855
:10D9E8004FF0010104F01EFB04484FF0010104F060
:10D9F80019FB07F11807BD4680BD00BFB864024097
:10DA08008864024000100140000C002090B585B0E9
:10DA180000AF78607B68FB60FB684FF06402A3F896
:10DA2800AC29FB6893F87D24384B5A7137484FF07E
:10DA3800060101F01BFDB860BB68DAB2334BDA713E
:10DA4800BB684FEA2323DAB2304B9A71FB6893F82C
:10DA58007F34012B34D1FB6803F5D26202F1020254
:10DA6800FB6803F5906303F10403F968B1F88014C7
:10DA78000C46104619462246F3F788FEFB6803F564
:10DA8800D26202F10202FB68B3F880341946FB68DF
:10DA980003F5F26303F10903F868B0F88204044659
:10DAA80010461A462346FFF755FFFB684FF0000261
:10DAB80083F87F24FB684FF0040283F87C2421E07C
:10DAC800FB6803F5D26303F1020318460F494FF0D0
:10DAD8000902F3F75BFEFB6803F5D26202F102026A
:10DAE800FB6803F5F26303F1090310464FF00901DF
:10DAF8001A4640F20713FFF72DFFFB684FF00102AB
:10DB080083F87C2407F11407BD4690BDE832002055
:10DB180080B400AFBFF34F8FBD4680BC704700BFD5
:10DB280080B500AF054A054BDB6803F4E061044BA0
:10DB380041EA0303D360FFF7EBFFFEE700ED00E0E7
:10DB48000400FA0580B500AF00F0C6F800F0BEF991
:10DB580000F0B2FA00F066FB00F010F800F006FBE7
:10DB680001F0A6FC00F0AEFB00F03CF84FF001001D
:10DB780000F0C4FB00F008FC80BD00BF80B582B097
:10DB880000AF4FF418433B604FF000037B714FF038
:10DB980001033B714FF00103BB714FF00003FB71B0
:10DBA8003B460E48194604F0E1FC4FF010033B6079
:10DBB8004FF000037B714FF001033B714FF00103FD
:10DBC800BB714FF00003FB713B460548194604F052
:10DBD800CDFC07F10807BD4680BD00BF000002402C
:10DBE8000004024080B5B0B000AF4FF060604FF065
:10DBF800010104F08FFE11F0CDFB12F081F900BF96
:10DC080012F090F90346012BFAD007F104031846E5
:10DC180011F0D0FB4FF001037B604FF000033B6233
:10DC28004FF40073FB624FF000033B634FF00003B7
:10DC3800FB634FF00003BB644FF000033B654FF0FC
:10DC480000037B654FF00003BB654FF48063BB6244
:10DC58004FF00003C7F884304FF00073C7F88830DE
:10DC68004FF40013C7F890304FF00003C7F898300E
:10DC78004FF00003C7F89C304FF00403C7F8A430F6
:10DC88004FF00073C7F8A8304FF48033C7F8AC30B2
:10DC98004FF48003C7F8B0304FF40053C7F8B430DE
:10DCA8004FF48043C7F8BC3007F1040318464FF01F
:10DCB800010111F053FC0246054B1A6005484FF06C
:10DCC800010112F071F907F1C007BD4680BD00BF20
:10DCD800A40600204000010080B584B000AF4FF6D4
:10DCE800FF73FB814FF01F004FF0010104F012FE9B
:10DCF8004FF480404FF0010104F094FE4FF480731C
:10DD08007B604FF003037B724FF002033B724FF0CE
:10DD18000003BB724FF00003FB7207F1040368486D
:10DD2800194604F023FC4FF0000004F00DFF4FF0FB
:10DD38008F037B6007F104036148194604F016FC61
:10DD48005F484FF000014FF00B0204F0CFFC5C4835
:10DD58004FF001014FF00B0204F0C8FC58484FF097
:10DD680002014FF00B0204F0C1FC55484FF00301CB
:10DD78004FF00B0204F0BAFC51484FF007014FF086
:10DD88000B0204F0B3FC43F603537B6007F1040372
:10DD98004C48194604F0EAFB4A484FF000014FF09E
:10DDA8000B0204F0A3FC47484FF001014FF00B02AF
:10DDB80004F09CFC43484FF008014FF00B0204F0BC
:10DDC80095FC40484FF00A014FF00B0204F08EFC1E
:10DDD8003C484FF00B014FF00B0204F087FC394828
:10DDE8004FF00C014FF00B0204F080FC35484FF067
:10DDF8000D014FF00B0204F079FC4FF03E037B60FD
:10DE080007F104033048194604F0B0FB2E484FF0E0
:10DE180001014FF00B0204F069FC2B484FF002019E
:10DE28004FF00B0204F062FC27484FF003014FF05B
:10DE38000B0204F05BFC24484FF004014FF00B0286
:10DE480004F054FC20484FF005014FF00B0204F099
:10DE58004DFC4FF040037B604FF001033B724FF0E5
:10DE68000003FB724FF002037B724FF00103BB7299
:10DE780007F104031348194604F078FB4FF0080330
:10DE88007B604FF000033B7207F104030D4819460D
:10DE980004F06CFB0B484FF0400104F019FCFB89BF
:10DEA80003F1FF33FB81FB89002BF8D105484FF0C4
:10DEB800400104F0FFFB07F11007BD4680BD00BF1D
:10DEC80000000240000402400008024080B5A6B0ED
:10DED80000AF4FF010004FF0010104F0A3FD4FF424
:10DEE800C063C7F880304FF0020387F884304FF0E2
:10DEF800000387F886304FF0000387F887304FF02B
:10DF0800020387F8853007F180036448194604F056
:10DF18002DFB62484FF009014FF0070204F0E6FBC1
:10DF28005E484FF00A014FF0070204F0DFFB4FF4A0
:10DF38009643C7F888304FF00003A7F88C304FF0AD
:10DF48000003A7F88E304FF00003A7F890304FF089
:10DF58000003A7F894304FF00C03A7F8923007F1AC
:10DF680088034F48194603F049FD4D484FF0010119
:10DF780003F018FE4FF480004FF0010104F0CAFCD2
:10DF8800484803F019FF4FF000637B64464BBB64BD
:10DF98004FF00003FB644FF000037B654FF0400334
:10DFA8003B654FF00003BB654FF48063FB654FF0A2
:10DFB80000033B664FF000037B664FF00003BB662F
:10DFC8004FF00003FB664FF00003BB674FF0000300
:10DFD8003B644FF000033B674FF003037B6707F197
:10DFE80044033048194603F0C1FF2D484FF0800123
:10DFF8004FF0010203F00AFE2A482C4904F000F908
:10E0080028484FF0010104F00DF8294803F0D4FE28
:10E018004FF00063BB60244BFB604FF000033B6193
:10E028004FF00003BB614FF000037B614FF000032A
:10E03800FB614FF480633B624FF000037B624FF05B
:10E048000003BB624FF00003FB624FF000033B6329
:10E058004FF00003FB634FF000033B644FF00003F5
:10E068007B634FF00303BB6307F1080310481946AD
:10E0780003F07CFF0A484FF040014FF0010203F023
:10E08800C5FD0B480B4904F0BBF809484FF00101E6
:10E0980003F0C8FF07F19807BD4680BD00000240A5
:10E0A80000100140B86402400410014000800028BC
:10E0B800886402400088002080B586B000AF4FF425
:10E0C80080104FF0010104F08BFC4FF480533B604B
:10E0D8004FF002033B714FF00003BB714FF0000398
:10E0E800FB714FF002037B713B461D48194604F053
:10E0F8003DFA1B484FF00C014FF0080204F0F6FA05
:10E108004FF004033B603B461648194604F02EFACC
:10E1180014484FF002014FF0080204F0E7FA4FF4F8
:10E12800E133BB604FF00003BB814FF00003FB817C
:10E138004FF000033B824FF00003BB824FF00C030B
:10E148007B8207F108030848194603F057FC064884
:10E158004FF0010103F026FD07F11807BD4680BD09
:10E1680000080240000C02400050004080B5A6B0F4
:10E1780000AF4FF400204FF0010104F031FC4FF4E0
:10E188004063C7F880304FF0020387F884304FF0BF
:10E19800000387F886304FF0000387F887304FF088
:10E1A800020387F8853007F180031C48194604F0FC
:10E1B800DDF91A484FF00A014FF0080204F096FA08
:10E1C80016484FF00B014FF0080204F08FFA4FF495
:10E1D800E133C7F888304FF00003A7F88C304FF0D0
:10E1E8000003A7F88E304FF00003A7F890304FF0E7
:10E1F8000003A7F894304FF00C03A7F8923007F10A
:10E2080088030748194603F0F9FB05484FF0010158
:10E2180003F0C8FC07F19807BD4680BD000802401E
:10E22800004C004080B586B000AF4FF020004FF0A2
:10E23800010104F0F7FB4FF0C0033B604FF002030D
:10E248003B714FF00003BB714FF00103FB714FF0BE
:10E2580002037B713B461948194604F087F91748B1
:10E268004FF006014FF0080204F040FA13484FF04F
:10E2780007014FF0080204F039FA4FF41653BB6057
:10E288004FF00003BB814FF00003FB814FF0000308
:10E298003B824FF00003BB824FF00C037B8207F1F7
:10E2A80008030748194603F0A9FB05484FF0010188
:10E2B80003F078FC07F11807BD4680BD000802404E
:10E2C8000014014080B582B000AF4FF4A06003F0A5
:10E2D800F5FC4FF03D033B714FF002037B714FF0AB
:10E2E8000003BB714FF00103FB7107F104031846EB
:10E2F80003F0F6FC07F10807BD4680BD80B584B081
:10E3080000AF0346FB804FF00003FB60FB88184614
:10E318004FF0110111F0F8FE0346FB60FB6843F073
:10E328000303FB60FB689BB2FA8810464FF01101AB
:10E338001A4611F043FF0346002B02D14FF00003A9
:10E348001CE0FB8818464FF0120111F0DDFE034671
:10E35800FB60FB6843F02003FB60FB689BB2FA8814
:10E3680010464FF012011A4611F028FF0346002B01
:10E3780002D14FF0000301E04FF00103184607F106
:10E388001007BD4680BD00BF80B586B000AF4FF016
:10E3980002004FF0010104F0BDFA4FF480404FF045
:10E3A800010104F03FFB4FF000033B754FF0000301
:10E3B800FB754FF008033B6107F110031948194634
:10E3C80004F0D4F84FF001004FF0030104F06EFBA5
:10E3D8004FF00803BB604FF000033B734FF00C0392
:10E3E8007B734FF00103BB7307F10803184603F072
:10E3F80035FF4FF4C06003F061FC4FF009033B7137
:10E408004FF000037B714FF00003BB714FF0010325
:10E41800FB7107F10403184603F062FC07F11807C3
:10E42800BD4680BD0004024080B582B000AF0346FF
:10E43800FB80FB8818464FF0100111F065FE03467B
:10E4480003F00103DBB2002B02D0FFF769FB09E000
:10E45800094B4FF000021A60084B1B684FF001028D
:10E4680083F87D24FB8818464FF0120111F04CFE0A
:10E4780007F10807BD4680BDA4060020E032002051
:10E4880080B400AFBD4680BC704700BF80B400AF09
:10E49800FEE700BF80B400AFFEE700BF80B400AF66
:10E4A800FEE700BF80B400AFFEE700BF80B400AF56
:10E4B800BD4680BC704700BF80B500AF21F0ECF9C5
:10E4C80080BD00BF80B500AF4FF0080003F044FFE7
:10E4D8000346002B07D04FF00100FFF7A5FF4FF0D0
:10E4E800080003F063FF80BD80B500AF4FF008005F
:10E4F80003F032FF0346002B07D04FF00100FFF76F
:10E5080093FF4FF0080003F051FF80BD80B582B043
:10E5180000AF4FF000037B604FF0400011F022FD88
:10E528000346012B0BD1104B1A6807F10403104660
:10E538004FF000011A464FF000031FF0FFFE4FF0A6
:10E54800400011F061FD4FF4803011F05DFD7B68F3
:10E55800002B04D07B68002B01D021F04BF907F188
:10E568000807BD4680BD00BFE80C002080B500AF9D
:10E578000748084903F0E2FD0346002B07D0064B85
:10E588004FF001021A700248024903F039FE80BDBB
:10E59800B8640240008000289906002080B582B047
:10E5A80000AF4FF000037B601348144903F0C6FD29
:10E5B8000346002B0FD0124B4FF001021A70114B7B
:10E5C8001A6807F1040310464FF000011A464FF08D
:10E5D80000031FF0B3FE0848084903F011FE7B68EA
:10E5E800002B04D07B68002B01D021F003F907F140
:10E5F8000807BD4680BD00BF88640240008800202F
:10E6080098060020E432002080B400AFBFF34F8F9B
:10E61800BD4680BC704700BF80B500AF054A054BBA
:10E62800DB6803F4E061044B41EA0303D360FFF7BE
:10E63800EBFFFEE700ED00E00400FA0580B485B0CA
:10E6480000AFF860B9607A6007F11407BD4680BC76
:10E65800704700BF80B487B000AFF860B9607A60D7
:10E668004FF00003FB8212E0FB8AFA68D3181A788D
:10E67800FB8AB968CB181B7852B25BB29A4202D0B7
:10E688004FF0010309E0FB8A03F10103FB82FA8AD8
:10E698007B689A42E8D34FF00003184607F11C073D
:10E6A800BD4680BC704700BF80B5ADF5286D86B00B
:10E6B80004AF07F10803A3F1040318604FF0000347
:10E6C800C7F87C3A4FF00003C7F8783A07F1080317
:10E6D800A3F104031B68C7F8743A07F5206303F134
:10E6E8001403184601F04AFAD7F8743A07F520627D
:10E6F80002F11402C3F82C2A4FF00003C7F8703A4D
:10E70800D7F8743A4FF00A02C3F8382AD7F8743A9F
:10E718004FF00002C3F8342AD7F8743AD3F8342AF1
:10E7280007F12803A3F11C031A60D7F8742A92F89A
:10E73800B03943F0200382F8B039D7F8743A4FF073
:10E74800020283F87D24D7F8743A93F8303A032B01
:10E7580040F0AB82D7F8743A93F8AA39002B40F00E
:10E76800A4829C484FF000014FF06002F3F710F9C3
:10E7780007F51F6318464FF000014FF01E02F3F72C
:10E7880007F9D7F8743A03F5407303F10303184601
:10E7980001F070FCC7F86C0AD7F8743A03F54073B7
:10E7A80003F1030307F51F621846114601F03AFC0E
:10E7B80007F12803A3F11C031B68184643F69821A8
:10E7C80006F000F807F51F6207F12803A3F11C0300
:10E7D80018461146D7F86C2A16F00AFCC7F87C0AC6
:10E7E800D7F87C3A002B16D0D7F8743AD3F8383AD1
:10E7F800002B14BF00220122D2B203F1FF31D7F857
:10E80800743AC3F8381A002A01D0FFF705FF40F61A
:10E81800B83020F095F9D7F8743A93F8AA39002B54
:10E8280040F04282D7F87C3A002BCBD16A481DF0E1
:10E83800DFFDC7F87C0AD7F87C3A002B08D007F12F
:10E848002803A3F11C031B68184616F069FC10E2A4
:10E8580061484FF000011DF02BFE5F484FF00001AA
:10E868001DF029FE5C485D495D4A1DF027FE5D4BA1
:10E878001B689B6858485C491A461DF022FE07F140
:10E888002803A3F11C0307F12802A2F11C0200923D
:10E89800514856491A46564B1DF016FE4E484FF041
:10E8A80001014FF416724B4B1DF014FE4A485149B2
:10E8B8001DF014FE07F12803A3F1180318464FF0C2
:10E8C80000014FF48062F3F763F807F12803A3F11E
:10E8D800180307F5206202F1140210461946D7F80A
:10E8E800742A01F0E7FBC7F8780A07F12803A3F1B7
:10E8F8001C031B68184643F6982105F063FF07F1CF
:10E908002803A3F1180334481946D7F8782A1EF0CB
:10E918009DF9C7F87C0A0DE0D7F87C3A13F5796FB2
:10E9280008D007F12803A3F11C031B68184616F04A
:10E93800F7FB9EE1D7F87C3A002BEDDD40F2FF3380
:10E94800C7F8783A07F12803A3F1180318464FF0DF
:10E9580000014FF48062F3F71BF807F12803A3F1D5
:10E9680018031D481946D7F8782A1EF0EBF8C7F89F
:10E978007C0AD7F87C3A13F5796F0DD0D7F87C3A32
:10E9880013F5104F0AD0D7F87C3A002B08DDD7F8DA
:10E998007C3AC7F8783A04E000BF02E000BF00E024
:10E9A80000BF07F12803A3F1180307F5206202F15D
:10E9B80014021046194601F051FD97F8193A012B37
:10E9C8001AD007F12803A3F11C031B68184616F098
:10E9D800A7FB4EE1F43200205C33002011F0000860
:10E9E80058330020A400002045E6000879500208AA
:10E9F800D550020864000020D7F8743A03F50A637A
:10EA080018464FF0000140F20712F2F7C1FFD7F89D
:10EA1800742A92F8B0396FF3451382F8B0394FF081
:10EA2800000387F8203A4FF002030093A34B0193A9
:10EA38004FF0000302934FF000030393A048A1494D
:10EA48004FF4A062D7F8743A1FF06EFF20F072F905
:10EA5800C7F8800AD7F8803AC7F8843AD7F8743AE2
:10EA68004FF0000283F87D24D7F8743AD3F8743A4B
:10EA780018464FF000014FF4C8724FF000031FF022
:10EA8800A7FC0346012B40F08D80D7F8743A93F821
:10EA98007E34012B79D1D7F8743A03F5B06303F1CA
:10EAA8000B031A46D7F8743A03F50A631046194659
:10EAB80040F20712FFF7CEFD0346002B05D1D7F829
:10EAC800743A93F8A939002B59D0D7F8743A4FF013
:10EAD800000283F8A929D7F8743A03F50A62D7F82F
:10EAE800743A03F5B06303F10B031046194640F27C
:10EAF8000712F2F74BFE4FF4F073C7F8103AD7F845
:10EB0800743A03F50A6307F5016107F521620846BF
:10EB180011461A4640F2071312F09EFB0346C7F847
:10EB2800103A07F5826318464FF000014FF48062EF
:10EB3800F2F72EFF07F501631846F3F7E9FD0346E0
:10EB480007F5016107F58262084611461A464FF03B
:10EB5800020301F06DF9C7F8680A07F582635A489D
:10EB68001946D7F8682A1EF071F8C7F87C0AD7F852
:10EB78007C3A002B63DDD7F8803AC7F8843AD7F897
:10EB8800743A4FF0000283F87E24D7F8743AD3F829
:10EB9800743A18464FF000014FF000024FF000039E
:10EBA8001FF03CFB20F0C6F8C7F8800AD7F8802A87
:10EBB800D7F8843AD21A43F698239A4225D9D7F837
:10EBC800803AC7F8843A97F8203A002B18D100F019
:10EBD800E9FF03463C4819464FF006021EF036F896
:10EBE800C7F87C0AD7F87C3A002B04DC4FF0020304
:10EBF80087F8193A24E04FF0010387F8203A04E037
:10EC08004FF0020387F8193A1AE007F12803A3F135
:10EC18001C031B68184605F0E7FDC7F8700A97F84B
:10EC2800193A012B0CD1D7F8703A002B08D1D7F834
:10EC3800743A93F8AA39002B3FF416AF00E000BFEE
:10EC480007F12803A3F11C031B68184616F068FA9D
:10EC58004FF0020387F8193A184B1B68002B08D0AD
:10EC6800164B1B6818461FF019FF144B4FF0000293
:10EC78001A6015481EF052F813484FF0000140F68C
:10EC88007C02F2F785FED7F8742A92F8B0396FF350
:10EC9800410382F8B039D7F8742A92F8B03943F0B2
:10ECA800200382F8B03900E000BF4FF0020387F874
:10ECB800193A41F288301FF043FF21E55433002010
:10ECC800D5EC000884FC02085C330020B0B5ADF533
:10ECD800026D86B000AF07F11803A3F114031860A2
:10ECE8004FF00003A7F832384FF00003C7F82C386C
:10ECF8004FF00003C7F8283807F11803A3F11403ED
:10ED08001B68C7F82438D7F82438D3F82C3A5B792D
:10ED1800012B40F0638140F2FF33A7F8223807F552
:10ED28008563A3F10C0318464FF000014FF480628D
:10ED3800F2F72EFED7F82438D3F8343A1846AF49FC
:10ED480005F040FD4FF00003C7F83438D7F83428F1
:10ED580007F58563A3F10C039A18B7F82218D7F8BA
:10ED68003438CB1AA64811461A461DF0EBFEC7F8F0
:10ED78002C08D7F82C3813F5796F1AD0D7F82C3817
:10ED8800002B40F32281D7F83428D7F82C38D31831
:10ED9800C7F83438D7F82438D3F82C1AD7F83428D9
:10EDA80007F58563A3F10C030846194600F06CFFCC
:10EDB80000E000BFD7F82438D3F82C3A5B7BD7F8AB
:10EDC8003428D21AD7F82438D3F82C3A1B689A4238
:10EDD80005D0B7F82228D7F834389A42B6DCB7F805
:10EDE8002228D7F834389A42C0F2F180D7F824386C
:10EDF800D3F82C3A9B79092B17D100F0F9FE03467A
:10EE08007F4819464FF006021DF020FFC7F82C086E
:10EE1800D7F82C38002B40F3DC80D7F82438D3F807
:10EE28002C3A4FF001021A7375E7D7F82438D3F853
:10EE38002C3A9B790A2B06D1D7F824384FF00002D8
:10EE480083F87D2467E7D7F82438D3F82C3A9B79E0
:10EE5800022B07D0D7F82438D3F82C3A9B79012B0A
:10EE680040F0A08007F11803A3F10C034FF480626F
:10EE78001A60D7F82438D3F82C3A9D68D7F8243884
:10EE8800D3F82C3A1C6807F13802A2F11C0207F1EA
:10EE98001803A3F10C03104619462A46234612F01C
:10EEA80001FBC7F81C08D7F81C38002B6ED1D7F81F
:10EEB8002438D3F8743A18464FF000014FF4C8725A
:10EEC8004FF000031FF084FA0346012B68D1D7F8EE
:10EED80024384FF0000283F8AE2907F11803A3F194
:10EEE8000C031A6840F207139A4274DC07F13803DE
:10EEF800A3F11C031B78022B3AD107F13803A3F1C5
:10EF08001C039B7803F107039BB21A4607F13803E9
:10EF1800A3F11C039B5C032B2AD1D7F8243803F5F3
:10EF2800906202F1040207F11803A3F10C031B68B5
:10EF38001C4607F13803A3F11C0310461946224664
:10EF4800F2F724FC07F11803A3F10C031B689AB22B
:10EF5800D7F82438A3F88024D7F824384FF00002D3
:10EF6800A3F88224D7F824384FF0010283F87F24CD
:10EF7800D7F82438D3F8743A18464FF000014FF008
:10EF880000024FF000031FF049F909E0D7F81C38D8
:10EF9800102B03D0122B00D001E000E000BF1DE0D1
:10EFA80000BFB8E6D7F82438D3F82C3A9B79082B59
:10EFB80013D100F043FE0346114819464FF00602EC
:10EFC8001DF044FEC7F82C0808E000BF06E000BFAB
:10EFD80004E000BF02E000BF00E000BFD7F824381B
:10EFE800D3F82C3A4FF002025A71064B4FF0000248
:10EFF8001A604FF000001FF051FD84E6804F1200A8
:10F008005C3300205433002080B584B000AF7860B2
:10F0180000BF4FF0010003F0CBFD0346002BF8D0F2
:10F0280003F0BCFDF860FB68184607F11007BD4601
:10F0380080BD00BF80B586B000AF78607B683B615B
:10F048003B6903F1380318464FF0000140F22222D1
:10F05800F2F79EFC3B6903F5167303F102031846A9
:10F068004FF0000140F22222F2F792FC3B6903F1D3
:10F07800380318464FF0000140F222224FF00003F7
:10F0880000F096FC3B6903F13803184688494FF0B5
:10F098002702F3F76DFB0346002B00F0F680854846
:10F0A80006F0D0FD02463B69C3F846226FF0FF0028
:10F0B80006F0C8FD02463B69C3F84A227E4806F0BE
:10F0C800C1FD02463B69C3F84E227B4806F0BAFDF3
:10F0D80002463B69C3F85222784806F0B3FD02465F
:10F0E8003B69C3F85622764800F0FCF8F860FB68E4
:10F0F8004FEA1343DAB2FB68DBB282EA0303DAB2FF
:10F108003B6983F8A620FB684FEA1342FB684FEA85
:10F1180003434FEA134382EA03034FEA1323DAB2A5
:10F128003B6983F8A520674800F0DCF8F860FB68C5
:10F138004FEA1343DAB2FB68DBB282EA0303DAB2BE
:10F148003B6983F8A420FB684FEA1342FB684FEA47
:10F1580003434FEA134382EA03034FEA1323DAB265
:10F168003B6983F8A320584800F0BCF8F860FB68B6
:10F178004FEA1343DAB2FB68DBB282EA0303DAB27E
:10F188003B6983F8A2203B694FF0000283F8A12075
:10F198003B694FF0010283F821223B6940F2BB1220
:10F1A800A3F844224FF00003FB750AE0FB7D7A6860
:10F1B800D3184FF0000283F82222FB7D03F10103EC
:10F1C800FB75FB7D212BF1D93B6903F161031846DF
:10F1D8003E494FF01C02F2F7D9FA3B6903F181036B
:10F1E80018463B494FF00C02F2F7D0FA3B6903F19D
:10F1F800E103184637494FF01B02F2F7C7FA3B699B
:10F2080003F5907303F10103184633494FF00602E2
:10F21800F2F7BCFA3B6903F5B07303F10103184632
:10F228002E494FF01702F2F7B1FA3B6903F5D07394
:10F2380003F1010318462A494FF01302F2F7A6FA20
:10F248003B6903F5F07303F10103184622494FF0B7
:10F258000602F2F79BFA3B6903F138031846144992
:10F268004FF02902F2F792FA3B6903F13803184686
:10F278004FF0000140F222224FF0000300F0ACFAF8
:10F288003B694FF0000283F821223B6903F51673AE
:10F2980003F102033A6902F138021846114640F2B6
:10F2A8002222F2F773FA07F11807BD4680BD00BFA6
:10F2B8008CFC02089602A8C00B02A8C0DEDE43D070
:10F2C800107AFF1F147AFF1F187AFF1FB8FC020874
:10F2D800D4FC0208E0FC0208FCFC020804FD020859
:10F2E8001CFD020880B485B000AF78607B681B689D
:10F2F800FB60FB68184607F11407BD4680BC7047E1
:10F3080080B584B000AF78607B68FB6003F048FD8F
:10F31800FB6893F8B03903F00103DBB2002B04D08B
:10F32800504B4FF400425A831BE0FB6893F8B03906
:10F3380003F01003DBB2002B0FD04A4B5B6903F4D8
:10F348000043002B04D1474B4FF400421A8308E0D6
:10F35800444B4FF400425A8303E0424B4FF40042BF
:10F368001A83FB6893F8B03903F00203DBB2002B71
:10F3780004D03D4B4FF010025A831BE0FB6893F812
:10F38800B03903F02003DBB2002B0FD0364B5B699A
:10F3980003F01003002B04D1334B4FF010021A83F3
:10F3A80008E0314B4FF010025A8303E02E4B4FF028
:10F3B80010021A83FB6893F8B03903F00403DBB238
:10F3C800002B04D0274B4FF400625A831BE0FB68E4
:10F3D80093F8B03903F04003DBB2002B0FD0214B78
:10F3E8005B6903F40063002B04D11E4B4FF40062E9
:10F3F8001A8308E01B4B4FF400625A8303E0194B51
:10F408004FF400621A83FB6893F8B03903F00803DD
:10F41800DBB2002B04D0134B4FF480525A831BE00D
:10F42800FB6893F8B03923F07F03DBB2002B0FD0D1
:10F438000C4B5B6903F48053002B04D1094B4FF448
:10F4480080521A8308E0074B4FF480525A8303E036
:10F45800044B4FF480521A834FF0FA001FF070FBF0
:10F4680054E700BF000002400004024080B485B0A9
:10F4780000AF786039604FF00003FB604FF0000385
:10F48800BB600AE0BB687A68D3181B78FA68D3189F
:10F49800FB60BB6803F10103BB60BA683B689A4232
:10F4A800F0DBFB68184607F11407BD4680BC7047BF
:10F4B80080B588B000AF4FF003004FF0010103F0B2
:10F4C80029FA4FF480504FF0010103F0ABFA4FF0E6
:10F4D80060037B604FF002033B724FF00003BB7286
:10F4E8004FF00103FB724FF000037B7207F1040336
:10F4F8003D48194603F03AF83B484FF005014FF0F4
:10F50800050203F0F3F838484FF006014FF0050202
:10F5180003F0ECF84FF020037B6007F10403334855
:10F52800194603F023F831484FF005014FF0050262
:10F5380003F0DCF844F204037B604FF00003BB7275
:10F548004FF00003FB724FF001033B724FF00303CF
:10F558007B7207F104032548194603F007F84FF4B6
:10F5680000437B604FF00003BB724FF00103FB7256
:10F5780007F104031D48194602F0F8FF4FF0000395
:10F58800BB814FF48273FB814FF000033B824FF045
:10F5980002037B824FF00103BB824FF40073FB82AE
:10F5A8004FF008033B834FF000037B834FF00703C2
:10F5B800BB8307F10C030E48194603F019FB0C48EE
:10F5C8004FF0010103F060FB084B4FF004021A836F
:10F5D800064B4FF480421A83044B4FF400425A837F
:10F5E80007F12007BD4680BD00000240000402402C
:10F5F8000030014080B584B000AF78600B46FB70E6
:10F608004FF00003BB81374B4FF400421A83FB785D
:10F61800184600F041FAFB78184600F093FAFB7898
:10F62800012B04D14FF0D80000F00CFA03E04FF0A2
:10F63800020000F007FAFB78002B28D17B684FEA1C
:10F6480013439BB24FEA8313BB81BB894FEA132351
:10F658009BB2DBB2184600F0F5F9BB89DBB218465D
:10F6680000F0F0F94FF04003FB7303E04FF0FF00A8
:10F6780000F0E8F9FB7B002B0CBF00230123DBB271
:10F68800FA7B02F1FF32FA73002BEFD119E0FB7815
:10F69800012B08D17B6803F47F034FEA1343DBB2E5
:10F6A800184600F0CFF97B6803F47F434FEA132331
:10F6B800DBB2184600F0C6F97B68DBB2184600F0EA
:10F6C800C1F9FB78184600F021FAFB78184600F0DB
:10F6D800F9F9044B4FF400425A8307F11007BD466D
:10F6E80080BD00BF0004024080B582B000AF034671
:10F6F800FB71104B4FF400421A83FB79184600F057
:10F70800CBF9FB79184600F01DFA4FF0C70000F05E
:10F7180099F9FB79184600F0F9F9FB79184600F0D9
:10F72800D1F9044B4FF400425A8307F10807BD464C
:10F7380080BD00BF0004024080B584B000AFF8600F
:10F74800B960FA807B717B79184600F0A5F97B795E
:10F75800184600F0F7F94FF0020000F073F97B79D2
:10F76800012B08D1BB6803F47F034FEA1343DBB2D4
:10F77800184600F067F9BB6803F47F434FEA132388
:10F78800DBB2184600F05EF9BB68DBB2184600F041
:10F7980059F908E0FB681B78184600F053F9FB6834
:10F7A80003F10103FB60FB88002B0CBF002301233E
:10F7B800DBB2FA8802F1FF32FA80002BEAD17B79BA
:10F7C800184600F0A3F97B79184600F07BF907F199
:10F7D8001007BD4680BD00BF80B586B000AFF86099
:10F7E800B960FA807B714FF00003FB754FF000039E
:10F7F800FB744FF00003BB744FF000037B744FF0B1
:10F8080000033B747B79002B03D14FF04003BB828C
:10F8180002E04FF48073BB82644B4FF400421A83BA
:10F82800BA8ABB68B3FBF2F102FB01F29B1ABB7404
:10F83800BB8ADAB2BB7CD31A7B74FA88BB8AB2FB68
:10F84800F3F39BB2FB75FB88BA8AB3FBF2F102FBB8
:10F8580001F29B1A9BB2FB74BB7C002B2DD1FB7D64
:10F86800002B15D1FA887B79F868B968FFF764FF2F
:10F8780094E0BA8A7B79F868B968FFF75DFFBB8ABC
:10F88800BA68D318BB60BB8AFA68D318FB6000E07B
:10F8980000BFFB7D002B0CBF00230123DBB2FA7DE8
:10F8A80002F1FF32FA75002BE3D1FB7C9AB27B7927
:10F8B800F868B968FFF740FF70E0FB7D002B25D1A1
:10F8C800FA7C7B7C9A421AD9FA7C7B7CD31A3B74EB
:10F8D8007B7C9AB27B79F868B968FFF72DFF7B7C4F
:10F8E800BA68D318BB607B7CFA68D318FB603B7C92
:10F8F8009AB27B79F868B968FFF71EFF4EE0FA887C
:10F908007B79F868B968FFF717FF47E07B7C9BB203
:10F91800FA88D31AFB80FA88BB8AB2FBF3F39BB24E
:10F92800FB75FB88BA8AB3FBF2F102FB01F29B1A62
:10F938009BB2FB747B7C9AB27B79F868B968FFF755
:10F94800FBFE7B7CBA68D318BB607B7CFA68D31853
:10F95800FB600DE0BA8A7B79F868B968FFF7ECFEBE
:10F96800BB8ABA68D318BB60BB8AFA68D318FB6035
:10F97800FB7D002B0CBF00230123DBB2FA7D02F1D3
:10F98800FF32FA75002BE5D1FB7C002B06D0FB7CFF
:10F998009AB27B79F868B968FFF7CEFE034B4FF44B
:10F9A80000425A8307F11807BD4680BD0004024093
:10F9B80080B584B000AFF860B960FA807B717B795C
:10F9C800184600F0BFF84FF0030000F03BF87B79D1
:10F9D800012B08D1BB6803F47F034FEA1343DBB262
:10F9E800184600F02FF8BB6803F47F434FEA13234F
:10F9F800DBB2184600F026F8BB68DBB2184600F008
:10FA080021F80BE04FF0A50000F01CF803461A4659
:10FA1800FB681A70FB6803F10103FB60FB88002B8D
:10FA28000CBF00230123DBB2FA8802F1FF32FA800F
:10FA3800002BE7D17B79184600F068F807F110072A
:10FA4800BD4680BD80B582B000AF0346FB7100BFE4
:10FA580010484FF0020103F053F90346002BF7D08A
:10FA6800FB799BB20B48194603F03CF900BF0948E3
:10FA78004FF0010103F044F90346002BF7D0054885
:10FA880003F022F90346DBB2184607F10807BD4622
:10FA980080BD00BF0030014080B582B000AF034692
:10FAA800FB71FB79184600F04DF84FF00600FFF7A0
:10FAB800C9FFFB79184600F029F807F10807BD4689
:10FAC80080BD00BF80B584B000AF0346FB714FF026
:10FAD8000003FB73FB79184600F034F84FF005007B
:10FAE800FFF7B0FF4FF0A500FFF7ACFF0346FB732D
:10FAF800FB7B03F00103DBB2002BF3D1FB79184643
:10FB080000F004F807F11007BD4680BD80B483B04B
:10FB180000AF0346FB71FB79002B02D0012B05D007
:10FB280009E0074B4FF004021A8304E0044B4FF43A
:10FB380080421A8300BF07F10C07BD4680BC70479E
:10FB48000004024080B483B000AF0346FB71FB7928
:10FB5800002B02D0012B05D009E0074B4FF004021F
:10FB68005A8304E0044B4FF480425A8300BF07F1E4
:10FB78000C07BD4680BC70470004024080B582B0C7
:10FB880000AF786078684FF000014FF05002F1F74D
:10FB9800FFFE7B684FF000021A7307F10807BD46A5
:10FBA80080BD00BF80B582B000AF4FF00000FFF706
:10FBB8002BFA78607B68DAB20C4B9A707B684FEA54
:10FBC8002323DAB2094BDA707B684FEA2343DAB2AF
:10FBD800064B1A717B684FEA2363DAB2034B5A71FA
:10FBE800024B184607F10807BD4680BD00000020FB
:10FBF80080B582B000AF4FF00000FFF705FA7860DB
:10FC08007B68DAB20C4B9A707B684FEA2323DAB22E
:10FC1800094BDA707B684FEA2343DAB2064B1A7154
:10FC28007B684FEA2363DAB2034B5A71024B1846DA
:10FC380007F10807BD4680BD0800002080B582B0E6
:10FC480000AF4FF00000FFF7DFF978607B68DAB2A9
:10FC58000C4B9A707B684FEA2323DAB2094BDA70AF
:10FC68007B684FEA2343DAB2064B1A717B684FEA86
:10FC78002363DAB2034B5A71024B184607F108079F
:10FC8800BD4680BD1000002080B487B000AFF8608A
:10FC9800B9607A604FF000037B617B68012B40F20A
:10FCA800C180BB681B7803F07F03002B04D0FB687E
:10FCB8004FF001021A7103E0FB684FF000021A715D
:10FCC800BB681B78FB74FB7C03F07F03FB74BB6889
:10FCD8001B7803F07F030A2B42D801A252F823F0C5
:10FCE80015FD00081FFD000829FD000869FD000832
:10FCF80069FD000869FD000869FD000869FD000844
:10FD080033FD000845FD000857FD0008FB684FF06B
:10FD180000029A7124E0FB684FF001029A711FE01B
:10FD2800FB684FF002029A711AE0FB684FF0080274
:10FD38009A71FB684FF002025A7174E0FB684FF049
:10FD480009029A71FB684FF000021A7308E0FB6819
:10FD58004FF00A029A71FB684FF000021A7300BF55
:10FD6800BB6803F101031B787D2B16D8BB6803F130
:10FD780001031B78002B10D0BB6803F101031B782B
:10FD88001A46FB681A60BB6803F10202FB689A60B6
:10FD9800FB684FF002025A7345E0BB6803F10103A8
:10FDA8001B787E2B22D1BB6803F102031B784FEA34
:10FDB80003234FEA03434FEA13437A6942EA0303F2
:10FDC8007B61BB6803F103031B781A467B6942EA2F
:10FDD80003031A46FB681A60BB6803F10402FB6858
:10FDE8009A60FB684FF004025A731CE0BB6803F189
:10FDF80001031B787F2B0CD1FB684FF000021A60BF
:10FE0800FB684FF003025A71FB684FF008025A73FF
:10FE180009E0FB684FF000021A60FB684FF002022D
:10FE28005A7300E000BF07F11C07BD4680BC70474D
:10FE380080B588B000AFF860B9607A60FB704FF0A9
:10FE48000003FB611CE04FF00000FFF7DDF80346FC
:10FE5800BB61BB69DAB207F11001FB69CB181A70F4
:10FE6800FB6903F10103BA694FEA1222D2B207F122
:10FE78002000C31803F8102CFB6903F10103FB6190
:10FE8800FB69012BDFD9BB681B7843F00103DAB2A9
:10FE9800BB681A707B687D2B51D84FF00203FB7545
:10FEA800BB681B7863F07F03DAB2BB681A70BB6863
:10FEB80003F101037A68D2B262F07F02D2B21A70FB
:10FEC800FB7DFB610FE0BA68FB69D318FA7DF9691D
:10FED8008A1A07F120018A1812F8102C1A70FB6987
:10FEE80003F10103FB61FB7D03F104031A46FB697F
:10FEF8009A42E8D84FF00003FB6118E0FB6903F170
:10FF08000603BA68D318F968FA698A181178FA6981
:10FF180002F0030207F12000821812F8102C81EA7F
:10FF28000202D2B21A70FB6903F10103FB61FA699C
:10FF38007B689A42E2D37B6803F106036DE07B6835
:10FF48007E2B61D97A684FF6FF739A425CD84FF0DE
:10FF58000403FB75BB681B7863F07F03DAB2BB68E8
:10FF68001A70BB6803F101034FF0FE021A70BB68F8
:10FF780003F102037A684FEA1222D2B21A70BB6800
:10FF880003F103037A68D2B21A70FB7DFB610FE0BC
:10FF9800BA68FB69D318FA7DF9698A1A07F1200152
:10FFA8008A1812F8102C1A70FB6903F10103FB611F
:10FFB800FB7D03F104031A46FB699A42E8D84FF027
:10FFC8000003FB6118E0FB6903F10803BA68D31862
:10FFD800F968FA698A181178FA6902F0030207F1D8
:10FFE8002000821812F8102C81EA0202D2B21A708C
:08FFF800FB6903F10103FB6149
:020000040801F1
:10000000FA697B689A42E2D37B6803F1080308E04F
:100010007A684FF6FF739A4202D94FF0000300E06E
:10002000FFE7184607F12007BD4680BD80B584B0C4
:1000300000AF786039607B6818464FF03A01F2F7FC
:1000400099F90346FB60FB68002B08D0FA687B68CF
:10005000D31A386879681A46F1F79CFB09E07B6887
:100060001846F2F759FB0346386879681A46F1F7E3
:1000700091FB07F11007BD4680BD00BF80B584B07D
:1000800000AF78607B6818464FF03A01F2F772F9DA
:100090000346FB60FB68002B09D0FB6803F10103FA
:1000A000FB60FB681846F0F729FC034601E040F2CC
:1000B000BB13184607F11007BD4680BD80B5ADF5EE
:1000C000087D00AF07F10C03186007F10803196001
:1000D00007F104031A6007F108031B68C7F81C3214
:1000E00007F118034FF01E021A6007F114034FF4D2
:1000F00080721A604FF00000FEF78AFF024607F197
:100100001C031A604FF00000FEF782FF024607F161
:100110001C035A604FF00000FEF77AFF024607F119
:100120001C039A604FF00000FEF772FF024607F1D1
:100130001C03DA6007F5FA7107F11C0307F11802D6
:10014000084611461A464FF0100311F089F807F1DE
:10015000F40318464FF000014FF48072F1F71CFCD5
:1001600007F1900318464FF000014FF06402F1F7D9
:1001700013FC07F12C0318464FF000014FF0640206
:10018000F1F70AFC07F104031B6803F5087303F198
:10019000020307F1F402104619464FF02002F1F76E
:1001A000F9FA07F104031B6803F5607202F1030218
:1001B00007F104031B6803F5886303F10403D7F810
:1001C0001C028849F0F722F80346D7F81C22D318FE
:1001D000C7F81C32D7F81C0283494FF02C02F1F704
:1001E000D9FAD7F81C3203F12B03C7F81C3207F1F8
:1001F00004031B6803F5407303F1030307F12C02AA
:1002000018461146FFF712FF07F12C03D7F81C021E
:1002100076491A46EFF7FAFF0346D7F81C22D3189F
:10022000C7F81C32D7F81C0271494FF03D02F1F7B4
:10023000B1FAD7F81C3203F13C03C7F81C3207F5BA
:10024000FA73D7F81C021946F2F708FA07F5FA73A1
:100250001846F2F761FA0346D7F81C22D318C7F8FC
:100260001C32D7F81C0263494FF00302F1F792FAEF
:10027000D7F81C3203F10203C7F81C3207F104035C
:100280001B6803F5707303F10303D7F81C025A4986
:100290001A46EFF7BBFF0346D7F81C22D318C7F85E
:1002A0001C32D7F81C0255494FF00D02EFF7AEFF94
:1002B0000346D7F81C22D318C7F81C32D7F81C0203
:1002C0004F49504AEFF7A2FF0346D7F81C22D31834
:1002D000C7F81C3207F1F40318464FF000014FF441
:1002E0008072F1F759FB07F104031B6803F52073D3
:1002F00003F1030318464FF0200100F08BF8C7F814
:10030000180207F104031B6803F5207303F10303CC
:10031000D7F8182207F1F40108461946F1F73AFA1E
:10032000D7F8183207F1F402D318184636494FF0BF
:100330000202F1F72FFA07F104031B6803F5287393
:1003400003F1030318464FF0200100F063F8C7F8EB
:100350001402D7F8183203F1020307F1F402D1189E
:1003600007F104031B6803F5287303F10303D7F8AF
:10037000142208461946F1F70DFA07F1900007F12B
:10038000F402D7F81812D7F81432CB1803F102038D
:1003900007F1140110F064FF07F19003D7F81C0275
:1003A0001A491A46EFF732FF0346D7F81C22D31832
:1003B000C7F81C32D7F81C0215494FF00502F1F7B7
:1003C000E9F9D7F81C3203F10403C7F81C3207F12E
:1003D00008031868F2F7A0F90346184607F50877EE
:1003E000BD4680BDC8FD0208E0FD02080CFE020803
:1003F00018FE020858FE02085CFE02086CFE0208A5
:1004000088FE02088CFE0208A4FE0208A8FE02086C
:10041000ACFE020880B485B000AF786039604FF060
:100420000003FB6013E0FB687A68D3181B78002B8D
:1004300009D1FB6803F101037A68D3181B78002BFC
:1004400001D1FB6808E0FB6803F10203FB60FA6876
:100450003B689A42E7DB3B68184607F11407BD4644
:1004600080BC704780B584B000AF78603960386870
:1004700020494FF00D02F2F77FF90346002B04D01C
:100480007B684FF002025A712FE038681A49F2F780
:100490007BFB0346FB60FB68002B04D17B684FF0BD
:1004A00002025A7121E0FB6803F11603FB60FB684E
:1004B00018461249F2F768FB0346BB60BB68002B85
:1004C00004D17B684FF002025A710EE07B6803F1A1
:1004D0003202B968FB68CB1A1046F9681A46F1F780
:1004E00059F97B684FF001025A7107F11007BD46B8
:1004F00080BD00BFB4FE0208C4FE020858FE020818
:1005000080B400AFBFF34F8FBD4680BC704700BFC3
:1005100080B500AF054A054BDB6803F4E061044B8E
:1005200041EA0303D360FFF7EBFFFEE700ED00E0D5
:100530000400FA0580B594B000AF786039603B687C
:100540007B644FF00003BB644FF001033B76786897
:1005500002F08EFDF864FB6C002B00F0E3807B68FA
:100560001B7A002B40F0D38007F13C0207F13A03DD
:10057000F86C11461A4604F07BF8FB6B184670497C
:100580004FF00502F2F7F8F80346002B2DD1FB6B74
:1005900018466C494FF00F02F2F7EEF80346002BB5
:1005A00003D1786800F030F9BCE0FB6B03F1050281
:1005B00007F10803786811461A4600F059FB034614
:1005C00087F8433097F84330002B00F0A28097F86B
:1005D0004330012B40F09F805B4A07F108037868A5
:1005E00011461A4600F044FB9CE0FB6B1846574945
:1005F0004FF00602F2F7C0F80346002B40F08D8062
:10060000FB6B03F10503184651494FF01602F2F750
:10061000B3F80346002B06D17B6C03F138037868EE
:10062000194600F0E9FBFB6B03F105031846494945
:100630004FF01602F2F7A0F80346002B1AD1FB6B1D
:1006400003F11B017B6C03F138027B8FA3F11B03C9
:100650009BB2786800F044FD7B6C03F5167303F1E0
:1006600002037A6C02F138021846114640F2222247
:10067000F1F790F8FB6B03F10503184636494FF08C
:100680001802F2F779F80346002B04D1786802F0DB
:1006900023FEFFF73DFFFB6B03F1050318462F49CF
:1006A0004FF00B02F2F768F80346002B37D12C4AC3
:1006B00007F10803786811461A4600F0D9FA7B8FD3
:1006C000BA6CD318BB64786802F0D2FCF864FB6C97
:1006D000002B26D007F13C0207F13A03F86C1146D3
:1006E0001A4603F0C5FFF86C03F062FF7B8FBA6C0B
:1006F000D318BB647B681B7A002BE4D0184A07F13F
:100700000803786811461A4600F0B2FA0AE000BF02
:1007100008E000BF06E000BF04E000BF02E000BF49
:1007200000E000BF786802F0D7FD034687F842304A
:10073000F86C03F01DFF07F15007BD4680BD00BFF8
:100740004803030850030308600303086C0303080D
:10075000740303088C030308A4030308C0030308FD
:10076000CC03030880B586B000AF78607B687B61FE
:100770004FF010004FF000014FF0000202F02CFB90
:1007800038613B69002B1ED038694FF000014FF0F3
:10079000500202F0B1FB0346FB7397F90F30002BB8
:1007A00011D138694FF0FF0102F00CFC386902F0FA
:1007B00029FCB8607B68B8681946FFF7BBFEB868CB
:1007C00002F042FBF2E74FF4FA701EF0BDF9CFE7FA
:1007D00080B586B002AF78607B68FB604FF00103A4
:1007E0000093074807497A684FF440730EF080FD84
:1007F0000246FB68C3F84C2A07F11007BD4680BDCE
:10080000D80303086507010890B5ADF5617D02AF17
:1008100007F10403186007F10C034FF000021A609F
:1008200003F104034FF000021A6003F104034FF0D8
:1008300000021A6003F104034FF000021A6003F192
:1008400004034FF000021A6003F104034FF00002AA
:100850001A6003F104034FF000021A7003F1010360
:1008600007F1280318464FF000014FF45272F1F7D8
:1008700093F8934B1B6803F10102914B1A60904B64
:100880001B6807F10C0210468E491A46EFF7BEFCB2
:1008900007F1280207F10C0310461946F1F746FD4F
:1008A00007F128031846F1F737FF034607F128023E
:1008B000D318184684494FF03402F0F76BFF07F164
:1008C00028031846F1F728FF034607F12802D3183A
:1008D00018467E494FF03602F0F75CFF07F1280317
:1008E0001846F1F719FF034607F12802D3181846F6
:1008F0001EF036FA07F128031846F1F70DFF0346FC
:1009000007F12802D318184671494FF03602F0F764
:1009100041FF07F128031846F1F7FEFE034607F1F1
:100920002802D31818466B494FF03B02F0F732FF0C
:1009300007F128031846F1F7EFFE034607F12802F6
:10094000D318184664494FF00F02F0F723FF07F160
:10095000040107F55D7207F55C7303F10203086893
:1009600011461A464FF0010302F092FAD7F8743399
:10097000DBB21A46D7F874334FEA1323DBB2D7F849
:1009800074134FEA1141C9B20C46D7F874134FEAF9
:100990001161C9B2084607F10C01009401900846A4
:1009A0004E49EFF733FC07F1280207F10C0310461C
:1009B0001946F1F7BBFC4A4B1B6893F87D34052BB5
:1009C0005ED801A252F823F0E1090108810A01086A
:1009D000010A0108610A0108210A0108410A010807
:1009E00007F128031846F1F797FE034607F128029E
:1009F000D31818463B494FF01802F0F7CBFE3FE002
:100A000007F128031846F1F787FE034607F128028D
:100A1000D318184634494FF01202F0F7BBFE2FE00E
:100A200007F128031846F1F777FE034607F128027D
:100A3000D31818462D494FF01602F0F7ABFE1FE011
:100A400007F128031846F1F767FE034607F128026D
:100A5000D318184626494FF01D02F0F79BFE0FE011
:100A600007F128031846F1F757FE034607F128025D
:100A7000D31818461F494FF01702F0F78BFE00BF3E
:100A800007F1040318681C4940F26C424FF0000360
:100A900002F0F4FB07F128031846F1F73DFE034688
:100AA00007F1040107F12802086811461A464FF0C1
:100AB000000302F0E3FB07F55F77BD4690BD00BF82
:100AC000A8060020DC030308E0030308140403085D
:100AD0004C04030884040308C0040308D00403087A
:100AE000E0320020E0040308F80403080C050308C2
:100AF0002405030844050308DCFE020880B584B021
:100B000000AF78607B68FB60FB681868FB689968D9
:100B1000FB689A88FB681B7CFEF74EFF07F1100705
:100B2000BD4680BD80B58EB000AF786039603B684F
:100B3000FB624FF000033B6307F10C0318464FF0D4
:100B400000014FF01E02F0F727FF83E04FF0000393
:100B500087F837307AE097F8373007F10C02D2186F
:100B6000FB6A1B7C1046396B4FF00102FEF724FF35
:100B700097F8373007F13802D31813F82C3C202BA4
:100B800008D097F8373007F13802D31813F82C3C07
:100B90000A2B43D1796807F10C0297F837300846E1
:100BA00011461A46F1F7E8FD0346002B2DD1FB6AEA
:100BB00003F1080319463B6B03F10102FB6A1B7C3E
:100BC000084611464FF00402FEF7F6FEFB6A03F1F9
:100BD0000C0319463B6B03F10502FB6A1B7C0846BC
:100BE00011464FF00402FEF7E7FEFB6A03F1110223
:100BF00097F83730104679681A46F0F7CBFDFB6A54
:100C000097F8372083F82F202EE03B6B03F10E037B
:100C10003B634FF0000387F837301BE097F837301D
:100C200007F13802D31813F82C3CFF2B04D1FB6AD0
:100C30004FF00002DA6017E03B6B03F101033B6306
:100C400097F8373003F1010387F8373097F83730DA
:100C50001D2B80D93A6B4FF6FF739A427FF676AF21
:100C6000FB6A4FF00002DA6007F13807BD4680BD2D
:100C700080B5ADF5BA6D00AF07F11003A3F1040321
:100C8000186007F10803196007F11003A3F10C03C2
:100C90001A6007F11003A3F10C031B68C7F8CC35E9
:100CA00007F12003A3F10C03D7F8CC25136007F15B
:100CB00008031868D7F8CC15FFF734FFD7F8CC3500
:100CC00040F2B4529A80D7F8CC35DB68002B00F0A4
:100CD00088807FE0D7F8CC35DA6840F2B3539A4287
:100CE0003CD907F11003A3F104031B681B7A002B06
:100CF00031D1D7F8CC05FFF701FFD7F8CC351A680A
:100D000007F11003A3F104031868114640F2B4522E
:100D10004FF0010302F0B2FA034687F8CB3597F99A
:100D2000CB35002B14D1D7F8CC359A68D7F8CC3511
:100D30009B88D218D7F8CC359A60D7F8CC35DA68CA
:100D4000D7F8CC359B88D21AD7F8CC35DA6041E099
:100D50004FF002034AE04FF0030347E007F11003AE
:100D6000A3F104031B681B7A002B30D1D7F8CC35D4
:100D7000DB689AB2D7F8CC359A80D7F8CC05FFF764
:100D8000BDFED7F8CC351968D7F8CC35DB689BB2F7
:100D90001A4607F11003A3F1040318684FF001038A
:100DA00002F06CFA034687F8CB3597F9CB35002B68
:100DB0000AD1D7F8CC354FF000029A60D7F8CC357D
:100DC0004FF00002DA6005E04FF002030EE04FF052
:100DD00003030BE0D7F8CC35DB68002B7FF47AAF48
:100DE00002E04FF0010301E04FF00003184607F561
:100DF000BA67BD4680BD00BF2DE9F04FADF5537D0C
:100E00001EAF07F15C03186007F15803196007F182
:100E100058031B68C7F8CC3207F1640318464FF03B
:100E200000014FF40072F0F7B7FD07F5197318468B
:100E30004FF000014FF06402F0F7AEFD07F16403DC
:100E40007B65D7F8CC32D3F80E32DBB23B65D7F8EE
:100E5000CC32D3F80E324FEA1323DBB2FB64D7F85F
:100E6000CC32D3F80E324FEA1343DBB2BB64D7F86F
:100E7000CC32D3F80E324FEA1363DBB27B64D7F87F
:100E8000CC32D3F81232DBB23B64D7F8CC32D3F891
:100E900012324FEA1323DBB2FB63D7F8CC32D3F81C
:100EA00012324FEA1343DBB2BB63D7F8CC32D3F82C
:100EB00012324FEA1363DBB27B63D7F8CC32D3F83C
:100EC0001632DBB23B63D7F8CC32D3F816324FEA96
:100ED0001323DBB2FB62D7F8CC32D3F816324FEAD9
:100EE0001343DBB2BB62D7F8CC32D3F816324FEAE9
:100EF0001363DBB27B62D7F8CC32D3F81A32DBB2A1
:100F00003B62D7F8CC32D3F81A324FEA1323DBB264
:100F1000FB61D7F8CC32D3F81A324FEA1343DBB275
:100F2000BB61D7F8CC32D3F81A324FEA1363DBB285
:100F30007B61D7F8CC32D3F81E32DBB23B61D7F8F5
:100F4000CC32D3F81E324FEA1323DBB2FB60D7F862
:100F5000CC32D3F81E324FEA1343DBB2BB60D7F872
:100F6000CC32D3F81E324FEA1363DBB29B46D7F87C
:100F7000CC3203F1A90AD7F8CC3203F1E909D7F84A
:100F8000CC3203F5947606F10106D7F8CC3203F59E
:100F9000B47404F10104D7F8CC3293F86930984660
:100FA000D7F8CC3293F86A309C46D7F8CC3293F815
:100FB0006B309E46D7F8CC3293F86C301D46D7F88C
:100FC000CC3293F86D301846D7F8CC3293F86E30A7
:100FD0001946D7F8CC3203F5F572D7F8CC327B60DE
:100FE000BB6C00937B6C01933B6C0293FB6B039394
:100FF000BB6B04937B6B05933B6B0693FB6A079378
:10100000BB6A08937B6A09933B6A0A93FB690B935B
:10101000BB690C937B690D933B690E93FB680F933F
:10102000BB681093CDF844B0CDF848A0CDF84C90F3
:1010300014961594CDF85880CDF85CC0CDF860E0DA
:1010400019951A901B911C927B681D93786D21490C
:101050003A6DFB6CEFF7DAF8C7F8C802D7F8CC3274
:1010600093F8E931002B0FD007F1640407F1640312
:101070001846F1F751FB0346E318184616494FF09E
:101080000202F0F787FB0EE007F1640407F1640346
:101090001846F1F741FB0346E31818460F494FF095
:1010A0000202F0F777FB07F164031846F1F734FB0F
:1010B000034607F15C0107F16402086811461A460D
:1010C0004FF0010302F0DAF807F53577BD46BDE8C9
:1010D000F08F00BF5C050308C0050308C4050308C2
:1010E00090B5C9B000AF07F10C04206007F108000B
:1010F000016007F104010A601A4607F102031A8031
:1011000007F104031B68C7F8103107F108031B68D7
:10111000C7F8183107F102031B88A7F81631D7F872
:10112000103103F1A90318464FF000014FF04002BF
:10113000F0F732FCD7F8103103F1E90318464FF00D
:1011400000014FF04002F0F727FCD7F8103103F50B
:10115000947303F1010318464FF000014FF0400271
:10116000F0F71AFCD7F8103103F5B47303F101035B
:1011700018464FF000014FF04002F0F70DFC4FF021
:10118000000387F81F3124E097F81F41D7F81801B2
:10119000EFF7B4FB0346DAB207F110031A55D7F89C
:1011A000183118464FF02401F1F7E4F80346C7F868
:1011B0001831D7F81831002B10D0D7F8183103F1B7
:1011C0000103C7F8183197F81F3103F1010387F8BD
:1011D0001F3197F81F31132BD6D900E000BFD7F885
:1011E000103103F5027303F1060307F110021846EC
:1011F00011464FF01402F0F7CDFA0FE0B7F81631B0
:10120000D7F81821D3181B78242B07D1B7F816313B
:10121000D7F81821D3184FF000021A70B7F816311A
:10122000002B0CBF00230123DBB2B7F8162102F11B
:10123000FF32A7F81621002BE0D1D7F8103103F1C7
:10124000A904D7F818311846F1F766FA0346204684
:10125000D7F818111A46F0F79DFAD7F81831184642
:10126000F1F75AFA034603F10103D7F81821D3180E
:10127000C7F81831D7F8103103F1E904D7F818315D
:101280001846F1F749FA03462046D7F818111A46CE
:10129000F0F780FAD7F818311846F1F73DFA03460F
:1012A00003F10103D7F81821D318C7F81831D7F87C
:1012B000103103F5947404F10104D7F8183118467D
:1012C000F1F72AFA03462046D7F818111A46F0F724
:1012D00061FAD7F818311846F1F71EFA034603F100
:1012E0000103D7F81821D318C7F81831D7F81031EF
:1012F00003F5B47404F10104D7F818311846F1F776
:101300000BFA03462046D7F818111A46F0F742FAAE
:10131000D7F818311846F1F7FFF9034603F1010336
:10132000D7F81821D318C7F81831D7F818311B7817
:10133000312B06D1D7F810314FF0010283F8E921A3
:1013400005E0D7F810314FF0000283F8E921D7F813
:10135000103118464FF0000140F222224FF00003F6
:10136000FEF73EFA07F10C031868D7F81011FFF7E3
:1013700043FD07F59277BD4690BD00BF80B5CAB06A
:1013800000AF07F10403186007F10403186801F0C7
:101390006FFEC7F82401D7F82431002B00F0E3805A
:1013A00007F104031B681B7A002B40F0DC8007F573
:1013B000907207F58F73D7F8240111461A4603F08F
:1013C00057F9B7F81E31B3F5887F40F0BD80D7F8E4
:1013D000203107F10C02104619464FF48872F0F7DD
:1013E000D9F9D7F8240103F0C3F807F10C03184624
:1013F00067494FF00402F1F7BFF90346002B0AD109
:1014000007F10403186863494FF00A024FF0010323
:1014100001F034FFA3E007F10C0318465E494FF0DA
:101420000402F1F7A9F90346002B1BD107F10C03C5
:10143000596807F10C035B891AB207F10C031B7A98
:101440005BB207F10C0000F10D00FEF7C9F907F1DE
:101450000403186851494FF004024FF0010301F0F2
:101460000DFF7CE007F10C0318464D494FF00402D4
:10147000F1F782F90346002B1DD107F10C035A68DE
:1014800007F10C031B7A5BB207F10C0101F10D01AE
:10149000084611464FF48072FEF78EFA07F10402F7
:1014A00007F10C03106819464FF488724FF00103DE
:1014B00001F0E4FE53E007F10C03184639494FF000
:1014C0000402F1F759F90346002B15D107F10C037B
:1014D0005A6807F10C031B7A5BB210461946FEF7F7
:1014E0008DF807F1040318682F494FF00A024FF0F6
:1014F000010301F0C3FE32E007F10C0318462B494B
:101500004FF00402F1F738F90346002B11D107F12F
:101510000C031B7A5BB21846FEF7EAF807F10403E6
:10152000186823494FF016024FF0010301F0A6FEA0
:1015300015E007F1040318681E494FF00A024FF046
:10154000010301F09BFE0AE007F1040318681A4941
:101550004FF00C024FF0010301F090FE0AE04FF053
:1015600005001DF0F1FA07F104031B681B7A002B3C
:101570003FF40AAF07F10403186801F0ADFED7F895
:10158000240102F0F5FF07F59477BD4680BD00BF4A
:10159000C8050308D0050308DC050308E4050308B3
:1015A000EC050308F4050308FC0503080806030816
:1015B00010060308280603083406030880B586B021
:1015C00000AF78607B687B614FF010004FF0000146
:1015D0004FF0000201F000FC38613B69002B1CD089
:1015E00038694FF000014FF0040201F085FC03461A
:1015F000FB7397F90F30002B0FD138694FF0FF01C3
:1016000001F0E0FC386901F0FDFCB860B868FFF754
:10161000B5FEB86801F018FCF4E74FF4FA701DF05D
:1016200093FAD1E780B586B002AF78607B68FB6043
:101630004FF002030093074807497A684FF4C073DC
:101640000DF056FE0246FB68C3F8502A07F110075A
:10165000BD4680BD44060308BD15010880B400AF37
:10166000BFF34F8FBD4680BC704700BF80B500AF51
:10167000054A054BDB6803F4E061044B41EA0303D0
:10168000D360FFF7EBFFFEE700ED00E00400FA0592
:1016900090B589B004AF78604FF000004FF00001C2
:1016A00003F088FF7B68FB60FB6893F84334002BF2
:1016B0000FD1FB68FA68D2F868245A60FB68FA68B0
:1016C000D2F86C249A60FB68FA68D2F87024DA6069
:1016D0000BE0FB684FF000025A60FB684FF000021D
:1016E0009A60FB684FF00002DA60FB6803F58E63D6
:1016F00003F104034FF00000194606F001FCFB68FB
:1017000003F58F634FF00100194606F0F9FBFB6803
:1017100093F8A120FB6883F82B20FB6893F8A220A4
:10172000FB6883F82C20FB6893F8A320FB6883F800
:101730002D20FB6893F8A420FB6883F82E20FB681B
:1017400093F8A520FB6883F82F20FB6893F8A62068
:10175000FB6883F83020F868FB6803F10401FB683C
:1017600003F10802FB6803F10C034FF0000400943E
:10177000084C0194084C029407F0ACFAFB68184638
:1017800007F090FBFB68184607F09AFB07F1140777
:10179000BD4690BD25EF01085154010890B585B0B4
:1017A00000AF78607B68FB60FB6893F84334002BE4
:1017B00005D0FB684FF0000283F8302A04E0FB6894
:1017C0004FF0020283F8302AFB6893F8303A032B7B
:1017D00000F28E8001A252F823F000BFED1701083D
:1017E0001D18010867180108CB180108FB68184686
:1017F00005F060F9FB684FF0010283F8302AFA68BF
:1018000092F8B0396FF3000382F8B039FA6892F8B1
:10181000B03943F0100382F8B0396EE0FB685B68C2
:10182000002B09D0FB68184605F066FEFB684FF0F8
:10183000030283F8302A60E0324B1B78002B0AD178
:10184000FB68184605F058FEFB684FF0020283F86B
:10185000302AFFF70BFF2B4B1B7803F1FF33DAB273
:10186000284B1A7049E0F968FB6803F58D62FB6844
:1018700003F58C6303F10C03F86800F58E640846E9
:1018800011461A46234607F073FAFB68D3F8603A0C
:1018900018464FF000014FF000024FF000031CF01B
:1018A000C1FCFB684FF0030283F8302AFA6892F813
:1018B000B0396FF3000382F8B039FA6892F8B039A2
:1018C0006FF3041382F8B03917E0FA6892F8B03970
:1018D0006FF3000382F8B039FA6892F8B0396FF309
:1018E000041382F8B0394FF000001DF0DBF804E07B
:1018F0004FF47A701DF028F900BF4FF0FA001DF088
:1019000023F961E718000020002103E00A4B5B582F
:101910004350043109480A4B42189A42F6D3094A07
:1019200002E0002342F8043B074B9A42F9D3FAF74E
:1019300087FFFBF705FA7047884303080000002083
:101940009806002098060020905B0020FEE700002B
:1019500080B485B000AFF860B9607A604FF00003E2
:10196000184607F11407BD4680BC704780B485B0A7
:1019700000AFF860B9607A604FF00003184607F1D5
:101980001407BD4680BC704780B483B000AF786058
:101990004FF0FF33184607F10C07BD4680BC704777
:1019A00080B483B000AF786039604FF0FF331846E1
:1019B00007F10C07BD4680BC704700BF80B483B000
:1019C00000AF78604FF0FF33184607F10C07BD46B3
:1019D00080BC704780B483B000AF786039603B68EA
:1019E000002B07D03B684FF000021A603B684FF0B5
:1019F00000025A604FF00003184607F10C07BD467D
:101A000080BC704780B58AB000AF786039604FF015
:101A100000037B624FF000033B624FF00003FB6169
:101A20004FF00003BB617B681B8A9BB27B627B6AC1
:101A300023F440537B623B68DB887A6A42EA030303
:101A40007B627B6A9AB27B681A827B689B899BB2B5
:101A50007B627B6A23F4B05323F00C037B623B6808
:101A60009A883B681B8942EA03039AB23B685B8908
:101A700042EA03039BB27A6A42EA03037B627B6A0F
:101A80009AB27B689A817B689B8A9BB27B627B6AF5
:101A900023F440737B623B689B897A6A42EA0303C2
:101AA0007B627B6A9AB27B689A8207F108031846C8
:101AB00000F076FE7A683A4B9A4203D07A68394B46
:101AC0009A4202D17B693B6201E03B693B627B68E1
:101AD0009B899BB29BB21BB2002B0FDA3A6A13466A
:101AE0004FEA83039B184FEA83029A183B681B68EE
:101AF0004FEA4303B2FBF3F3FB610EE03A6A13468D
:101B00004FEA83039B184FEA83029A183B681B68CD
:101B10004FEA8303B2FBF3F3FB61FA69224BA3FBA9
:101B200002134FEA53134FEA03137B627B6A4FEAB7
:101B300013134FF0640202FB03F3FA69D31ABB617B
:101B40007B689B899BB29BB21BB2002B10DABB69EE
:101B50004FEAC30303F13202134BA3FB02134FEA14
:101B6000531303F007037A6A42EA03037B620FE030
:101B7000BB694FEA031303F132020B4BA3FB0213C1
:101B80004FEA531303F00F037A6A42EA03037B62BE
:101B90007B6A9AB27B681A8107F12807BD4680BD2F
:101BA00000100140001401401F85EB5180B483B048
:101BB00000AF78600B46FB70FB78002B08D07B6889
:101BC0009B899BB243F400539AB27B689A8107E0E9
:101BD0007B689B899BB223F400539AB27B689A81FD
:101BE00007F10C07BD4680BC704700BF80B483B0CE
:101BF00000AF78600B467B807B884FEAC3534FEA87
